:020000040000FA
:1000000000F80202456D000065320000E13F00008B
:1000100000000000000000000000000000000000E0
:1000200000000000D04501001846010065320000C4
:10003000000000000000000065320000A173000015
:10004000F13100006532000065320000656D00008E
:10005000E9470000ED680000F5310000E9320000DA
:100060004917000085160000653200006932000063
:10007000BD47000045850000E56C0000116D0000E3
:10008000653200006532000065320000F576000040
:10009000157700006532000065320000653200000F
:1000A000957700009F770000F3310000F96B0000A6
:1000B00065320000556900000000000000000000EB
:1000C0000348854600F09CFE0048004761C20000DE
:1000D00000F8020230B50B46014600202022012420
:1000E00009E00D46D5409D4205D31D469540491B6C
:1000F0002546954040191546521E002DF1DC30BDB5
:1001000070B500242546002801DA01244042002968
:1001100001DA01254942FFF7DDFFAC4200D0404241
:10012000002C00D0494270BD03460B439B0703D00F
:1001300009E008C9121F08C0042AFAD203E00B78AC
:100140000370401C491C521EF9D27047D2B201E024
:100150000270401C491EFBD270470022F6E710B522
:1001600013460A4604461946FFF7F0FF204610BD25
:10017000CAB2401E4178401C8A4202D00029F9D1FF
:1001800000207047421C0178401C0029FBD1801AD6
:10019000704730B504460020034600E05B1C9342E4
:1001A00003D2E05CCD5C401BF8D030BD30B50546D5
:1001B0000020034600E05B1C934205D2EC5CC85C67
:1001C000201A01D1002CF6D130BD00000FB400B5CB
:1001D0008DB009900B9010A900200091C0430A90A7
:1001E00000200C9006480690064807906A4609A829
:1001F0000F9900F06DFC0DB008BC04B0184700006A
:10020000F10A0000110B0000FFB5002083B0009040
:1002100050680190916914460026976804988847B1
:1002200005460C990698084305D009E0A169761C9B
:10023000049888470546216A284688470028F5D152
:10024000681C03D00198C00704D017E00020C04309
:1002500007B0F0BD2068011D2160006800900DE02E
:100260000198C00704D1009805700098401C0090C8
:10027000A169761C7F1E049888470546002F1CDD67
:10028000681C1AD0069800280FD0E817C00E401935
:1002900041118A0006994009511840012A1A09683B
:1002A000012090400142DBD107E00C980028D7D113
:1002B000216A284688470028D2D0E16904988847F7
:1002C0000C98002807D1002E05DD0198C00702D147
:1002D000009800210170A068B84204DD0C98002845
:1002E00004D0002F02D00120C043B1E73046AFE771
:1002F00070B5064610F0DEFC046805460A220021AF
:10030000304600F071FC2C6070BDF8B502464A40E2
:10031000D40F42004B0052085B089A4202D20246B8
:10032000084611464A0023D0C30D4A00DDB2120E22
:10033000AD1A202D35DA49020126490AF6058A1937
:10034000002C00D0524220214F1B1146B9402A41B7
:100350001018C20D9A4221D0002C17D0012D08DCB4
:10036000DA05801AD20F8019D207DBB200F07CFCCC
:10037000F8BDDA05801A012340001B06C01880185A
:100380005A428018CA0F1043490007E04908C207C3
:100390001143DA05801A80194008801800F05CFCCF
:1003A000F8BD61000122511A001BF7E70122D207B4
:1003B0005140AAE70122D2075040A6E7024670B595
:1003C0004A40D30FDB0740002DD04A002AD0010E4F
:1003D000140E000212020919400A520A8418E5019B
:1003E00004465443000A120A2E045043A419421929
:1003F000200CC543AA18120C0125AD03521C52193A
:1004000012047F39240400D0521C104301D4400050
:10041000491EC2B20C06C0092018401C4008802AA0
:1004200002D003E0002070BD40084000002900DA3F
:100430000020184370BD70B502464A40D50F4000F9
:100440004A00ED0740085208002814D0002A12D0B4
:10045000C40DD30D41020120C0055202490A520ABF
:10046000E41A091812187D34914201D3641C00E08B
:100470004900002C01DA002070BD0023914201D315
:10048000891A0343400849000028F7D100290AD0FF
:10049000914202D10121C90705E0914201D2012117
:1004A00001E00121C943E005C018401900F0D4FB68
:1004B00070BD0000F0B507460846584087B0C00F31
:1004C000049048000E46590040084908BC1A88416B
:1004D00005D2384631461E4617460B46024658009E
:1004E000400810434CD0300D039040055900400D9A
:1004F000490D0590401A0290402872DA1803012134
:10050000000B09050843019004980092002805D0CB
:1005100001995242002088410092019002984021A6
:100520000A1A0199009800F099FA05460C466B46A4
:1005300007CB00F0B4FAC0197141039A0E0D0023E5
:10054000D71756401A467A40164344D0049A002AD8
:100550002DD0029A012A039A15DC1205C01A914186
:1005600001263605001C7141D20F059ED20700936B
:10057000019202962A46234600F0BCFB07B0F0BD6C
:1005800038463146FAE71605224A0F46B218C01A15
:10059000B74101210905001C4F4100187F41114658
:1005A00018187941E20F10436D19644113E0E20716
:1005B0006D0815436408C2071443039A0126120507
:1005C000C01A91413605001C7141CE0740083043E6
:1005D0004908C01851412A46234600F07EFBCDE76A
:1005E000FFE7049801224000C117121A00238B4133
:1005F00004983146C417381AA141EEE730B40124FB
:10060000E407634030BC55E730B40124E40761409F
:1006100030BC4FE70000E0FFF0B51FB488B00B9985
:100620000998002448400999C00F490049080991D8
:10063000C0070B990090490049080B910999089847
:10064000A64608431CD00B990A98084318D009986D
:1006500001244000420D4800410D09982405000383
:10066000000B204309900B980003000B20430B90D4
:1006700050181C494018002201901446104605E00D
:10068000002001460DB0F0BD032801DA034600E06A
:1006900003239C46C11A0AAE0AE05F0008ADED5B79
:1006A0004F00F75B7D430027AA187C41491C5B1E65
:1006B0006145F2DD410004AB5A522104120C0A4399
:1006C000240C401C0828DFDB01980290009970463A
:1006D00001910090059B049A0799069800F00AFB87
:1006E000D0E700000DFCFFFFF0B50C465C4085B084
:1006F000E40FE40703944C00002664085900944674
:10070000490802460296224321D062460A431ED07F
:100710006200570D4A000E032303550D01240246C3
:100720002C492405781B1B0B360B4018234326430A
:10073000614600901C46501AB44103D30098401CF7
:10074000009002E0921800985B41002803DA002034
:10075000014605B0F0BD0020012109050746864687
:1007600011E064461D46141BB54106D36546521B75
:10077000B341744607430C43A646CD0740084908D9
:10078000284392185B4105460D43EAD110461843B1
:1007900013D06046194650407140084306D0604669
:1007A000101AB34106D20122002306E000220123E1
:1007B000DB0702E00122D243531000987446010582
:1007C000381C6141029C039D0019694100F085FAC3
:1007D000BFE70000FD0300000122D207002800DB74
:1007E000101A002900DB511A814201D801207047FC
:1007F000002070470122D207002800DB101A0029D0
:1008000000DB511A814201D201207047002070475D
:100810000122D207002800DB101A002900DB511A40
:10082000814201D301207047002070470122D20786
:10083000002800DB101A002900DB511A814201D97F
:1008400001207047002070470122D207002800DBFA
:10085000101A002900DB511A814201D10120704792
:100860000020704710B5002904DB0C460121C907A0
:100870004042A141002B04DB1C460123DB0752420E
:10088000A341801A994101D3012010BD002010BD61
:10089000C217C10F504010B54018CA079623002157
:1008A00000F0E2F910BD10B500229623114600F0C9
:1008B000DBF910BD0EB5C217C10F5040CA07401872
:1008C0000021054B0293019200910A460B4600F06D
:1008D00011FA03B000BD0000330400000EB5054955
:1008E0000291002100910A460B46019100F002FAA4
:1008F00003B000BD33040000C20F410040020123D9
:10090000400ADB05D207090EC0187F2901DA002052
:100910007047962903DC9623591AC84001E096399E
:100920008840002AF4D04042704741004002012232
:10093000400AD205090E80187F2901DA002070478D
:10094000962903DC9622511AC84070479639884090
:100950007047000070B5CD0F4A0009030123090B51
:100960001B0519430B4BED070024520D9A4201DA87
:10097000002070BD074B34339A4203DC9A1A00F012
:100980007DF802E00449511888402C43F1D04042E0
:1009900070BD0000FF030000CDFBFFFFC20FD207B8
:1009A000400040080BD0C10D0723DB01C9184002ED
:1009B0000905400A1143C20840071143704700204F
:1009C00001467047CB0FDB07490010B549080246C6
:1009D0000A4307D00A0D07240903E401090B121B7F
:1009E000002A01DC002010BDC900440F0C43C100E7
:1009F000E018D205801800F02FF910BDF0B51FB433
:100A00000646002082B005464024019100901BE07C
:100A1000019922460F46304600F030F8049A059BB3
:100A2000801A994110D310461946224600F016F854
:100A3000361A8F410197224601200021009F00F0C5
:100A40000DF838184D4100902046641E0028DFDC68
:100A5000019B00982946324607B0F0BD10B5202A08
:100A600004DB0146203A9140002010BD9140202334
:100A70009C1A0346E3401943904010BD10B5202A4C
:100A800004DB0846203AD040002110BD0B46D3407D
:100A9000D0402024A21A91400843194610BD10B539
:100AA000202A06DBCB170846203A1041C1170B431A
:100AB00006E00B461341D0402024A21A914008437F
:100AC000194610BD02681378511801601846704726
:100AD00010B5D160044951610449116200211161CE
:100AE000114600F0ADF910BDC50A00002D0E000042
:100AF0004268002A08D001680B78491C002B03D0FB
:100B0000521E06C0184670470121C160881E7047FA
:100B10004268002A0BD0C3680168002B07D18368A4
:100B20008B4204D0491E521C06C000207047002092
:100B3000C04370470FB400B589B00A460DA90091B3
:100B400000230C99002ACB60234B0693234B079379
:100B500001D0042300E00023214A0292214A089296
:100B6000019302466B46002000F095FB09B008BCDB
:100B700004B01847F0B585B007460020C043019087
:100B80001E46002015460C460091029104903B46FB
:100B90006A46314604A8FFF7CDFF04990246601863
:100BA000002D05D0002901D0034600E023462B602C
:100BB00000290ED0002A02DD0099814209D0001BD5
:100BC000019000943B466A463146029404A8FFF720
:100BD000B1FF05B0F0BD0000F10A0000110B0000EC
:100BE000FFFFFF7F2D0E0000F7B5009C0F4600268B
:100BF0002578641C002D05D000F014F90068405DD4
:100C0000C007F5D12B2D02D02D2D18D0641E3946EA
:100C10002046029A00F06AFC002F04D03968A142F5
:100C200001D1009939607105022400290BDA404294
:100C3000002803DD10F03EF80460A007FEBD01208F
:100C400080020643E3E70028F8DA10F033F8046086
:100C50000048FEBDFFFFFF7F002904DA401C490069
:100C600001D140084000704770B40024050C05D144
:100C70001024000402D1002921D01124050E01D135
:100C800000020834050F01D10001241D850F01D198
:100C90008000A41C002801DB4000641C002908D04F
:100CA00020252E1B0D46F540A14000D001212943EF
:100CB000084301061B1B000ADB1D02D5002070BC87
:100CC0007047DB05181880180029F8DA401C490025
:100CD000F5D170BC40084000704710B5002B08DA11
:100CE0000024401C614192185B411A4301D1400825
:100CF000400010BDF0B51FB482B005460C0003D013
:100D000008460FF0BFFF02E00FF0BCFF20300246A4
:100D1000009021462846FFF7A1FE049B059A044651
:100D20000F4618431143084314D0184610431BD0F4
:100D3000009840210A1A18460599FFF79FFE0546BC
:100D40000E46009A05990498FFF788FE084305D0DF
:100D5000012004E02046394607B0F0BD0020C1174D
:100D600005430E432C43374300990E986305401A00
:100D70007905E40A00220C43FD0A0A3002D500205E
:100D80000146E9E70105101969410C9C0D9D001908
:100D90006941FFF7A2FFDFE74A0009030123090BBE
:100DA0001B0519430A4B10B5520D9A4202DA002076
:100DB000014610BD064B34339A4203DC9A1AFFF702
:100DC0005DFE10BD034BD218FFF748FE10BD0000BA
:100DD000FF030000CDFBFFFF10B5002904DB012459
:100DE000E40740428C412146002B04DB1C460123D2
:100DF000DB075242A341994200D1904210BD00004E
:100E0000064C0125064E05E0E36807CC2B430C3C5D
:100E100098471034B442F7D3FFF756F92840010041
:100E200048400100004870475016010010B50446C4
:100E3000FFF7F8FF0068005DC007C00F10BD00009D
:100E4000F3B58DB000200A9001200B9000260846D3
:100E50000C300C4609906269012109989047051EE3
:100E60002ED0252D2DD0216A8847002818D0626900
:100E7000012109989047216A88470028F7D1411E2F
:100E800062690998904700E0761CA1690D9888472F
:100E9000216A88470028F7D1E1690D988847DAE789
:100EA000A1690D9888470746A84201D1761CD2E770
:100EB000E1690D9888477F1C02D10A98002877D0F5
:100EC00049E1002762693D463946099890472A283A
:100ED0000CD16269012109989047012506E00A2199
:100EE0004F433F18303FEBD4102005436269012186
:100EF00009989047014630390A2903D29B498F420D
:100F0000DEDCECE7E90600D4994F6C280AD04C28C7
:100F100010D0682824D06A282ED074280CD07A28C3
:100F20000AD00DE062690121099890476C2823D00E
:100F300004211CE0202005436269012109989047A3
:100F4000A760656065284FD026DC582839D01ADCA8
:100F5000452849D012DC252834D04128B0D143E0BF
:100F60006269012109989047682802D008210D4341
:100F7000E6E70120C002DEE70220DCE7462833D0A6
:100F800047282CD130E05B2870D061282CD0632812
:100F90006CD0642823D161E06F284FD009DC66282B
:100FA00022D0672820D0692826D06E2817D12EE0BD
:100FB000CDE070284DD073286FD075284ED078289A
:100FC0000DD154E0A1690D9888470546252800D128
:100FD0006CE7E1690D9888476D1C00D16DE7BAE0B8
:100FE0000A224CE00A2252E0012023466A46C0430E
:100FF0000D9900F050F9A3E02846402108436060B5
:10100000A807234601D5002239E000223FE0E80787
:1010100000D020E72068011D21600068290501D566
:10102000067018E7290701D5068014E7A90703D53C
:10103000F117066041600EE706600CE72846402184
:1010400008436060A807234601D5082217E008225C
:101050001DE0484928460840606016E028464021C7
:1010600008436060A8072346BCD5B9E715E02846C9
:10107000402108436060A80707D5234610220120BD
:10108000C0430D99C046C0465AE0234610220120B5
:10109000C0430D99C046C04652E000210C910B465A
:1010A0000091632802D05B2807D043E0E80601D412
:1010B0000120A060012000903CE0626901210998B4
:1010C00090475E2805D101200C900146626909987D
:1010D00090472169002906D10B4601AA8F00491CBF
:1010E000D3510829FADB002835D0216900290ED117
:1010F000C117C90E09184A11930001AA9A18490983
:101100004901411A01201368884003431360626952
:101110000121099890475D28E5D10C98002808D056
:10112000002001AB81005A58401CD2435A50082875
:10113000F8DB01AB01202246C0430D99FFF764F8AC
:1011400000280ADA401C06D10B98002803D00020A2
:10115000C0430FB0F0BD0A98FBE7E90702D10A9936
:10116000491C0A91361800200B9074E6CCCCCC0CAC
:10117000FFFFFF7FF1F7FFFFFFB5087889B0154645
:10118000FF2805D0491C2D2804D00022002407E0A8
:1011900000240BE00122F9E70A235C430419491CEF
:1011A0000878FF28F8D1002A00D06442002004907B
:1011B0002A7801462D2A01D02B2A0FD16D1C2D2A09
:1011C00002D00022049209E00122FBE700260A2255
:1011D00033466D1C00F0DDF9381871412F78FF2F70
:1011E000F4D10C9AA218069202460A4304D0FF23B7
:1011F000069A9133DA4205DA002109980A4606C0B8
:101200000DB0F0BD0024B74AB54D2646079200F058
:101210000DFA029006980391002801DA474200E097
:10122000074639050020AF4A001C5141019100904A
:1012300012E0F80707D022462B4630460799FFF701
:10124000EBF90646079122462B4610461946FFF752
:10125000E3F904460D467F10002FEAD10698019B62
:101260000028009A0399029806DAFFF73DFA324601
:10127000079BFFF739FA05E0FFF7CEF93246079BE7
:10128000FFF7CAF9049A002A02D00122D20751407E
:10129000099A03C2B4E7FFB591B000200990002578
:1012A000ED432E209E685C681F460190B9696D1C55
:1012B000129888470090396A88470028F6D100982C
:1012C000401C0AD00D20C0018443002E12DD00987E
:1012D0002B2809D02D280DD103E00020C04315B0E4
:1012E000F0BD012080020443B9696D1C1298884743
:1012F000761E009003A9600501D52D2000E02B206B
:101300006A461073491C0CA80F9102900AE0B96953
:101310006D1C1298884700900120400204431398E6
:10132000761E0560002E02DD00983028EFD001996E
:101330000098884245D18020044308E00998401E67
:1013400009900120400204431399681C0860B969A0
:101350006D1C761E1298884700903028EED030E041
:101360000199884205D1200603D480200443761ECB
:101370001DE000980FF06CFD002825D001214902E6
:101380000C43009807AA0F9903323038761E914219
:1013900008D208700F98401C0F90200607D50998B6
:1013A000401E03E0200602D40998401C0990A005C5
:1013B00002D51399681C0860B9696D1C129888479A
:1013C0000090002ECCDC59E0002E57DD00986528F7
:1013D00001D0452852D1A00550D5032000028443F6
:1013E000B9696D1C761E129888470090002E0CDD9E
:1013F0002B2804D02D2808D1FF2001300443B969DF
:101400006D1C12988847761E0090E00501D52D21AD
:1014100000E02B21029801700298401C029001907C
:1014200025E00120400204430EA902980131761EF6
:1014300088420ED20098029930380006000E0870DB
:1014400003D10299019881420AD90298401C029066
:1014500006E0E00501D5244801E023484042099018
:10146000B9696D1C12988847009013980560002E8A
:1014700004DD00980FF0ECFC0028D2D1F969129835
:1014800088470F99FF200870029903AA087000206E
:101490000A900B900CA90AA8099BFFF76DFEA00506
:1014A00002D40120C0431AE72420044209D0E007F7
:1014B00013D138680B9A0A99031D3B60006806C077
:1014C0000BE00B990A98FFF77DFA0146E00704D17B
:1014D0003868021D3A60006801602846FFE6000097
:1014E000000014400000F03FF1D8FFFFF7B582B0D4
:1014F000029C00272078641C15460197302802D0F2
:10150000002D15D015E020780127641C782804D020
:10151000582802D0002D09D00BE0002D01D0102D4D
:1015200007D1002710252078641C02E0082500E080
:101530000A250026009610E0009901276943081843
:10154000020C294680B2714300908E1838048642FE
:1015500001D3012001902078641C294600F056F840
:101560000028E9DA0398002805D0002F01D0641E76
:1015700000E0029C04600198002806D00FF09AFB5E
:1015800002210160C81E05B0F0BD00993004084377
:10159000F9E7F0B51FB486B00020009001900290EA
:1015A0000698069980B204900798090C020400146A
:1015B000114307900027089D099806913E463C4636
:1015C00003900398A9B20204000C039004982D0C18
:1015D0001543484300212246FFF740FAC7197141DD
:1015E00010340E46402CECDB3846029AFFF736FAF0
:1015F000009A019B80180090594102980191103087
:1016000002904028CCDB00980BB0F0BD3A2800D205
:101610003038202302469A43412A01D310463738F6
:10162000884201D30020C043704700000EB5054A30
:1016300002920022009213460192FFF75BFB03B077
:1016400000BD00003304000030B58C180278401C47
:1016500013071B0F01D10378401C120906D1027831
:10166000401C03E005780D70401C491C5B1EF9D13D
:1016700001E00B70491C521EFBD1A142E6D30020B1
:1016800030BD000010B52148016A8A0715D44A0709
:1016900015D4C90732D01E498A89002A15D0531E95
:1016A0008B8182688C6904C48C610A691B040DD02B
:1016B000002A22D10121016010BD022100E0042195
:1016C000C16113488021416110BD0A69012A09D115
:1016D000026801239A430260C361FF206830993099
:1016E0000C4A106001204861CA69002A05D0886947
:1016F00009898B00C01A904710BD10BDFF226832C7
:10170000054806A109A30CF075FFC04608D00140AA
:101710008895010280E200E0A02501004144435F7A
:1017200049525148616E646C65720000556E65786F
:101730007065637465642041444320696E7465720A
:10174000727570740D0A000070B582B000230193A9
:10175000444801688A6A4C6813252540132D02D13C
:10176000CB689B07DB0F4361930772D453070AD4FE
:10177000D30711D1130724D5048F838E1C1B102C83
:101780000EDD102310E0042088620220032142A213
:101790000DF08CFF02B070BD0120886202B070BDF8
:1017A000048F1B1B1C0610D0DBB20024058FC66AF9
:1017B00075192D5D0D74641CA342F7D1048FE318D5
:1017C0000387D20607D400212FE04B6A0824A343E5
:1017D0004B62D206F7D5CB68C28E448F141B5B04D4
:1017E000DB0EA34201D3438FD31ADAB2002A16D0FC
:1017F000097D438F046BE1540199012A10D0012324
:101800001C46890145582D7D41184E8F9B19096B47
:10181000CD54641CE3B201999A42F2D800E0002151
:101820008B01C3185C8FA2185A878A0181184B8FCD
:10183000CC8EA3420BD301230B618058002242625D
:10184000CA6B002A03D03A31098801A8904702B038
:1018500070BD02208862044804A1084A08A30CF065
:10186000C9FEC0466C900102B92501004145535F95
:1018700049525148616E646C65720000CE020000EE
:1018800041455320696E707574206F766572666C81
:101890006F770D0A00000000414553206F7574708A
:1018A000757420756E646572666C6F770D0A000042
:1018B000F0B581B001243F2900D993E00346806848
:1018C000456B2D688E0001A7BE59B7460B1A000064
:1018D000271A0000031A0000031A0000E51900008F
:1018E000E5190000E5190000E5190000E519000000
:1018F000E5190000E5190000E5190000E5190000F0
:10190000E5190000391A0000551A0000E519000019
:10191000E5190000E5190000E5190000E5190000CF
:10192000E5190000E5190000E5190000E5190000BF
:10193000E5190000E5190000E5190000E5190000AF
:10194000E5190000E5190000E5190000E51900009F
:10195000E5190000E5190000E5190000E51900008F
:10196000E5190000E5190000E5190000E51900007F
:10197000E5190000E5190000E5190000E51900006F
:10198000E5190000E5190000E5190000E51900005F
:10199000E5190000E5190000E5190000E51900004F
:1019A000E5190000CD190000CD190000CD19000087
:1019B000CD190000CD190000CD190000CD1900008F
:1019C000CD190000CD190000CD1900004348006971
:1019D0000024022809D001280DD0002802D103CA12
:1019E00004F0E8FE204601B0F0BD03CA04F0D4FEC6
:1019F000204601B0F0BD03CA04F0F2FE204601B05B
:101A0000F0BD022931D0022430E0344D00242C6195
:101A10006C619849354A01F0A1FD6869401C686114
:101A2000204601B0F0BD01F0D3FD284602F040F899
:101A30000024204601B0F0BD284909690C234B431E
:101A40002749CA58C918496801F088FD0024204672
:101A500001B0F0BD0024204604F07AFE0128C1D177
:101A60001E483030204900241CE001241B490F6926
:101A70000C26314679431A4A51188968214208D008
:101A800000247D1C15490D614C61042D10D31549AE
:101A900006E012494869401C4861032812D32949CD
:101AA00000241846224601F0B3FF204601B0F0BDE5
:101AB0006E430B498A598919496801F04FFD204648
:101AC00001B0F0BD0E20009000240A2228462146D5
:101AD00001F08EFF204601B0F0BDC046AC98010277
:101AE00054160100501D0100301D01001E3101007F
:101AF000B0B504290FD804468068C04679440979F6
:101B000049008F44020A0E1C1700104910A201F070
:101B100025FD0020B0BD0120B0BD01F059FD002021
:101B2000B0BD00250321284604F022FE06492046C8
:101B30002A4602E003490022204601F069FF002006
:101B4000B0BDC046401D0100C01D0100881300004B
:101B5000415445300D0A0000B0B582B001240A2975
:101B600010D883687944097949008F440E29050506
:101B70000B0B0B0B0B0B1A001949096800242246AA
:101B800001F046FF204602B0B0BD5068144908601D
:101B9000144915A2184601F0E1FC0024204602B0C9
:101BA000B0BD0024019403CA09A201AB02F04EF8B3
:101BB0000228E7D1019804F02FFE204602B0B0BD04
:101BC000184601F005FD0024204602B0B0BDC04615
:101BD0002B4353513A2025642C252A0D0A0000007E
:101BE000709901028813000041542B4353510D0A90
:101BF00000000000B0B582B00546002404F006FEE7
:101C000001280DD108498C60E86B426853684B602D
:101C1000009401926A4601F0FBFE204602B0B0BD7E
:101C2000E443204602B0B0BDB0930102B0B5054612
:101C3000881E02280AD3A868012913D0002915D1CB
:101C40000C490DA201F08AFC0020B0BD0220014623
:101C500004F08EFD064900242846224601F0D8FEF5
:101C60002046B0BD01F0B4FC0020B0BD0120B0BDE5
:101C7000101D01008813000041542B4346554E3D72
:101C8000300D0A00B0B5E0B00324E1016D462846EE
:101C90000EF0E0FF204621462A460DF007FD002009
:101CA00060B0B0BDF0B597B00820149064201390D8
:101CB0002548109002200E904B20C0011690234D15
:101CC00028461430129001270F97B8021190032074
:101CD0000EA905F051FE0026F443002802D020464C
:101CE00017B0F0BD0C35284601F0F0FE0028F6D103
:101CF00080200C9016490B910A90164809901648BE
:101D00000890164807901648069039200590154807
:101D10000490154803900D95144D03A9284601F031
:101D200087FC0028DBD1009501970F4C104911A2C8
:101D3000124B204601F020FE1149204601F050FED2
:101D40003446204617B0F0BD28BE0102C0960102FD
:101D500028C20102A8C20102352E0000852E000013
:101D6000052E0000D01E0100DC98010238C70102D8
:101D7000B01C01004149523738304500D01D0100E8
:101D8000851C000010B50348002404700EF0FEFB13
:101D9000204610BD889D010280B501F053F9002056
:101DA00080BD0000F0B58DB00E4600270C970B9754
:101DB0000A970997089707970697059702908068F2
:101DC0000490406B0068019004F0BCFC04465BA1E9
:101DD00005220392FEF7EAF95A4D00281ED05AA1B7
:101DE00005222046FEF7E2F9002817D058A1052267
:101DF0002046FEF7DBF900280FD059A10522204626
:101E0000FEF7D4F9002809D057A105222046FEF795
:101E1000CDF9002807D156A500E04FA505A820213F
:101E20002A4601F0E5FF01203F2E00D936E0C046EA
:101E30007E4436797600B7443340474A57313131D2
:101E4000313131313131653031313131313131314F
:101E50003131313131313131313131313131313172
:101E600031313131313131313131313131311F1F86
:101E70001F1F1F1F1F1F1F1FBE48416A04290CD1AF
:101E8000039A426287620C2050433D490A58081861
:101E9000416805AB049801F061FB38460DB0F0BD18
:101EA000B44C00206062A062CD49364A049801F02B
:101EB00055FBA06A401CA062EFE7049801F088FB84
:101EC000019801F0F5FDE8E7AA48406A05E0A94954
:101ED000486A01220243032A1CD1A649421C4A62D5
:101EE0008F62062ACFD30BE0A2494A6A012013462B
:101EF0000343052BD2D1501C48628F62062803D3BE
:101F00001E490DE09B48406A0C2141431C48425841
:101F10004018BDE7886A401C8862032805D316492B
:101F20000022029801F074FDB7E70E200090002116
:101F30000A220198029B01F05BFDAEE73436303097
:101F400030000000463101003436303032000000ED
:101F50003436303031000000554E494E45540000B3
:101F60003436303036000000343630303300000074
:101F700043544E4554000000B01C0100001D0100F8
:101F800084160100C630010070B5022956D30F290E
:101F900007D1784C217A012905D1002222728F497C
:101FA0004AE0012070BD866801F0B6FD002004F013
:101FB000D7FB012803D10020032104F0D9FB002521
:101FC000284604F0C5FB012804D130346A490022B8
:101FD000204631E0304600F0EBFD00282ED03046A0
:101FE000FFF708FE002829D004F0CCFB012807D118
:101FF0005F498D60F06B4268E26252684A601AE0A5
:10200000022004F0A5FB012808D159498D61F06B2D
:102010004268E26252684A6110310CE0022004F02A
:102020009FFB01280AD152498D62F06B4268E2623F
:1020300052684A6220312A4601F0EAFC002070BD55
:1020400010B582B003460120272931D87944097997
:1020500049008F442C132D2D162D2D2D2D2D2D2D7A
:102060002D2D2D2C2D2D2D2D2D2D2D2D2D2D1C2DB2
:102070002D2D2D2D2D2D2D2D2D2D2D2904F0DCFE7A
:1020800015E0DF490022184601F0C2FC0FE00020F5
:10209000019003CA08A201AB01F0D8FD012806D1C6
:1020A000019804F0F5FF02E00248012101720020CE
:1020B00002B010BDAC9801022B51495552433A2051
:1020C00022636C6F736564222C25640D0A00000086
:1020D000B0B502294AD30F2914D18568002004F035
:1020E0003FFB012803D10020032104F041FB002421
:1020F000204604F02DFB012806D1D94830301E4976
:10210000002231E00120B0BD2846FFF773FD002812
:102110002CD004F037FB012808D115498C60E86BFE
:102120004268CF4BDA6252684A601CE0022004F039
:102130000FFB012809D10E498C61E86B4268C84B3E
:10214000DA6252684A6110310DE0022004F008FBA7
:1021500001280BD106498C62E86B4268C04BDA62F9
:1021600052684A622031224601F052FC0020B0BD84
:1021700038900102AC980102301D010080B502299F
:1021800005D3042905D19E49002201F041FC00201D
:1021900080BD012080BDC046B0B50546881E02281E
:1021A0000AD3A868012913D0002915D10C490DA222
:1021B00001F0D4F90020B0BD0220032104F0D8FAC8
:1021C000064900242846224601F022FC2046B0BDE4
:1021D00001F0FEF90020B0BD0120B0BD501D01008E
:1021E0008813000041542B4346554E3D310D0A00E3
:1021F00010B50F290BD001291DD000291DD1FFF7E3
:10220000C1FD0020022104F0B3FA002010BD0446F5
:10221000002004F09DFA012803D10020022104F0DF
:10222000A7FA002004F09CFA012804D104490022F6
:10223000204601F0EDFB002010BD012010BDC0467E
:10224000401D0100F0B581B00124322928D805468F
:102250008768786B0668C0467944097949008F44DD
:102260002F3F1919191F1F1F1F1F1F1F1F1F221F5D
:102270001F1F1F1F1F1F1F1F1F1F1F1F1F1F1F1F6E
:102280001F1F1F1F1F1F1F1F1F1F1F1F1F1F1F1F5E
:102290001F1F26001E4900242846224601F0B8FBD5
:1022A000204601B0F0BD1B48017800291FD0184915
:1022B00000242846224601F0ABFB204601B0F0BDC9
:1022C0000024FC623969384688470028FAD0114852
:1022D0000470FC62FFF756FD0E20009001220EE014
:1022E000304601F0E5FB0024204601B0F0BD01219D
:1022F0000170FFF751FD0E200090002405223046AA
:1023000021462B4601F074FB204601B0F0BDC046CB
:10231000D01C01007499010210B586B0034601205B
:102320003B2900D956E0C0467944097949008F44D9
:1023300050505151335151515151515151515151AD
:10234000515151515151515151515151515151517D
:10235000515151515151515151515151515151516D
:102360005151515151391D1D1D1D1D1D002005903C
:1023700003CA02AA009218A205AB01F067FC02286A
:1023800027D1039A029817A1FDF710FF002820D14A
:10239000059804F07DFE1CE0B5490022184601F0C6
:1023A00037FB16E0002002900590049003CA05AAAE
:1023B000019204AA00920DA202AB01F047FC03288F
:1023C00007D1049A0599029804F032FF029804F0AC
:1023D000CDFE002006B010BD25642C2025700D0A0E
:1023E00000000000434C4F53454400002B5245432E
:1023F000454956452C25642C25643A0D0A2565006F
:10240000201D0100012901D80020704701207047DC
:10241000B0B50546881E03280BD2104604F0BAF961
:102420000F48C16A00242846224601F0F1FA2046EE
:10243000B0BDAC6801290BD000290ED104F084F99D
:102440000346084908A2204601F088F80020B0BDE4
:10245000204601F0BDF80020B0BD0120B0BDC0464F
:10246000AC9801028813000025730D0A00000000DB
:1024700070B582B001240F293DD803468568686B8A
:102480000668C0467944097949008F4407141E3410
:102490003434342F373434343434434E66480024D3
:1024A00004708461C461012101716649664A28464D
:1024B00001F054F81FE0284601F08AF8304601F098
:1024C000F7FA0024204602B070BD5B480024047176
:1024D0008269042111430278002A2ED0052958D19F
:1024E000016A491C016259D2624961E0524B187875
:1024F0000024002831D0204602B070BD4E4B187821
:10250000012816D103CA183351A201F09FFB002005
:1025100002B070BD48480024846101210171007837
:102520004849002812D1484A11E0434E307900282A
:102530001BD00024204602B070BD052932D10024F2
:10254000012101708461C46101713E493F4A2846FE
:1025500001F004F8204602B070BD03CA183340A24F
:1025600001F074FB204602B070BD002004F0F8F8C2
:10257000012803D10020032104F0FAF800242046AA
:1025800004F0E6F8012816D130362D4900243046F3
:102590004BE000210162C169491CC1610E2000901D
:1025A00000241CE0C169491CC161652915D330496B
:1025B0000024184639E02846FFF71CFB00289AD073
:1025C00004F0E0F8012812D11C4900248C60E86B6B
:1025D0004268F26252684A6027E00E2000900222B0
:1025E0003046214601F004FA204602B070BD0220B8
:1025F00004F0AEF8012809D1104900248C61E86B81
:102600004268F26252684A6110310EE0022004F022
:10261000A7F8012800D06EE7084900248C62E86B17
:102620004268F26252684A622031224601F0F0F9B3
:10263000204602B070BDC046AC980102389001023D
:10264000301D010088130000E2300100ED30010070
:102650002B43475245473A20252A2C256400000089
:102660002B435245473A20252A2C256400000000C0
:10267000201D0100E01C0100B0B584B001243B29FD
:1026800000D937E0134605468068C0467944097989
:1026900049008F444B5532322F2F2F2F2F2F2F2FA2
:1026A0002F2F2F2F2F2F2F2F2F2F2F2F2F2F2F2F3A
:1026B0002F2F2F2F2F2F2F2F2F2F2F2F2F2F2F2F2A
:1026C0002F2F2F2F2F2F2F2F2F2F1D1D1D1D1D1D86
:1026D0000024039403CB01AA00921C4A03AB01F02F
:1026E000B5FA022806D1029A019819A1FDF75EFDFC
:1026F00000280FD0204604B0B0BD1848006804F090
:10270000C7FC174900242846224601F081F92046DB
:1027100004B0B0BD1148006804F0BAFC10490022B2
:10272000284601F075F9204604B0B0BD0B490B6096
:102730001E210CA200F012FF0024204604B0B0BD00
:1027400000F046FF0024204604B0B0BD4632010030
:10275000434C4F5345204F4B000000007899010235
:10276000F01C010041542B434950434C4F53453D0D
:1027700025640D0A00000000F0B589B00446012070
:102780003B2900D9AAE01646A7687A6B1568C046AF
:102790007944097949008F44536AA071A1A1A1A18C
:1027A000A1A1A1A1A1A18AA1A1A1A1A1A1A1A1A130
:1027B000A1A1A1A1A1A1A1A1A1A1A1A1A1A1A1A109
:1027C000A1A1A1A1A1A1A1A1A1A1A1A1A1A11D1D01
:1027D0001D1D1D1D0027089703CE06AA0092414A21
:1027E00008AB01F033FA022877D13F480568089812
:1027F000854272D1079A069E3CA130460592FDF7AC
:10280000D5FC002847D03DA13046059AFDF7CEFC07
:10281000002840D03CA13046059AFDF7C7FC0028AF
:10282000314E5AD1284604F04DFC7068401C70604F
:1028300003283CD303207060306804F0BBFB36E013
:1028400029480660304604F009FC059026480068D7
:1028500004F0D8FB04902448006804F0DFFB0499DE
:10286000019102900598012827D02EA026E0384635
:1028700000F0AEFE284601F01BF92EE01A4D286844
:1028800004F020FC6868401C686003280FD3002215
:102890006A6022490DE0144E7760284604F028FC57
:1028A000306804F06BFD002801D01B4900E00C49A2
:1028B0000022204601F0ACF80FE019A000901A4960
:1028C0001AA23846334600F049FE0E20009000213F
:1028D000B4222846234601F08BF8002009B0F0BD51
:1028E000F01C01004632010038970102414C52456C
:1028F00041445920434F4E4E45435400434F4E4EA2
:10290000454354204F4B0000434F4E4E4543542007
:102910004641494C00000000901D0100B01C010020
:1029200054435000554450008813000041542B4339
:10293000495053544152543D25642C222573222C76
:10294000222573222C25750D0A000000B0B582B037
:1029500014468A1E022A12D38568012917D000293D
:102960001CD1204604F040FB00901E210EA22846F8
:10297000234600F0F3FD0024204602B0B0BD094913
:102980000024224601F044F8204602B0B0BD28469B
:1029900000F01EFE0024204602B0B0BD01242046F7
:1029A00002B0B0BDA01D010041545E4845415254E3
:1029B000434F4E4649473D312C25642C25750D0A61
:1029C00000000000F0B583B014468A1E022A1CD312
:1029D0008568012921D0002926D1164F3C60204668
:1029E00004F0F4FAFDF7CEFB0646386804F0EEFA80
:1029F0007108009101901E210FA22846234600F085
:102A0000ADFD0024204603B0F0BD09490024224654
:102A100000F0FEFF204603B0F0BD284600F0D8FDD0
:102A20000024204603B0F0BD0124204603B0F0BDD1
:102A3000F01C01007C99010241545E48454152540A
:102A4000424541544845583D25642C25752C257335
:102A50000D0A0000F0B585B0044601203B2900D9DD
:102A600085E0A5687944097949008F443F547F5B2C
:102A70008080808080808080808080806080808076
:102A80008080808080808080808080808080808046
:102A90008080808080808080808080808080808036
:102AA00080801D1D1D1D1D1D0020049003CA02AA4B
:102AB0000092304A04AB01F0C9F8022856D12E48E2
:102AC00085680498854251D1039E029F2BA1384608
:102AD0003246FDF76BFB00283AD02AA13846324631
:102AE000FDF764FB002841D128461DE0224CA2607E
:102AF000104604F09FFA002838D001F010FAE06088
:102B0000002833D0A36840680090234923A22846B8
:102B100000F024FD2AE018480021C160284600F09A
:102B200057FD23E01448806804F0B2FA19E000F081
:102B3000BFFD012804D11048C16803C900F0C0FEE0
:102B40000D48C0680CC81349284600F047FD0DE049
:102B5000284604F06FFA0028074907D0C96801F039
:102B6000B4F90B490022204600F052FF002005B0C6
:102B7000F0BDC046463201003897010253454E442D
:102B8000204F4B0053454E44204641494C00000025
:102B9000F01C0100204E00008813000041542B431C
:102BA000495053454E443D25642C25750D0A0000BF
:102BB000F0B583B0074600F0AFFF0026304604F0C2
:102BC00043FA032835460BD10421284604F0C6FBFE
:102BD000F86B51492A4600F01BFF304603B0F0BDA8
:102BE00002970024204604F02FFA0428254609D134
:102BF0000298C06B49492A4600F00AFF2646304633
:102C000003B0F0BD0027384604F01EFA05283D4603
:102C100009D10298C06B40492A4600F0F9FE3E46B1
:102C2000304603B0F0BD01970125284604F00CFAA8
:102C30000328029FC8D00125284604F005FA04287D
:102C4000D6D00125284604F0FFF90528019FE0D0E1
:102C50000225284604F0F8F90328029FB4D0022583
:102C6000284604F0F1F90428C2D00225284604F0D1
:102C7000EBF90528019FCCD0254C2068401C03218E
:102C8000FDF73EFA0D46084604F0DEF90628029FDD
:102C900008D1284604F0CEF9002803D001F03FF90E
:102CA00000282AD1681C0321FDF72AFA0D460846A0
:102CB00004F0CAF9062808D1284604F0BBF9002818
:102CC00003D001F02CF9002817D1681C0321FDF76F
:102CD00017FA0D46084604F0B7F90021CE4306283E
:102CE00000D07AE7284604F0A5F9002800D174E75F
:102CF00001F015F9002800D16FE72560F86B054950
:102D00002A4600F085FE0026304603B0F0BDC046DE
:102D100080990102B01D0100701D0100801D01009D
:102D200080B58AB00620042108F012FB4B20C001B8
:102D300009900820079064200690B448143005904C
:102D40000648039002200190012002908002049026
:102D5000032001A904F010FE0AB080BD28BE0102C4
:102D6000B0B582B001220F293ED803468068446B7B
:102D70002468C0467944097949008F44071F2527F4
:102D8000343535353535353535350A152749002281
:102D900004E02649CA68092A20D8521CCA6016498C
:102DA000164A00F0DBFB1EE0002003F0D1FC0128F6
:102DB00019D11E4830300E49002212E000F008FC04
:102DC000204600F075FE0EE00D4908E00E20009050
:102DD00000210122204600F00BFE04E005490022FC
:102DE000184600F015FE0022104602B0B0BDC046E5
:102DF000301D0100101D010088130000F930010092
:102E0000C01C010080B5032004F09EFD80BD0000C1
:102E10000648416B0020002905D0054A914203D0A5
:102E200049680029FAD1704701207047AC98010227
:102E3000001D0100B0B514460D460846114600F0CD
:102E4000ECFE012816D1285D002813D1002C0BD0F0
:102E50006019401E00780A2806D10320084A01465E
:102E60002B460CF023FC05E00320054A01462B46C7
:102E70000CF01CFC03202946224604F051FEB0BD94
:102E80008F300100F0B585B0054604A80024047019
:102E9000E743002D12D0EA68002A0FD0686A0028A4
:102EA0000CD0A86A002809D0401EE96A814200D3EC
:102EB0008EE004A928469047002803D03C462046CF
:102EC00005B0F0BD514EE86A411CE962696A049A96
:102ED0000A54E86A696A002202920A54E86A0928D8
:102EE00006D1696A09224848FDF753F900283ED007
:102EF0003078411E022908D800F00EFEB168401A51
:102F00004349884264D8414E30780A2820D00128AD
:102F100023D16E6A3A213046FDF72AF9002847D0BE
:102F2000019002980390E96A03AB304639A200F0A1
:102F30008DFE02284CD10398002849D00A21334A3B
:102F4000117001990818696A401AC01C50602FE07E
:102F50007068E96A81422BD13AE004A800780A2817
:102F60000FD00D2814D101202863E86A1AE001204F
:102F7000307000F0D1FDB0603078411E0229BBD91D
:102F8000C3E7296B012904D102202863E86A03E022
:102F9000296BE86A022905D1022817D10298E86254
:102FA000286305E0012803D1686A00783E280FD025
:102FB000A86AE96A401E81420AD2EA6804A9284642
:102FC00090470028114E00D17DE777E702982863EB
:102FD000E96A686A00F021FE01280FD16B6AE86A8D
:102FE000002806D0C018401E00780A2801D10DA282
:102FF00000E010A2032001460CF058FB03480470C7
:10300000204605B0F0BDC046D2290100C09601029D
:10301000DC0500002B524543454956452C252A2CFA
:1030200025643A005B415420526563765D20257328
:10303000000000005B415420526563765D202573DB
:103040000D0A000010B5064C2078002108F03CF96C
:10305000044806F0E1F92078012108F035F910BDA7
:103060003696010260E31600B0B50F2001F01EFB9A
:10307000194D6870287033282AD120243721204622
:1030800001F060FB2120032101F05CFB22204021A4
:1030900001F058FB2320082101F054FB3020AA2125
:1030A00001F050FB0D4802210187322001F04AFB5C
:1030B0003320012101F046FB5F21204601F042FB55
:1030C0000F2001F0F3FA28700A2006F0A5F9B0BD30
:1030D00002480021C187B0BDD495010212A70102A8
:1030E000F0B583B001903A4C2120029060723948CB
:1030F00000886070384FF9886171BA6ABA61374ADE
:1031000012782270000AA070080AA071BD78C3204E
:1031100006020AF009FB01998D420DD17D21C900FB
:10312000FCF7D8FF0D4639810AF0FEFA28182D4920
:103130004118B878464303E04E43294971180646C2
:103140008D19FD620AF086FA40190AF0DFFE064684
:103150000D462548007B0AF065FD24490988222296
:10316000A15482B2D20B801802B2D0175210B218FA
:103170006841130E029D6355130C202563553B6D6A
:10318000A3761D0AE5761D0C25771B0E6377234673
:103190002233090A5970A277BA64F864BA65F865EF
:1031A000100AE0770AF0C0FAF861FB6A28210122D0
:1031B00020460DF0D5FC0AF0B7FA786108F086FCDD
:1031C0000028FBD1042008F03FF8002003B0F0BD38
:1031D000EAD00102CC97010238960102A4970102BD
:1031E000609E010060DB0000AE900102B09701021A
:1031F00070477047B0B582B0194C2068056801A9C6
:103200000020087007E090470198401C01A9087051
:10321000C0B2082822D2012211048140294209D0DB
:103220002268516080002018826A002AECD001A830
:103230000121E8E7130283402B4201D0022104E080
:1032400082402A42E0D00321134622685360800066
:1032500020188268002AD7D001A8D4E702B0B0BDF8
:10326000BC920102FEE7000010B509480168CA6976
:1032700020231343CB610269032A08D1012293055D
:103280000C689C430C605102C26E0A43C26610BDBA
:103290003093010281B010B581B00393002807D0AC
:1032A000C16A002904D003AB0093C46A0021A0477F
:1032B00001B010BC01BC01B00047000080B502465F
:1032C00008480068002807D091B2120C03889A427F
:1032D00003D040690028F9D180BD002200F0F4FA43
:1032E00080BDC04634C70102F0B581B05C4C206897
:1032F000856BE80707D0E168002904D000208847E3
:10330000206801218163A80707D52169002904D01D
:1033100001208847206802218163680707D5616919
:10332000002904D0022088472068042181632807EF
:1033300007D5A169002904D0032088472068082107
:103340008163E80607D5E169002904D00420884795
:10335000206810218163A80607D5216A002904D0BE
:1033600005208847206820218163680607D5616AA7
:10337000002904D006208847206840218163280660
:1033800007D5A16A002904D007208847206880213A
:1033900081630126E80507D5E16A002904D03702D8
:1033A0000820884720688763A80507D5216B002976
:1033B00004D077020920884720688763680507D50D
:1033C000616B002904D0B7020A2088472068876310
:1033D000280507D5A16B002904D0F7020B208847E8
:1033E00020688763E80407D5E16B002904D0370320
:1033F0000C20884720688763A80407D5216C002922
:1034000004D077030D20884720688763680407D5B8
:10341000616C002904D0B7030E20884720688763B9
:10342000280407D5A16C002904D0F7030F20884792
:1034300020688763E80307D5E16C002904D03704CE
:103440001020884720688763A80307D5216D0029CD
:1034500004D07504112088472068856301B0F0BD51
:10346000C093010202480068411E88417047C0466F
:10347000C0970102F0B58DB0002862D004464068C4
:1034800000285ED0A06840285BD8E56A002D58D09F
:103490000746204640300026039003E0019E4AE0A4
:1034A000039848E0402101220691FCF74FFEAE420E
:1034B00002963ED200203146019009900398069B67
:1034C0003E46002EEAD0606A0491405C079009985D
:1034D000401C05900021042708916518EA5C012A28
:1034E00017D10A966268D3191B1F1B68099E9E5D3F
:1034F0000798864208D1059D5B5D002B0A9E22D06D
:103500000898401C089003E0403500222A70A66805
:10351000069B0837491CB142DFD308980028BFD06A
:103520000499491CE06A8142059809900398C8D320
:1035300001E003983E463746E56A029E761CAE429D
:10354000B0D30DB0F0BD616A0B91E16A0C91D15915
:103550000BAA204600F09CF80DB0F0BD81B0B0B5CC
:1035600083B00D460446079307AB02938069E16977
:103570000DF070FB206265480078002803D1216AB5
:10358000A06900F09FF96369A169226A2046984703
:103590000146A06B002905D069460C600021224B32
:1035A0000A460CE000F084FA7D2081002846FCF7F2
:1035B00091FD0246A06B69460C6000211B4B00F098
:1035C000D3FA002003B0B0BC02BC01B00847C0462B
:1035D00080B5806B00F06CFA002080BD70B582B0C1
:1035E0000D460446466911461A46B0470146A06B8F
:1035F000002907D069460C6000210B4B0A4600F0F9
:10360000B3FA0EE000F054FA7D2081002846FCF762
:1036100061FD0246A06B69460C600021034B00F07F
:10362000A3FA002002B070BD153700002B37000050
:1036300070B50D460446802100F0C0FA2868E063AA
:1036400068686060A868A060E868E0602869206138
:1036500068696061A869A061E86900262662E06186
:10366000286A6062686A2663E662A062A86A60638C
:103670002046383000F02AFA002802D0F6433046BF
:1036800070BD2148016821600460304670BDC046AD
:1036900070B514460D460646881E032802D8B06B46
:1036A00000F006FAF06B2946224600F00DF970BDD5
:1036B00016480178012048407047C04670B512484E
:1036C0000468002C1FD0114E11A52169204688479F
:1036D000002815D1307800280DD1E16A606A00F029
:1036E0009CFA0146606A012903D0E16A00F0E8F81B
:1036F000284600F0E3F82046FFF7BCFE0020E06219
:103700002468002CE1D170BD30C7010228C7010236
:103710000D0A000010B50446806B00F0C9F9E06B9B
:103720000521002200F0D0F810BD10B50446806BD2
:1037300000F0BEF9E06B0421002200F0C5F810BDD6
:10374000F0B581B000910646C7680468A01C3946F0
:10375000FCF7C0FC00257068814201D1ED430BE00D
:10376000601C3946FCF7B6FC316032695143B068E1
:1037700008180099FCF7D8FC284601B0F0BDB0B598
:10378000012400250560446008300EC0B0BD70B54E
:103790000E460446C1680068401CFCF79BFC0025EF
:1037A0006068814202D1ED43284670BD22695043D2
:1037B000A16841183046FCF7B7FCE1686068401C1E
:1037C000FCF788FC6160284670BDB0B50024002875
:1037D0000DD0054600688842FDD3401A286068680D
:1037E0004018E968FCF776FC69602046B0BDE44308
:1037F0002046B0BDB0B5002400280ED005460068B4
:1038000040182860EA689042FDD8A8684018114620
:10381000FCF760FCA9602046B0BDE4432046B0BD83
:10382000F0B583B0164602460027F843002E22D09A
:103830001C46002B1FD00D46D168136899421AD937
:10384000CB1AAB4217D39268019252198A423A4678
:1038500007D9019A8A1A0292029A52199342029A3D
:1038600009D3029201981018FCF734FC31600298D9
:1038700040192060384603B0F0BD4068704780684A
:10388000704702460020002A04D01060506090600B
:10389000D1607047C0437047002803D00168484298
:1038A0004841704701207047002805D00168C06872
:1038B000411A484248417047012070470020704734
:1038C0000020704700207047F0B583B014460D46C5
:1038D00006464088012818D1306900280CD0A9007C
:1038E000405801782D2910D0F368716809686A463C
:1038F0001160506010A205E0F368706800686946C6
:1039000021C115A23046FFF7C5FC7768FB68304639
:10391000294622469847012808D00AE0C368304665
:103920002946224698477F68012802D178680028F6
:10393000F4D103B0F0BDC04646534D3A252D38733F
:103940002053544154453A252D323873204556456D
:103950004E543A25730D0A0046534D3A252D3873BF
:103960002053544154453A252D323873204556454D
:103970004E543A25750D0A00F0B581B0002828D0C4
:103980001E460C460546079B06980090002068627C
:10399000A862E862104909886B8029800F4B1F6874
:1039A0006C60009BAB602B460C33C4C3A861E8611C
:1039B0002862481C0849088008480560002C08D087
:1039C0006C60002128460A46FFF77EFFA468002CA1
:1039D000F6D101B0F0BDC046B8CA010234C7010239
:1039E00002460020002A01D0D1627047C0437047D0
:1039F00010B582B004AC24881B881B041B196C46CC
:103A00002360024B00F0B0F802B010BDBD320000E0
:103A1000F0B597B01646029105464268002A30D0AC
:103A200001966A6001210024284616462246FFF7C7
:103A30004BFF3046029FBE4232D003A85021FCF714
:103A40008CFB32467268002F0CD003AF029811C76E
:103A50004068083F824209D0394608313C46002878
:103A60000F46F4D1002A019EDBD10AE0019E38689E
:103A70006860002128463246FFF726FF7F68002F46
:103A8000F5D102988468002C08D06C60002128468B
:103A90003246FFF719FFA468002CF6D117B0F0BD2D
:103AA00000212846019E3246FFF70EFFE9E700009D
:103AB000014600201F2901D9C043704718224A43FC
:103AC000344901238B5089188860704710B5002154
:103AD000CC4300280BD00A4A1368002B09D01832B7
:103AE000491C2029F8D306D106A0FFF7E7FE20469F
:103AF00010BD0123136001600024204610BDC046A4
:103B0000B8C7010274696D65722049442069732049
:103B100066756C6C0D0A0000264800687047C04648
:103B200070B520241B4D234E2868022817D1306819
:103B3000A968EA68401A904211D96969002907D03A
:103B40002879002807D0022028603068A86004E0A7
:103B50000120286003E00120286028698847183583
:103B6000641EE1D170BDC046F0B5044600201F2C94
:103B700001D9C043F0BD059D18266643054C0227B8
:103B8000A751A41921710B4909682646083626C693
:103B90006361F0BDB8C7010206480168491C0160B5
:103BA0000548416802680023521C02604B41436093
:103BB0007047C0466CAB010270AB010280B5FCF7E8
:103BC000CCFA80BDB0B50278002A24D0441C002174
:103BD000084601E0573A08E023460001D5B2302DEF
:103BE0000C4611D3392D02D8303A14460CE0412D41
:103BF0000C4609D3462D01D8373AF6E71446613C06
:103C0000E4B2062CE6D30024E2B280185C1C1A78D9
:103C1000002AE1D1B0BD0020B0BD10B502460120A0
:103C200000290DD00023D45C202C02D37F2C04D398
:103C300007E00D2C01D00A2C05D15B1C8B42F2D37E
:103C400010BD002010BD002010BD000081B0F0B5F7
:103C500084B0099300230393002800D1C2E0002A16
:103C600000D1BFE009AB03931678002E00D1A8E085
:103C70005623DB43009300231D46002900D1A2E018
:103C8000252E3FD1971C52781446643C0023142CF7
:103C900043D8C0467C4424796400A7440A99A3A36E
:103CA000A3A3A3A3A3A3A3A34CA3A3A3A3A3A3A33B
:103CB0005F000297039A131D039312680192012279
:103CC000002317461E460478FF0703D02D2C01D190
:103CD000164607E02746303F092F09D80A275F43D9
:103CE0003B19303B491E401C00270029EBD13946C7
:103CF000029A019C002C03D0012E00D15B4223606C
:103D00006B1C06E00378B3425BD1491E521C401C79
:103D10002B461678002EAFD164E02A2A62D13A7879
:103D20000378934204D0491E401C0029F8D1002199
:103D30006B1C3A46EDE7039A131D03933E78126815
:103D40000023C45CB44233D0491E5B1C0029F8D167
:103D50003C46C7180021002A2ED12EE00297039A74
:103D6000131D039312680023009E0778302F18D389
:103D70003A2F02D2344627340BE0612F03D3672F4A
:103D8000344606D30DE03C46413C052C09D8344668
:103D900020341B011B19DB19491E401C0029E4D1EA
:103DA0000021029C002A00D013606B1C2246B0E761
:103DB0003C46C718002A00D009C26B1C2246384670
:103DC000A7E700230EE0252E0BD15178652908D1F5
:103DD00003990A1D03920968002900D008606B1C32
:103DE00000E02B46184604B0F0BC02BC01B0084706
:103DF00081B010B581B00C46039303AB00930CF077
:103E000029FFA04200D3601E01B010BC02BC01B06B
:103E1000084770B504460020002A1BD0002C19D09A
:103E2000002B17D014600120022B13D32578002D0E
:103E300010D0641C01208D4205D1651E00262E7015
:103E400085005451401C984204D2661C2578002DF0
:103E50003446F0D170BDB0B504467821FCF788F93E
:103E6000002805D158212046FCF782F9002828D0E7
:103E70004278002A23D0841C0021084623460001F2
:103E8000D5B2302D0C4613D3392D01D8303A0EE07F
:103E9000412D0C460CD3462D01D8373A07E0144685
:103EA000613CE4B2062C01D3002401E0573A1446E9
:103EB000E2B280185C1C1A78002ADFD1B0BD002065
:103EC000B0BD2046FCF714FAB0BD70B5044600261C
:103ED000F043002C0DD00D4600290AD020461030AA
:103EE0000121FFF772FCA96820342046FFF76DFC22
:103EF000304670BD70B504460026F043002C0DD04E
:103F00000D4600290AD0204610300121FFF772FC2F
:103F1000A96820342046FFF76DFC304670BD70B5AF
:103F20000024002814D00546064610363046FFF718
:103F3000B3FC01280CD028462030FFF7ADFC012847
:103F400006D02C683046FFF798FC0C2141436418DA
:103F5000204670BDF0B583B000250295019500287C
:103F60001FD00C460646074610373846FFF79CFC24
:103F7000002816D13046203002AA01AB2146FFF7B7
:103F80004FFC00280DD135683846FFF778FC0C212E
:103F90004143B068029A101868506D186C6001981F
:103FA000A860284603B0F0BD70B505460C20584304
:103FB0000024904211D2121A461829606860AE603F
:103FC000EA60284610301946FFF75BFCE9682035A7
:103FD0002846FFF756FC204670BDE443204670BDDE
:103FE00004217046084204D0EFF30983EFF30882FE
:103FF00003E0EFF30883EFF309829BB004A8F0C05D
:1040000044464D4656465F4608A8F0C01846F0C8DC
:104010006846F0C018690C90202018440D9058692B
:104020000E9098690F90D8691090EFF3108011905E
:10403000EFF3148012900949086813900849086842
:104040001490084908681590074908681690179356
:1040500018927046199068460AF0E6FC04ED00E0FC
:104060000CED00E010ED00E014ED00E0F0B581B0E3
:10407000032600243046214607F06AF90425284625
:10408000214607F065F90127304639463A4607F0E0
:10409000F3F830462146324607F082F92846394681
:1040A0003A4607F0E9F802212846224607F078F957
:1040B00001B0F0BDF0B589B008900425284607F09E
:1040C000C3F80A27384605F0A7F9284607F0CCF8C8
:1040D0000324204607F0C0F807900526304605F077
:1040E0009BF9284607F0B0F8384605F095F92846C0
:1040F00007F0BAF8204607F0AFF80690304605F012
:104100008BF9284607F0A0F8384605F085F92846CF
:1041100007F0AAF8204607F09FF80590304605F012
:104120007BF9284607F090F8384605F075F92846DF
:1041300007F09AF8204607F08FF80490304605F013
:104140006BF9284607F080F8384605F065F92846EF
:1041500007F08AF8204607F07FF80390304605F014
:104160005BF9284607F070F83846019705F054F9D6
:10417000284607F079F8204607F06EF8029030469E
:1041800005F04AF9284607F05FF8384605F044F98B
:10419000284607F069F8204607F05EF807463046E3
:1041A00005F03AF9284607F04FF8019805F034F980
:1041B000284607F059F8204607F04EF804463046E6
:1041C00005F02AF9284607F03FF80699481E814174
:1041D0000A460799481E8141480080188000059AC8
:1041E000511E8A4151004018049A511E8A4180187C
:1041F0008000039A511E8A4151004018029A511EB4
:104200008A4180188000791E8F4179004018611E14
:104210008C4106190898002803D0032007F014F8F1
:1042200002E0032007F020F80A24204605F0F4F805
:104230000425284607F018F8204605F0EDF8284632
:1042400007F002F8F0B209B0F0BD70B504460420E2
:1042500006F0FAFF60B2002803D4032006F0F4FF52
:1042600002E0032007F000F80A25284605F0D4F8FC
:104270000426304606F0F8FF284605F0CDF8304613
:1042800006F0E2FF284605F0C7F8600603D40320D5
:1042900006F0DAFF02E0032006F0E6FF0A252846D2
:1042A00005F0BAF80426304606F0DEFF284605F091
:1042B000B3F8304606F0C8FF284605F0ADF8A00672
:1042C00003D4032006F0C0FF02E0032006F0CCFF79
:1042D0000A25284605F0A0F80426304606F0C4FF5B
:1042E000284605F099F8304606F0AEFF284605F05E
:1042F00093F8E00603D4032006F0A6FF02E00320B3
:1043000006F0B2FF0A25284605F086F80426304656
:1043100006F0AAFF284605F07FF8304606F094FF25
:10432000284605F079F8200703D4032006F08CFF17
:1043300002E0032006F098FF0A25284605F06CF8F5
:104340000426304606F090FF284605F065F8304612
:1043500006F07AFF284605F05FF8600703D40320D3
:1043600006F072FF02E0032006F07EFF0A252846D1
:1043700005F052F80426304606F076FF284605F090
:104380004BF8304606F060FF284605F045F8A007D8
:1043900003D4032006F058FF02E0032006F064FF78
:1043A0000A25284605F038F80426304606F05CFF5A
:1043B000284605F031F8304606F046FF284605F05D
:1043C0002BF8E00703D1032006F03EFF02E00320B4
:1043D00006F04AFF0A24204605F01EF80425284668
:1043E00006F042FF204605F017F8284606F02CFF9D
:1043F000204605F011F870BDF0B581B00326002508
:10440000012430462946224606F036FF304606F0A3
:104410002BFF0626304604F0FFFF042006F024FFA1
:10442000304604F0F9FF032006F016FF00281BD0E9
:10443000681CFA2D0546F6D30425284606F004FF2D
:104440000326304606F000FF0A27384604F0E4FF52
:10445000284606F009FF304606F006FF384604F00D
:10446000DBFF204601B0F0BD032001210A4606F023
:1044700003FF042006F0E8FE0024204601B0F0BD52
:10448000B0B50446C00703D1032006F0DDFE02E00C
:10449000032006F0E9FE0825284606F0E5FE28463A
:1044A00006F0D2FEA00703D4032006F0CDFE02E002
:1044B000032006F0D9FE0825284606F0D5FE28463A
:1044C00006F0C2FE600703D4032006F0BDFE02E042
:1044D000032006F0C9FE0825284606F0C5FE28463A
:1044E00006F0B2FE200703D4032006F0ADFE02E082
:1044F000032006F0B9FE0825284606F0B5FE28463A
:1045000006F0A2FEE00603D4032006F09DFE02E0C2
:10451000032006F0A9FE0825284606F0A5FE284639
:1045200006F092FEA00603D4032006F08DFE02E002
:10453000032006F099FE0825284606F095FE284639
:1045400006F082FE600603D4032006F07DFE02E042
:10455000032006F089FE0825284606F085FE284639
:1045600006F072FE60B2002803D4032006F06CFE51
:1045700002E0032006F078FE0824204606F074FED0
:10458000204606F061FE0724204606F06DFE204618
:1045900006F05AFEB0BDF0B581B0032700243846BE
:1045A000214606F0C5FE3846214606F0D1FE01251B
:1045B00038462946224606F05FFE0526384629463B
:1045C000324606F0EDFE08273846214606F0C0FECA
:1045D00038462946224606F04FFE384629463246DE
:1045E00006F0DEFE07273846214606F0B1FE3846C3
:1045F0002946224606F040FE38462946324606F055
:10460000CFFE01B0F0BD000080B50B2006F024FE07
:1046100012490A78002804D0002A12D003F0C4F806
:1046200080BD012AFAD1002008700F49C8830C49C7
:1046300008700C48012101700BF054F903F0B4F834
:1046400080BD0748012202700A70064800210170EF
:104650000BF06CF903F0A8F880BDC0461C90010275
:10466000189001021990010212A701020248406944
:10467000811E484248417047F095010280B5FDF720
:1046800011FB002801D00020C04380BD80B5FEF79B
:10469000BFFB80BD10B504480F2100242246FFF760
:1046A00013F9204610BDC046DC980102F0B581B078
:1046B00007460324204606F0D7FD0425284606F0C9
:1046C000D3FD204606F0C0FD0A26304604F0A4FEC5
:1046D000284606F0B9FD3220FFF7B7FDFFF78CFE44
:1046E000F8B2FFF7B2FDFFF787FE204606F0BCFDEB
:1046F000284606F0B9FD204606F0A6FD304604F037
:104700008BFE284606F0A0FD3320FFF79EFDFFF745
:1047100073FE0020FFF7CEFC0746284606F094FD06
:10472000204606F091FD304604F076FE284606F05D
:104730009BFD204606F098FD304604F06DFE38469D
:1047400001B0F0BDF0B581B00091074603242046CA
:1047500006F08AFD0426304606F086FD204606F067
:1047600073FD0A25284604F057FE304606F06CFD1E
:104770003220FFF76AFDFFF73FFEF8B2FFF765FD55
:10478000FFF73AFE0098FFF760FDFFF735FE304671
:1047900006F05AFD204606F057FD284604F03CFE80
:1047A000304606F061FD204606F05EFD284604F026
:1047B00033FE284604F030FE01B0F0BD80B5074856
:1047C00001210170064802680A4302600548026838
:1047D000002A02D000200146904780BDBECA0102D7
:1047E0001C100050C0CA0102F0B599B0F548017B19
:1047F000C67A427B0E92F44C221F1368F34A126869
:10480000069242780C9202790592C76A04931F407F
:1048100001200F907A0200D5BCE03A0200D5BFE03B
:10482000FA0102D50F9802062260502508968A19CF
:104830001826BB0102D50F98430623604123079534
:1048400069430A96354655431426FC0210D50F9845
:10485000040538463746DC4E3460DA4CA469B4644B
:10486000D84CE4697464DA4C241D34603E46074633
:1048700090000B90D8040D90681809900E9B73431C
:104880000F988203B902D04D22D50F9841052960B7
:10489000CC480E961646024681692965C16969654C
:1048A00009990D9801430898000108180B994018C0
:1048B000C018C849098892794A4380180A301C46B2
:1048C00005F08AF8234632460E9EC04988672A6062
:1048D0000F98C404380300D52C60F80302D50F9854
:1048E000000428600F984104B80300D529603804FB
:1048F00000D4E4E1039402910E9308920D980B9971
:104900000C180A980C9941430C910F98C0030B9016
:10491000286007F0ADFE002801D005F03FF80C98A4
:10492000005B410B43D1099800190E994018059975
:10493000090140180E90E74D287B079B4343E97A15
:104940000A010D9C2243D21841188B00D2180A9BF1
:104950004B43D1186A7B564389190E9E2A79101849
:10496000DF4A12884243881816903068C000800DD4
:1049700010A9C882002511957079C0077ED110A8B2
:104980000F998182069C00940020E8A2049B0AF003
:104990008DFE78E00F98820522603A0200D43FE74E
:1049A0000F98C2052260FA0100D53BE73DE70721D9
:1049B00049030840032149038842089A00D07EE158
:1049C000069707F0ABFA0020169009901590C14C9D
:1049D000E07A217B08180A99414380000D9A104320
:1049E0004118627B0E9672438A186178A379079EFC
:1049F0007343D718FA683F26324063789A420C977F
:104A00006ED105960A9A4A4380580F210A07024040
:104A10000398401EC04B1B68DB0903409818109098
:104A20000F98C0020B90B868800767D42C46283CCA
:104A300009F0B2FD05462068000609D5C3208401AF
:104A4000786A400704D409F0A7FD401BA042F7D9BB
:104A500005980002B96849080140B34803688268B4
:104A6000B868C40C20202040DB0700D095E000236C
:104A700010221D461C460E9E0B9FB1E010A8858299
:104A8000B0681190069C701D924B1979E20707D10E
:104A9000491C1971D97A1A798A4202D31D7100E032
:104AA000D97001784278120251188278120489185C
:104AB00003229143017035715878401C5870D87AA0
:104AC000197B08185978884200D85D70D879401E43
:104AD000D871596B002901D010A888477E4DEDE0B0
:104AE00010A80B998182F86830406378009000200C
:104AF0007CA20F990AF0DAFD0E9E94E0388A874A6C
:104B0000024010A8C2822022BA5C9307DB0F3C68E7
:104B1000C3720F9B1A4082726205D20C0D9B1A431E
:104B20001692FA68130E0372BB69FC697C4D2D68FE
:104B30002D0C05745204920F427211931394654C1C
:104B4000A07B002809980E9E0B9F5FD075480068D7
:104B5000007A0328099859D00C98007D084009284C
:104B6000099853D1C320840109F016FD05460C981D
:104B7000406A41070BD4594909680906890F06D1D3
:104B800009F00AFD401BA042F1D90C98406A41038C
:104B90000898884310A9888237E0D2070E9E0B9FA1
:104BA00003D108230022154619E00C9B9A68029C49
:104BB000224211D19A68520C0224944300221346D7
:104BC00015460DE0C4CF010228A000503CA10050C2
:104BD000FC1F0000C0CF010204250022134614462A
:104BE0000843104318432843204310A988823842C1
:104BF0000BD10C9B198A494A0A4010A9CA8219682C
:104C00004905C90C0D9A11431691324C2921615C5A
:104C1000002908D03037B84205D010A90846113015
:104C2000123109F015F8E77A2A48047BE51929487A
:104C300000790E9027484078401C2946FBF74AFA35
:104C400088000D9A1043189007996143380110436A
:104C500040182049497B4E4380191C216943401864
:104C60000E9909191B4B1E4A12884A438018179047
:104C7000099A0C998A60987B002800D04A6298793A
:104C8000401C9871187B99798142069F00D39A71D4
:104C90005978491C5970D97A0818597888420E4DAC
:104CA00000D85A70187A401E18722820185C002804
:104CB00004D0996B002901D010A88847089A1742A0
:104CC00002D00F98000328601C480449486019B0BE
:104CD000F0BDC046C4CF010228A000503CA1005046
:104CE000C0CF0102485720455420696478202564CC
:104CF00020616E6420455420696478202564206911
:104D00006E2052582064657363206D69736D617401
:104D100063680D0A0000000038200040FF03000017
:104D2000943000402C940102604000404D414320EB
:104D30004556542025782025780D0A00FFFFFF03F3
:104D4000F0B5A5B01E460C9208910024239422A928
:104D50000C8016A90C8024A909250D80598C0D9171
:104D6000FBF7B8F92A99012900D0DFE03189012940
:104D700000D0DBE0318C012900D0D7E00D9900296B
:104D800000D1D3E0224607962C990B912B990691DE
:104D900080B205900F9415A8058090000E900C9994
:104DA0000C582E460025204629461746FBF714FDD1
:104DB0000028119636D12C200A97784308990818B4
:104DC00017A90A4668C868C2E8C8E8C2E8C8E8C2C5
:104DD000079F119880B280000E5822AD019523A83C
:104DE000009020463946059A069B04F023FB0F9855
:104DF000401C0F90288800282DD03B8A239913ACA3
:104E0000039416A8029014A8019015AE009617A856
:104E100024AA04F0E9FC2588308811900120149E12
:104E20000A9A05E013A8058014952E4628463A46AE
:104E30000E9F51000B9B119C5C52591808830D84E6
:104E4000D81986600F981885521C0D9882426DD033
:104E500024A805889FE7099616A8002505801495C3
:104E600024A80688239812902F46109503E06D1C05
:104E7000A8B2B04213D8A8B2800017A90C58204697
:104E80001299FBF7B7FC0028F1D1002FEFD115A83C
:104E9000058016A80127078014941094E7E715A849
:104EA0000288B01A012805D115A80680099F149719
:104EB000119628E010200799095E0129119221DB43
:104EC000551CA8B20C18109F0E9B099403E06D1C92
:104ED000A8B2844218DDAAB2B242F8D8800017AA5C
:104EE00010581090394634461E46FBF775FC334681
:104EF0002646099C0028EAD115A80580109F149722
:104F00001195E4E7109F0E9B1C463E4638461299C9
:104F1000FBF791FAFBF7F0FC0546052800D30525C1
:104F200013A8058001200A9A274682E725B0F0BD24
:104F3000F0B58BB00243159A149C139E2BD00546F6
:104F400001A856C0129CD869196A09900A911E4698
:104F50009F6B0123009309A807AA0146059306F059
:104F600045FA716C3846FBF766FA0746E06A616BF2
:104F7000FBF761FA002D069613D0044611980199AB
:104F8000012924D10921081A0421069A515E884278
:104F900029D16425B1E000203080207010700BB062
:104FA000F0BDB08800226425002829D00592694907
:104FB0003846FBF73BFC0028049C039E6FD16649F2
:104FC0003846FBF733FC00281DD05A2567E03C2506
:104FD000082800D191E05F492046FBF727FC002814
:104FE00019D0502589E00A291DDB1D293BDC5949D0
:104FF0003846FBF71BFC0022002854D05A253AE023
:105000003346049C39E055493846FBF70FFC00282D
:1050100021D0502543E050492046FBF707FC0028EB
:105020002ED0462569E03C25012866D04949204616
:10503000FBF7FCFB0028D4D147492046FBF7F6FBE1
:105040000028EED145492046FBF7F0FB002854D15B
:10505000434920466EE042493846FBF7E7FB00280B
:105060001CD128251BE03B493846FBF7DFFB00221B
:10507000002832D05025049C069B0299039E41E0F3
:1050800036492046FBF7D2FB002836D1344920466A
:10509000FBF7CCFB00282FD114252EE037250299F1
:1050A000059A069B2EE005922B493846FBF7BEFB7E
:1050B000002896D129493846FBF7B8FB0028B0D123
:1050C00027493846FBF7B2FB0028049C069B02994F
:1050D000039E059A3BD11E2514E005921E493846D1
:1050E000FBF7A4FB00289CD11C493846FBF79EFB2C
:1050F00000281DD03C2500E02325049C069B029936
:10510000039E059A258032700020087030780028B0
:105110000CD118681349FBF77BFB002806D12088C7
:10512000102803D30F3820800BB0F0BD0BB0F0BDBA
:105130000B493846FBF77AFB0028049C069B029932
:10514000039E059A01D11425DCE72325DAE72D25F6
:10515000D8E7C046CDCCCC3DCDCC4C3DCDCCCC3C25
:105160000AD7233C0000204070B588B00C460646A4
:105170004088002820D0FBF796FB059005A804A9DD
:1051800001252A4606F09CFB3088B188081AFBF7F7
:105190007FFB0390049903A807AA2B4606F050FB57
:1051A0005249079D2846FBF741FB002808D0BF2045
:1051B0000006206008B070BD0020206008B070BDFF
:1051C0004B492846FBF716FB002804D03F20000679
:1051D000206008B070BD47492846FBF727FB002830
:1051E00001D0002010E000212846FBF71FFB00281B
:1051F00001D0022008E040492846FBF717FB0028B1
:1052000001D0042000E0062001957F21C90502910C
:1052100080003A49091801A806AA022306F0C4FA38
:105220000698206008B070BDF0B587B00C46054602
:105230004768002638463146FBF706FB002802D0B7
:10524000266007B0F0BD049704A803A901263246E2
:1052500006F036FBA8682968FBF7A8F802900399C6
:1052600002A806AA334606F0EBFA2049069D284616
:10527000FBF7DCFA002804D0BF200606266007B042
:10528000F0BD1B492846FBF7B5FA002804D03F20A3
:105290000606266007B0F0BD16492846FBF7C6FA99
:1052A000002801D0002010E000212846FBF7BEFABC
:1052B000002801D0022008E00F492846FBF7B6FA83
:1052C000002801D0042000E0062000957F21C905B8
:1052D0000191800009490918684605AA022306F0D1
:1052E00063FA059E266007B0F0BDC046CDCC0C3FEA
:1052F000295C0FBFCDCC4C3ECDCC4CBE34940102CA
:10530000F0B587B00C4606467F270088002801D0FC
:10531000FD0503E0B08800282ED0334DFBF7C3FA1B
:1053200003907088FBF7BFFA049003A802A9012636
:10533000324606F0C5FA029904A806AA334606F0DA
:105340007FFA2A49069E3046FBF770FA002802D001
:105350003F20010641E026493046FBF74BFA002882
:1053600002D0BF20010638E022493046FBF75EFA42
:10537000002805D0002024E00020206007B0F0BD08
:105380001D493046FBF752FA002801D0022018E0F0
:105390001A493046FBF74AFA002801D0042010E0F1
:1053A00017493046FBF742FA002801D0062008E0F2
:1053B00014493046FBF73AFA002801D0082000E0F3
:1053C0000A200096F905019180000F4909186846E6
:1053D00005AA022306F0E8F905992846FAF7EEFF38
:1053E000206007B0F0BDC046000080BF0000384319
:1053F0003333733F0000C842000070420000204277
:105400000000A0410000C04054940102F0B59DB0DE
:1054100015460B917F210391C9051C9102911B91A7
:1054200019A900248C80199418941794598C06910A
:10543000198C0F91DE8B998B0791997805911F88B4
:105440002B21CA432799914201DB7F0015E04022BE
:10545000D243914211DC4922D243914202DB7908C6
:10546000CF190AE05322D2439142EEDA5D22D243B1
:10547000914201DBBF0000E0FF000A971396269ED1
:10548000597E00290BD0002132460F46D170917011
:1054900051701170121D7F1C5C7EA742F6D30C93D5
:1054A00011952599149122990D91159041088C42DE
:1054B00011D2FD4A2346A00084583454270A451CC3
:1054C0007755250C871CF555240EC01C34545B1CE5
:1054D0009CB2A142EFD8239810900120099000902F
:1054E00030463146149A159F3B4605F08DFF0D98C6
:1054F00000060890400E139D00D186E068000490DD
:10550000002F3FD0002210461146144606E01C46EC
:105510001146159F401C82B2BA420ED283B2AB42F2
:10552000F8D09200149B9A5E0FB2BA42034600DC98
:105530002346BA42EBDC0A46E9E7002F25D00022D9
:1055400010461146129206E012931146159F401C18
:1055500082B2BA4214D283B2AB42F8D0A5B2AB4207
:105560000CD09200149B9A5E0FB2BA42034600DC44
:10557000129BBA42139DE7DC0A46E5E7139DE6E776
:10558000129903E00024214600E0002112911098B6
:105590000183C4828582049FF057FBF779F9792152
:1055A000C9050E91FAF70AFF1099C86109980743D7
:1055B000F057FBF76DF90E99FAF700FF109F38626C
:1055C0002004C40B3057FBF763F90E99FAF7F6FE87
:1055D0007862601C3056FBF75BF90E9C2146FAF7A7
:1055E000EDFEB86212980004C70BF057FBF750F9B4
:1055F0002146FAF7E3FE109CE062781C3056FBF778
:1056000047F90E99FAF7DAFE2063119805800C9895
:10561000407E410000278D4228463A46149E1ED304
:105620000A9880B28AB29300F45E84420BDA491C75
:105630008AB2AA42F6D9002728463A4681B2691AA8
:10564000012910D01BE0F018119B1980078808046D
:105650000FD0500040008019001F0288084681B218
:10566000691A01290BD1A800301811990D800788FB
:1056700026E00020024681B2691A0129F3D00A9976
:1056800089B2079B4B43BB421AD306998A4217D86B
:105690000599002914D0401C82B2891803E0401CEF
:1056A00082B291420CD983B2AB42F8D89200B35E79
:1056B000BCB2A342F3DDB218119B18801788EEE745
:1056C00012970B980580119800882B1A002B16DD75
:1056D00002210F9A1143032942D10E93411C421E0D
:1056E00010B281420EDA0E98032824DB0C98808CCD
:1056F000012820D019A818A9FFF736FD1FE00020C7
:1057000018902BE00026F443374608E0B8B240007A
:1057100019AD2B527F1C521C10B28142E3DB13B235
:10572000A3423346F2DD159B98423346EEDA800001
:10573000149B1B5AEAE719A818A9FFF7E1FD149E6C
:10574000139D0F9A012A13D0032A11D0022A04D1E3
:1057500011980088281A02280ADA0020179034E0ED
:10576000022A01D1022BB8DA00201890012AEBD1CD
:10577000681C691E0FB2B84208DA0C98808C0128A8
:105780001DD119A817A9FFF7BBFD1CE00022D343C8
:10579000144608E0A5B26D0019AF7E53641C491C85
:1057A0000FB2B842E9DB0DB29D421646F2DD159DFF
:1057B000AF421646EEDABD00149E765BEAE719A802
:1057C00017A9FFF7D1FC149E139D249F189C1799CD
:1057D0002046FAF7EBFD0F99012900D820463860E2
:1057E0000D98002800D1CBE011990888109FB88649
:1057F0000888281AB880129880B2FBF754F87921EB
:10580000CC052146FAF7DAFD2146FAF7D7FDB86351
:10581000119F3888002849D081008919091F0988FB
:10582000129C0C191599884203D280008019808837
:10583000041915984300534916AA304605F0C2FFD3
:10584000169810994864FBF770F8A4B2A04201D1F1
:105850004D480FE0001BFBF726F81C901CA81BA965
:10586000012206F02DF82046FBF71DF801461B9893
:10587000FAF7A4FD109908603988491B4A1C92B2B6
:10588000032A02D20021159F17E009B20229159FB1
:1058900012DB3F210906FAF7C9FF002802990CD153
:1058A0000998810709E0C046402100400020129C71
:1058B00015998842B9D3BCE734491098016108981A
:1058C000800E5DD0002F1CD00022114614461046D9
:1058D0004B1B1DB2ED135B196B40139D1BB2920065
:1058E000B25E53431818A418491C8AB2BA42EFD3C7
:1058F000FAF7D9FF06462046FAF7D5FF002C03D168
:1059000000E000260398C0051C901CA81BA90125D7
:105910002A4605F0D5FF1B9C20463146FAF74EFD7E
:10592000014610988160002F119422D00024274650
:10593000264613951291B8B2FAF7B5FF1299FAF705
:1059400035FD0546A0001499085EFAF7A1FF01464F
:105950001398C00785432846FAF730FD01463046C4
:10596000FAF7D3FC06467F1CBCB215988442E2D3FA
:1059700000E0002611983146FAF720FD1099C86022
:105980001DB0F0BD10A50102000020410000404004
:10599000F0B58FB00692F74A09AF70CA70C770CAE7
:1059A00070C70328079320D88800F3A10858F64948
:1059B000FAF7ABFC0446F549FAF7A7FC0D90F44959
:1059C0002046FAF7A2FC0C90F2492046FAF79DFC1B
:1059D0000B90F1492046FAF798FC0A90EF492046CF
:1059E000FAF793FC0990EE4969E0042822D00628D2
:1059F00020D88800EBA10858EE49FAF786FC044647
:105A0000ED49FAF782FC0D90EC492046FAF77DFC4F
:105A10000C90EB492046FAF778FC0B90E9492046B8
:105A2000FAF773FC0A90E8492046FAF76EFC0990F1
:105A3000FD4944E00838022821D88800FBA1085815
:105A4000D149FAF762FC0446FC49FAF75EFC0D9076
:105A5000FB492046FAF759FC0C90FF2081052046AF
:105A6000FAF753FC0B90F7492046FAF74EFC0A90E0
:105A7000CA492046FAF749FC0990FE491FE0880010
:105A8000F1A10858F449FAF740FC0446F349FAF743
:105A90003CFC0D90F2492046FAF737FC0C90F14996
:105AA0002046FAF732FC0B90EF492046FAF72DFC1E
:105AB0000A90EE492046FAF728FC0990EC49009438
:105AC0002046FAF722FCEC4909680E90EB4804687E
:105AD000EB4801684808EB4F05463D400022002D89
:105AE00008922DD0CA01120E07D0280CE90D12D150
:105AF0004000E649085AE6490AE0C903090E0CD0FD
:105B0000280AE90B10D14000E049085A8F2189008A
:105B10004018E4300DE0DC490AE081B27F2905D865
:105B20004800DA49085A04E0D94901E08F21890088
:105B3000401800B2FAF7ACFED649FAF73FFC02462D
:105B40000292039507252606D34B1A68002A089867
:105B500040D0791C8A420BD21102090E13D0110CCD
:105B60001F46D00D1FD14800C849085AC84907E050
:105B70001F46110E002A13D44800C449085AC249CE
:105B80004018E4301FE011041F46090E0ED0110A20
:105B9000D00B12D14800BD49085A8F218900EFE788
:105BA000BE4808180FE0B84808180CE091B27F29E9
:105BB00006D84800B549085A05E0B548081802E07B
:105BC0008F218900501800B2FAF762FEB149FAF746
:105BD000F5FB3B460590159F2C40F50E5B69B049DF
:105BE0001940089810D0DA02D20E34D0C80B3E21EA
:105BF0000140A648405AA6494018E43000B2FAF7DE
:105C000047FEA449FAF7DAFB0490149E6800A5A1A8
:105C1000085EFAF73DFE0146A00009AA1058FAF7FF
:105C200074FB0146B8B20128089F019102D1022CF1
:105C30000AD9A74F052C24D1189808900C2D20D8EC
:105C40000B2D16D3A44918E00027022C089718D072
:105C50008120C70515E01A04120E00D1CAE0080A17
:105C6000C90B00D0CDE040008849085A8F21890037
:105C7000C2E7092D00D2C7E096490898FAF745FB1C
:105C8000089001200021B542034600D30B46052CA5
:105C900000D308461799169A1A9C199D1843069B1B
:105CA000012B12D1079B402B22D1002840D038462F
:105CB000FAF72BFB01460198FAF727FB01460098FB
:105CC000FAF774FB059A04998AE0079B402B1FD1D1
:105CD000002838D03846FAF718FB01460198FAF741
:105CE00014FB01460098FAF761FB059A049977E0E6
:105CF000002833D03846FAF708FB01460198FAF736
:105D000004FB01460098FAF751FB059A049967E0F5
:105D100000285BD03846FAF7F8FA01460198FAF7FE
:105D2000F4FA01460098FAF741FB059A049957E006
:105D300002981146FAF73AFB0399002900D1674807
:105D4000059A04994CE002981146FAF72FFB039943
:105D5000002900D16148059A049941E00298114652
:105D6000FAF724FB0399002900D15C48059A0499AD
:105D700036E0C046CC160100000068C1000088C1B2
:105D800066665EC1000084C1000084410000B44129
:105D900000004841000020400000F0C0000084C125
:105DA0000000F841333323C1000050C19A9929C142
:105DB0009A9949C19A9949413333CB4166667641F4
:105DC000CDCCAC40333393C09A9949C10298114667
:105DD000FAF7ECFA0399002900D14048059A049992
:105DE00028601046FAF7E2FA0899FAF7DFFA20601D
:105DF0000FB0F0BD99B27F2911D848002349085A45
:105E0000FCE623494018F9E6C12001060898FAF794
:105E10007CFA0890062D00D933E7002030E78F2167
:105E200089005818EAE6C0463333F341000058C1F0
:105E30009A9961C19A9969C1000084C10000AC417E
:105E400000003841000008C1CDCC80C1CDCC88C154
:105E500033338FC1333397C133339741CDCC8C412A
:105E60003333F3409A9919C0666646C1333397C1FC
:105E7000CDCCB4410000D4410C0000405030004073
:105E800068400040FFFFFF007C080000D41A0100BA
:105E90005C050000919AF63C642000409C0B0000D9
:105EA000FFFF1F00FAFFFCFFFEFF000002000400DE
:105EB000060008000A000C000E001000120014007A
:105EC000160018001A001C001E00200022002400EA
:105ED000000080BF0000A0C0000040C00000DCC285
:105EE000F0B5FFB0ECB017460E460D900021E991D9
:105EF000E891DC91999198919791969114911391D1
:105F000012919AA8F49DF39CF29A002E00D1E6E13A
:105F10000B938030F09B1180099529602546DBACFE
:105F2000218095AC21800C952980DA917F24E405AD
:105F3000B994B894B794B694B594B494B394B29415
:105F4000B194B094AF94AE94AD94AC94AB94AA9445
:105F5000A994A894A794A694A594A494A394A29475
:105F6000A194A0949F949E949D949C949B949A94A5
:105F7000046644668466C466046744678467C467CD
:105F8000046444648464C464046544658465C465CD
:105F9000046244628462C462046344638463C463CD
:105FA000046044608460C460046144618461C461CD
:105FB000B0090B250B2800D3AE011095012B0B9DCA
:105FC00000D070E12B89012B00D06CE1298C0029D5
:105FD0000E9200D18BE16B8C002B00D1FAE1AA8CE0
:105FE0003021695C002900D188E10892109F5F434D
:105FF0001196304639460F93FAF76CF80590FAF788
:1060000047FC01462046FAF716FA8321C905FAF73C
:10601000D5F9064696A8021D119887420A9200D823
:1060200079E155A811909AA9069196AF15463A467E
:10603000059C234605F0B8FB15A80F9006992A4643
:10604000234605F0B1FB02230D93384631463A460C
:1060500005F0F6FB012308930093E8AA1092384656
:10606000394605F0C3F9E898DD901198069D294658
:106070003A46234605F098FB0F9829460A9A23468C
:1060800005F092FB384631463A460D9B05F0D8FBA9
:10609000089B009338463946109A05F0A7F9E8980E
:1060A000DE9011982C4629463A46059D2B4605F070
:1060B0007BFB0F9821460A9A2C462B4605F074FB71
:1060C000384631463A460D9B05F0BAFB089B0093D3
:1060D00038463946109A05F089F9E898DF9011980A
:1060E000069D29463A46234605F05EFB0F98294651
:1060F0000A9A2346254605F057FB384631463A466C
:106100000D9B05F09DFB089B009338463946109A7D
:1061100005F06CF9E898E0901198069C21463A4603
:106120002B4605F041FB0F9821460A9A2C462B4638
:1061300005F03AFB384631463A460D9B05F080FBA8
:10614000089B009338463946109A05F04FF9E898B5
:10615000E1901198069D29463A46234605F024FB16
:106160000F9829460A9A2346254605F01DFB384616
:1061700031463A460D9B05F063FB089B0093384679
:106180003946109A05F032F9E898E2901198069C89
:1061900021463A462B4605F007FB0F9821460A9AFE
:1061A0002B4605F001FB384631463A460D9B05F07B
:1061B00047FB089B009338463946109A05F016F9BC
:1061C000E898E390119821463A462B4605F0ECFA00
:1061D0000F9821460A9A2B462C4605F0E5FA3846D8
:1061E00031463A460D9B05F02BFB089B0093384641
:1061F0003946109A05F0FAF8E898E4901198069D4F
:1062000029463A46234605F0CFFA0F9829460A9ABE
:106210002546234605F0C8FA384631463A460D9BD6
:1062200005F00EFB089B009338463946109A05F09E
:10623000DDF8E898E5901198069C21463A462B46F1
:1062400005F0B2FA0F9821460A9A2B4605F0ACFAEF
:10625000384631463A460D9B05F0F2FA089B00930A
:1062600038463946109A05F0C1F8E898E69011983A
:1062700021463A462B4605F097FA0F9821460A9A8E
:106280002B4605F091FA384631463A460D9B05F00B
:10629000D7FA089B009338463946109A05F0A6F8BD
:1062A000E898E7907AE010880C9A1080999198917C
:1062B000DA9E08460F46099DF59CFAF777F82860A4
:1062C000DC9827606060A6600C34DDA80EC80EC4A0
:1062D0002EC82EC42EC82EC47FB06CB0F0BDFF20D7
:1062E00010800021296020807FB06CB0F0BD0022BA
:1062F00001233021695C002900D076E6DDAA1ACF9F
:106300001AC23ACF3AC23ACF3AC20B213046F9F715
:10631000E1FE054642E000200690059D0796089F95
:106320001190069801460D9C0F9A4A43D219109B72
:106330005A43119BD218D200A35889002E4655AD5E
:106340006B503546121DA25815AB5A50401C01B275
:106350008E42E9DC55A89AAE96AC314622462B46D1
:1063600005F022FA15A831460A9A2B4605F01CFAC8
:10637000022320460799224605F062FA0123009382
:10638000E8AA2046214605F031F8119B9800DDA9C6
:10639000E89A0A505B1C0B2B1846C1D1F19EDDA870
:1063A0009AA9DCAA0B2305F0FFF909210E980F9199
:1063B00001800B98C168DC9C2046F9F7FFFF01467D
:1063C000A8B2E69F0F281BD808280DD30846F9F776
:1063D0009CFF14E0FF2010800021099A11600C99A5
:1063E00008807FB06CB0F0BD042803D3812208463A
:1063F000D10502E0412208461106F9F7DFFF014608
:106400002B20C04386420D9704DB0846F9F77DFF39
:10641000014603E04020C043864244DD0E9A0C9CB6
:106420000B98408A002811D00B98038A95A80390F6
:10643000DBA80290DAA801900094DDA80D4603F0D5
:10644000D3F929462488DA9E099D68E011910F98B6
:10645000208000273D46109705E00E9804887F1C99
:10646000B8B2A04211D8B8B28000DDA90C582046BD
:106470001199FAF7BFF90028EFD1002DEDD10C9852
:10648000078001250F971094E7E7DBA805800F9A96
:1064900090B2201A012811D10C9804800D9FDA9730
:1064A0003E46099D3AE04920C043864200DA8BE02F
:1064B000FF2208469105F9F781FFA9E710200B9903
:1064C0000E5E012E00DA90E0551CABB21846A1B268
:1064D000AAB28A4217D805E00E990C88A1B2AAB2D6
:1064E0008A4210D88000DDA90C58204610991F461A
:1064F000FAF772F93B46002805D10C9805800B98F5
:10650000068A0F95109430B2C1186D1CA8B2814252
:10651000E2DC109EDA960F9C099D0D9F1199304682
:10652000F9F789FFFAF7E8F9052800D3052095A9BE
:106530000880A0B20E990988814218D9401C611EBA
:106540000CB2A04218DA12A898A9FEF76DFE0E98B8
:106550000188481C491E0CB2A04221DA12A899A950
:10656000FEF762FE99999898099D0D9FA4E6002177
:106570009891999108469FE60022134608E09CB244
:10658000A40012AF3D515B1C491C0CB2A042DADBE7
:106590008DB20A2D1546F2D8A400DDAD2D59EEE7D7
:1065A0000022134608E09CB2A40012AF3D515B1CD0
:1065B000491C0CB2A042D1DB8DB20A2D1546F2D88F
:1065C000A400DDAD2D59EEE75320C043864200DB29
:1065D0001BE70E460B9881692046FAF7FDF8002864
:1065E0000C9C08D10B98808B07E01446099D0D9FE9
:1065F0001199109E93E70B98C08BFAF754F9014656
:106600003046F9F7DBFE119021E70000F0B58BB0C2
:106610001C4609930E46034600200A904048008815
:10662000224F05970AA9049103940292109C0194A9
:10663000012500950B21414389B230331C4A304675
:10664000FFF74EFC3868079078680890B8680690A5
:1066500033480088334F009501940297324E30360C
:106660003249334A3346FEF76BFB0698F8620798C7
:10667000386308987863099800882E4905912E4957
:1066800004912E4903910297019000962C4B2846C5
:1066900029462A46FEF74CFC432001060A98F9F7E2
:1066A0008DFEFAF729F90BB0F0BDC046D8A401025F
:1066B00094DC0102F0B589B00F9F0E9C002815D024
:1066C0001098079016480088164E012500950191F4
:1066D00002960893144B30331449154AFEF730FBE9
:1066E000089BF76207983063746303E00D484763C3
:1066F000C462002518880F4905910F4904910F497C
:10670000039108490291019007483030009001211F
:106710000B4B28460A46FEF70BFC09B0F0BDC046FD
:106720007CAB010258D101023C9E01028C9D01020A
:1067300000D0010208A2010278AB010218AB0102ED
:1067400020AB01023048704700487047BCAB0102E3
:10675000800037490918C86B0022CA637047C046D9
:10676000800033490918886C00228A647047C0464B
:1067700080B52F4AD369002B01D0126A98470020B8
:1067800080BDC0460249087800220A707047C046A2
:106790002CC701020020704780B5182905D8034690
:1067A0008A1E03481946F9F7BFFC002080BDC04689
:1067B00080AB0102B0B502460020022901D2C043DD
:1067C000B0BD8C1E0F2C07D8044D2846114622461A
:1067D000F9F7AAFC00202855B0BDC0469CAB0102C9
:1067E000B0B502460020022901D2C043B0BD8C1EC4
:1067F0000F2C07D8044D284611462246F9F794FC81
:1068000000202855B0BDC046ACAB0102084908784D
:1068100000220A707047C046B0B50446044DAA680D
:10682000002A02D0E968204690472C610020B0BDC4
:1068300048970102B0B5D64D286A002819D02848DB
:10684000007800281BD0012829D127480068CF49AB
:106850008A8A904224DA2878002804D00020287000
:10686000022001F0DBFE0020687068621D4908709C
:10687000B0BD0020686268701A490870B0BD287801
:10688000002803D10120287001F0C8FE154801211D
:106890000170002068626970C04313490860B0BD90
:1068A00001246C706A6A531C6B62C98A884209DDD4
:1068B000132AF4DB287800280DD12C70204601F033
:1068C000ADFE08E0132AEADB2878002803D12C70FB
:1068D000204601F0A3FE0020686202480470B0BDAB
:1068E00038960102359601025C96010280B5124885
:1068F00001681F220A40026003200840022812D1CA
:106900000E480268D30D02D0FF231B06D2180C4B91
:106910001A600C4A12680C4B1A6080680B4A10808F
:10692000000C0B4A10801A488268002A02D0826844
:106930000020904780BDC046742000406440004065
:1069400014D001027830004018D00102A09E01024C
:106950004ED1010280B50D48016889070FD5052188
:1069600001600B48C178002908D00021C170C168BE
:10697000002903D0C26841680020904780BD0548C7
:1069800005A10B4A0BA307F035FEC0462C040040BE
:106990001C940102383401005048595F54494D4558
:1069A000525F49525148616E646C6572000000008C
:1069B0008D0A0000556E65787065637465642069A2
:1069C0006E746572727570740000000070B50446D4
:1069D000401E012814D80320084011D13F20400355
:1069E0000818050B281980280AD8164E317801207E
:1069F0004840294603F052FE641E6D1C002CF5D160
:106A000070BDC04680B50020014603F08FFB002812
:106A100000D080BD0B480121017080BD70B51646C5
:106A20000C460546FF22F9F791FB05483118054849
:106A30000278012050402A46234603F0D7FC70BD5F
:106A400000E0070410A701020120000370470120A5
:106A500040037047F0B585B04A484B49016005F0E6
:106A60005BFD4A4EF08A5221494F7852B18A50223A
:106A7000B952B48D4022BC52B388FB62B27A3A71EB
:106A8000B2893A827982B8820493BB877D20C5009F
:106A9000F1882846F9F71EFBF881601E84416000EA
:106AA0003862B08B3B2801D83C20B0830020F083B3
:106AB000308B384908802120C0007080728C0F20F4
:106AC00011460140130B6B435B1811050C0F642139
:106AD0004C431B191206140F0A2254431B192E4C47
:106AE0002380B38C1C4604401F0B6F433C191F05C9
:106AF0003F0F4F43E4191B061B0F5343E318274C6A
:106B00002380F38C1C4604401F0B6F433C191F0568
:106B10003F0F4F43E4191B061B0F5343E318204F4D
:106B20003B80338D18401C0B6C4320181C05240F30
:106B30004C4300191906090F51434018194C208085
:106B4000032519A228462946049B08F0AFFD70884A
:106B5000C1B20091030A18A22846294608F0A6FDF2
:106B60000D4803880D48008839882288094C2488FC
:106B700000AE17C618A22846294608F097FD05B0B2
:106B8000F0BDC046D0950102457D000012A701026C
:106B9000A0970102FC950102F4950102F69501020D
:106BA000F8950102FA950102C9E8B1B849443A20C2
:106BB0002578202E0D0A0000B9CCBCFEB0E6B1BE8F
:106BC0003A5557422D3447CAD6BBB7205625642EB6
:106BD00025642E200D0A0000B7FECEF1C6F7B5D809
:106BE000D6B73A2025642E25642E25642E25643AD6
:106BF00025642E0D0A000000F0B583B0304800680F
:106C0000C16B0901890F01D003B0F0BDC16BC06B2E
:106C10002C4D05404800400F08260296864002276A
:106C2000384602F029FB01907043C10B4A1B2648ED
:106C30005043F9F765FA044607F01EFC032123A22E
:106C400038461F4F0091234608F030FDF88A00288F
:106C500017D0019840012946F9F73CFA464318221B
:106C6000324001200F2A014600D8002173095B1829
:106C70001B4CA3420DD8194DED1A6D050F2A0CD8E7
:106C80000CE038680021C160112002F0E5FA03B081
:106C9000F0BD5D1C6D050F2A00D956422A0C029DDD
:106CA0002E4009018919A34202D80098000400E08F
:106CB0004004081880183968086303B0F0BDC04666
:106CC000AC940102FFFF1F0040420F0052434F33BC
:106CD000324B2070706D2025640D0A00FF07000004
:106CE000FE7F0000B0B582B0154908688269D207FE
:106CF0000CD00122C2610D69002D07D000686C46DE
:106D0000214607F09BF900212046A84702B0B0BDFC
:106D1000B0B582B00A490868026C92070ED5026CC1
:106D2000012313430364CD68002D07D000686C462F
:106D3000214607F083F900212046A84702B0B0BDE4
:106D4000AC94010206480168032291430160016886
:106D500001220A43026000F02FFB07F0AFFBC046A0
:106D60002800004080B50D490868002810D5224849
:106D700002680423032A01D01A4300E01A460A607D
:106D80001E490A68002A02D041680020904780BD51
:106D900003A00CA19E2211A307F02CFC2C10014093
:106DA000696E636C7564652F647269766572732FA2
:106DB0006D6B5F736C6565705F74696D65722E6372
:106DC00000000000534C4545505F54494D45525F0B
:106DD00049525148616E646C65720000556E657869
:106DE00070656374656420736C65657020696E748A
:106DF00065727275707400000C90010254D101022A
:106E0000B0B582B004460078002811D0094D01A920
:106E100008702868416A0029FCD101A901220020DC
:106E2000034609F0E9F9611C607800280C46EED1B0
:106E300002B0B0BDE894010210B5D64C2168062915
:106E40000FD8012002468A4058210A4209D020600A
:106E50000020A0602369002B03D06269002002217A
:106E60009847CB482258062A12D801210B46934056
:106E7000582213420CD02150201800218160036950
:106E8000002B05D0AD20C0002258012002219847D8
:106E900047482258062A11D801210B469340582210
:106EA00013420BD021502018002181600369002B70
:106EB00004D003482258022001469847002010BD04
:106EC000BC0A0000F0B581B00024022803D9E443D5
:106ED000204601B0F0BD17460B46094E464309480F
:106EE0008519284618302A2107A2FCF781FF422085
:106EF0002F52032003498851204601B0F0BDC046FF
:106F0000540500003CAC010225730000F0B585B0CB
:106F1000C64D2C68002C0CD0C34FC44CE659002E33
:106F20000CD0234FE659002E0DD00020C04305B0F1
:106F3000F0BD01AC0FC400272E4608E001AE0FC61D
:106F4000E619012703E001AE0FC6E6190227DA4C65
:106F500030462146FCF732FE022030607C4329197E
:106F6000029D4D60CF60039808610498486108460F
:106F70004430CC310122560210233246FDF714F87A
:106F8000CE480019B32189004118012D05D1B83030
:106F900001233246FCF7F3FB04E074301023324641
:106FA000FDF702F801980760002005B0F0BDC0466B
:106FB000A80A000001460020022901D9C0437047F9
:106FC000DD4A4A43DD4988507047C046022806D84A
:106FD000E8494143E84840180249401870474B20AF
:106FE00080007047D4040000022802D94B208000A2
:106FF0007047E8494143E84840184D21090140588D
:107000007047C046032801DB03487047E14941430C
:10701000E14840181830704745320100022806DC6C
:10702000DC494143DC4840184221405A7047002067
:107030007047C046032801DB00207047D549414313
:10704000D548401844307047022804DCD1494143F8
:10705000D1484058704700207047C046022805DCE0
:10706000CC494143CC4840184068704700207047E5
:1070700080B5022801D9002080BDC6494143C648D9
:1070800040184430FCF74BFF01464042484180BD68
:10709000B0B50024E14302280FD8BE4A4243BE4B9C
:1070A0009D58042D09D0991801220A600B69002B04
:1070B00005D04A690221984721460846B0BD2046BE
:1070C000B0BDC04610B50024022801D9E04310BD70
:1070D000B0494143B04A0723535051180B69002B64
:1070E00003D04A69002421469847204610BDC04677
:1070F000F0B581B00024022803D9E443204601B052
:10710000F0BD0546A3486843A34906220A500F185C
:10711000384644303946CC310122560210233246DB
:10712000FCF742FF786801280CD1B32080003918A1
:107130003846B83001233246FCF721FB3B69002B6F
:107140000CD1DBE7B32080003918384674301023A7
:107150003246FCF729FF3B69002BCFD07A69012129
:1071600028469847204601B0F0BDC04610B500241F
:10717000022801D9E04310BD86494143864A51188F
:107180000B69002B02D04A6903219847204610BDA5
:10719000540500003CAC0102F0B583B01746002452
:1071A000E24302281AD8002B18D00D4679494143F2
:1071B0007948461870680128029312D1002F0AD02E
:1071C000B836002429193046FCF7E1FA002825D109
:1071D000641CA742F6D1029807600022104603B053
:1071E000F0BD019274363046FCF799FE002811D0AC
:1071F00003464268BA4209D2196828461D46F8F784
:1072000093FF2B466868029908600194304619463E
:10721000FCF75BFE019A104603B0F0BD02980460D3
:107220000022104603B0F0BD540500003CAC010242
:10723000F0B581B004460020C343022C02D91846A1
:1072400001B0F0BD15460E461B4A62431B498F181C
:107250007968012910D1002D28D01C460090B8373C
:1072600038463146FCF76CFA002821D1761C6D1E99
:10727000F6D1009801B0F0BD009074373846294629
:10728000FCF768FE00280CD00446006831462A4608
:10729000F8F74AFF38462146FCF72CFE009801B06B
:1072A000F0BD07A02146FCF709FB009801B0F0BD36
:1072B000204601B0F0BDC046540500003CAC0102C0
:1072C000536F636B65745B25755D20526563762033
:1072D0004275666665722046756C6C0D0A0000008A
:1072E000F0B583B0154607460022D043022F19D8C7
:1072F000002D17D000AB07C30F4878430F490E1875
:10730000443630462946FCF725FE00280CD00446BA
:10731000006801992A46F8F707FF30462146FCF736
:10732000E9FD029803B0F0BD05A03946FCF7C6FAA6
:10733000009803B0F0BDC046540500003CAC01020B
:10734000736F636B65745B25645D2073656E642089
:107350006275662066756C6C0D0A0000024600209E
:10736000022A04DC0B4B53430B4AD1507047C043F5
:107370007047C046540500003CAC0102022801D908
:1073800000207047034941430348401803494058CF
:107390007047C046540500003CAC0102CC0400001C
:1073A00080B504480168491C01600069002800D0CC
:1073B000804780BDC0DC010201480249016070477E
:1073C000689001020026B80310B5C3480024446148
:1073D00010300221024A2346FFF798FD204610BDD7
:1073E0008D74000070B584B0FDF750F9012814D1F8
:1073F000FCF792FB1F4D6969022914D0002909D1BD
:10740000A97800291FD0A969411A062902D30021B1
:10741000A970A861002004B070BD16480021416128
:10742000002004B070BDE969421A13490E2A02D83F
:107430000A78002AEED0E8610020087000F004F914
:10744000002004B070BD01266E61AB88E8882989F0
:107450006A8900AC07C4B102084C09A22046FCF7B7
:10746000C7FC2869AA892146FFF72CFDAE700020D1
:1074700004B070BDF09501022C93010228C30102F3
:1074800025752E25752E25752E257500F0B58DB028
:10749000032925D87944097949008F440109111637
:1074A0005B48416901291BD1002141610DB0F0BD4C
:1074B00057484169012913D1022141610DB0F0BD46
:1074C0005348002141610DB0F0BD00250095504C9E
:1074D00020695049504A6B46FFF75EFE002801D0F4
:1074E0000DB0F0BD03204DA2014608F0DFF8494879
:1074F0004DA10A22F8F74DFE002812D045484DA1B3
:107500000F22F8F746FE0028EAD142482C2101AAB2
:107510000C23FCF77EFC0298FCF754FB60870DB04F
:10752000F0BD3C482C2101AA0C23FCF772FC049806
:10753000FCF748FB608780B2664EB1888142CFD1AC
:107540000298FCF788FCE062039801794279120204
:1075500051188279C3791B029A1812045118827843
:10756000C378077840780002C0191B029A181204E9
:107570001018206261620598FCF724FBA08706982A
:10758000FCF769FCE0870798FCF765FC4027E053AF
:107590000898FCF760FC42216054E16A491E062904
:1075A00001D801226270062927D8C046794409799A
:1075B00049008F440318111C221E1500E08FB08271
:1075C000E05BF082A08FB18D814216D0BA490222D1
:1075D0000A60B085B94800E01A48012101700CE04A
:1075E0000120B08709E0B4480560B58505E0B5879E
:1075F00003E0C0B23C214143B1830120607000F040
:1076000023F806F0C3FE2562656265700DB0F0BD1B
:10761000F095010228C30102FF030000CAD5B5BDE1
:10762000CAFDBEDD0D0A000024696E7374727563B5
:10763000742C0000246D6573736167655F726570FB
:107640006C792C0034960102F0B5C7B0214CA088AB
:107650001490214D28781390FBF704FF1290A08D11
:107660001190287810901D4800780F90A08A0E90F5
:10767000E08A0D901A48C0C81A490A6849686B78B0
:10768000194C24682035089209910A950B930C94A3
:107690001298009011980190109802900F98039002
:1076A0000E9804900D9805A9C1C11398002801D027
:1076B0000F4A00E00D4A15ADC8212846149B09F079
:1076C000ADFA0246044800692946FFF709FE47B0B3
:1076D000F0BDC04612A70102F0950102A897010271
:1076E00038980102309801025C960102512901008C
:1076F0001029010080B582B00E4908680022C260DE
:107700000192CA68002A02D0016801A8904702B01D
:1077100080BDC04680B582B0064908690022C260BB
:1077200001220192CA69002A02D0016801A890478B
:1077300002B080BD04930102F0B582B0644C2078A1
:10774000009000281DD0124B24330025019504E041
:107750009B1C6D1C0098854215D262196026905DB5
:10776000471C97550928F3D80199C8B222181C88DC
:1077700097554000064A10188484554C491C0191C5
:10778000E6E7002001900198207002B0F0BDC046ED
:107790005498010280B5002008F0E6F980BD80B55C
:1077A000012008F0E1F980BDF0B581B003F0D4FC10
:1077B000164CE060A178002901D001B0F0BD21791C
:1077C0000029FAD10121217100281BD08D02281A2D
:1077D000A168814216D05A4E2F46A068305C2169BC
:1077E0008847A068401CA060681EA168814201DD36
:1077F0000020A060E168A068022F03D3691A7F1EF1
:107800008842EAD10020207101B0F0BDC09501028C
:10781000B0B5294C2368002B07D0022B0DD0012BCB
:1078200039D109F00DF900F001FC09F0E7F82368FF
:10783000022B1FD0012B18D02DE0204D28780028D6
:107840002FD003201EA2014607F030FF0020287031
:1078500009F0F6F800F032FD1C4D287009F0CEF862
:1078600028780028E3D001202060194800214181B8
:10787000012310E011480178002909D114494A89EF
:10788000531C4B81152A03D301220270002048812A
:1078900008F07CFE2368032014A2014607F006FFCF
:1078A000B0BD0B48408914210B1A032009A20146E0
:1078B00007F0FCFEBBE7C046C0970102C49401027A
:1078C000BFAAC6F4CBD1CBF70D0A0000A5970102E1
:1078D00038960102B5C8B4FDBDF8C8EBCBD1CBF7E3
:1078E000C4A3CABDA3BA25640D0A0000555742D7E8
:1078F000B4CCACA3BA25640D0A00000070B50E2507
:1079000000242846214603F023FD0D20214603F0E4
:107910001FFD0124204608F02FF804262846314692
:1079200003F016FD0920314603F012FD204601F058
:10793000E9FAA2020249034B204608F01BFB70BD86
:10794000C0CB0102AD01010080B5032810D8002989
:107950000ED07C224243BF488018C268012A07D15A
:107960002030FBF714FF002801D00020C04380BD69
:107970000020C04380BDC046F0B589B00022D54389
:10798000032800D9ABE00C46002900D1A7E0009500
:10799000216A0727534DA9420EDC574DA9421ADD33
:1079A000564A91422FDC4B22D501A9423ED0120209
:1079B00091424BD1042246E04B4A914217DD4B4A9B
:1079C00091422ADCE1221203914231D0494A91428C
:1079D0003CD10C2237E04B252E01B14233D06A0155
:1079E000914227D0AA01914230D102222BE0E1221C
:1079F0005502A94220D09502A9421FD0D20291423D
:107A000024D109221FE04B225202914218D0E122D8
:107A1000120291421AD1062215E0E122520391424C
:107A200010D0334A914211D10D220CE003220AE01A
:107A30000A2208E0012206E0072204E0082202E010
:107A4000052200E00B22D1002D4A57587C214143EA
:107A5000804A505056182068B0606068F060A16895
:107A60003161E26872610025059503230493039553
:107A7000029501970695079501231B02089301289B
:107A800007D000280AD18818009A8018B161F061E7
:107A900004E0304620300123FBF771FE206970635B
:107AA0006069B063E069B067A069F063706801A9BC
:107AB00008F08CF92068012806D83046403023466B
:107AC00010330ECBFCF770FA6068012807D1301D27
:107AD0007036006801220B4B314608F04BFA2846FD
:107AE00009B0F0BDFFC10100FF0F0E00FF1F1C0019
:107AF00080841E0040420F007F250000FF9500009B
:107B000010170100C5010100B0B50C467C214843A7
:107B1000504A15182846FCF751F86C600020B0BD9B
:107B2000F0B583B00024E743032800D98EE00E4669
:107B3000002900D18AE01546002A00D186E07C2188
:107B40004143444841188868022832D001283AD07D
:107B500000282BD1EFF31080C00702D1EFF3108083
:107B600072B602910846403001902946FCF7F2F9BE
:107B7000002863D0014601980F46FCF7BBF938682E
:107B800031462A46F8F7D0FA0198FCF7C8F9EFF326
:107B90001081C90703D1EFF3108172B662B6029962
:107BA0004D6806C82C4B284608F026FB204603B03B
:107BB000F0BD4868002431462A46234608F01CFBE5
:107BC000204603B0F0BDEFF31080C00702D1EFF301
:107BD000108072B602910846403001902946FCF7A9
:107BE000B9F900281ED0014601980F46FCF782F92A
:107BF000386831462A46F8F797FA0198FCF78FF96A
:107C0000EFF31081C90703D1EFF3108172B662B6AA
:107C100002994D6806C8104B284608F0EDFA204638
:107C200003B0F0BDEFF31080C0070FD1EFF3108069
:107C300072B662B63C46204603B0F0BDEFF310804A
:107C4000C00703D1EFF3108072B662B63C462046FF
:107C500003B0F0BD38BC0102C9040100B0B582B068
:107C6000602833D0622843D0642854D101A82F491A
:107C70000180EFF3108072B600242046214602F006
:107C800055FA2B4D002805D101200203002029467A
:107C900002F0A6F9103501AA02232046294602F077
:107CA0007DFE62B623A0FFF7ABF864201B490C529F
:107CB00006F06CFB1A4801F0AFFBBFF34F8F194879
:107CC00019490160BFF34F8F00BFFDE760201349E2
:107CD00000220A5206F05AFB114801F09DFBBFF347
:107CE0004F8F104810490160BFF34F8F00BFFDE771
:107CF00062200A4900220A520A8006F047FB08481F
:107D000001F08AFBBFF34F8F064807490160BFF3BC
:107D10004F8F00BFFDE702B0B0BDC04612A7010201
:107D2000A08601000CED00E00400FA05AAAA0000FC
:107D300000D00204BDF8C8EBC9FDBCB6C4A3CABDDF
:107D40000D0A0000F0B5D1B0A74EA8490A78002A64
:107D500025D0F28B002A22D1A54FBA68082A00D973
:107D600090E0930001A4E3589F46C046917D000037
:107D7000857E0000857E0000957E0000BF7E0000AD
:107D8000C97E0000D37E0000A37E0000DD7E0000DF
:107D9000552800D0BBE00120B86051B0F0BD497853
:107DA000002900D1B7E0924D6A7996498854A979A3
:107DB000A871E971521C6A710A2800D0ABE00D2944
:107DC00000D0A8E003A8019037A800902C463034DA
:107DD0008C488D491DAB2246F8F7F8F9E8608BA175
:107DE00005222046F8F7D5F900282AD1F08B002883
:107DF00005D0032087A2834B014607F057FC1DA83E
:107E00000024214609F0D3FBA861E961824B224698
:107E1000F8F728FD002814D1804800F099FF1DA82C
:107E20000024214609F0C3FB2862696237A8214675
:107E300009F0BDFBA862E96203A8F8F759FA2861C6
:107E400000E0286900266E71002806D0744806708C
:107E5000744801210170744806806A489621F8F739
:107E60007CF91DA864242146F8F777F937A8214644
:107E7000F8F773F903A82146F8F76FF96E71EE80F1
:107E800051B0F0BDAA2838D1012A36D10220B860FD
:107E900051B0F0BD0421B9600021B970787051B0C3
:107EA000F0BD3979534A5054481C38717978491FCC
:107EB000C0B281422FD10820B86051B0F0BD052278
:107EC000BA60887051B0F0BD0621B960B87051B089
:107ED000F0BD0721B960387051B0F0BD7A78062A3C
:107EE00002921AD3531F0025424A2C46565DA4190C
:107EF000A4B26D1C9D42F9DB10E0032807D1022AD1
:107F000005D10120F8700320B86051B0F0BD002009
:107F1000B870B860787051B0F0BD00242018029A93
:107F2000821888781118BD7849193C780919FA78AF
:107F3000002A00D0C91C2C4EC9B2FF2935D1012816
:107F400009D0022831D11E2D36D1FFF7D7FC0120F0
:107F5000F08351B0F0BD284A9471032010719070E5
:107F6000AA2050705520107068085071651DD5709A
:107F7000400031181646D01D2246F8F7D5F8301DBE
:107F8000E11CEAB2D21C037892B2D218401C491EFE
:107F9000F9D1A019D143C171090A01720934012034
:107FA00000233146224608F027F90020B870B86057
:107FB0003871787051B0F0BD70190E4E31462246BE
:107FC000F8F7B2F83078012802D12846FFF746FECC
:107FD00006F0DCF9BFF34F8F084809490160BFF391
:107FE0004F8F00BFFDE7C04612A7010218900102A3
:107FF000109801025CCB0102849901020CED00E0B3
:108000000400FA05C4CA0102AD280100474E4747E3
:1080100041000000257300000000F03F79AB010231
:1080200014940102379601027AAB0102F0B589B0CF
:1080300008F03AFD8348844903F0D6FD834C0027BD
:10804000E77005F071FBE0610424204603F00CF9B1
:108050007F4A3846394608F059FD03F037FD0028BD
:10806000FBD105F061FB79498861C878012815D1F9
:10807000824E30788249097881420AD1707A20286C
:1080800007D17079B179090208187E49898D884233
:1080900021D0042003F0D8F809B0F0BD6D4806F0F7
:1080A000EFF96D4C237803206CA2014607F0FEFA2D
:1080B0002078411C21700628EBD36E480221016014
:1080C0002770624847816C4801210170042003F049
:1080D000BBF809B0F0BD049405F026FB5B4A906143
:1080E000B07A9070034605907079B17909020D1845
:1080F000D58031460B315C00634803912246F8F786
:1081000013F8A1190B31604832302246F8F70CF809
:10811000059800287DD05B48808906905B48006800
:1081200008900024059F02E0641CBC4256D0600009
:108130005549095A089A8A42F6D153490918488E76
:10814000069A801848864149097800290FD0504B7B
:10815000243300221E88AE420FD09B1C521C914239
:10816000F8D10B460A4600B217290AD90EE00023BF
:108170001A4600B2172904D908E0D3B200B2172971
:1081800004D88B4202D1491C304B19702F498918F1
:1081900060230026CE5451003D4A51188D84012899
:1081A000C2DBF8F787FB00273A463A4BF8F734FA78
:1081B00007900E462548406AF8F77CFB3A46059F33
:1081C000344BF8F729FA02460B4607983146F8F780
:1081D00071F9F8F7BFFB1D494862A5E7002F0ED0E3
:1081E0002A4801680020039C227863781B029A18B1
:1081F000914206D0A41C401C8742F5D109E000271B
:1082000007E0C4B22046FAF76BFF10488778A74210
:1082100002D13846FAF764FF0E4806F031F90B49EF
:1082200004980856174A938D496A009101900320DB
:1082300019A2014607F03AFA042003F005F809B044
:10824000F0BDC046BDF80000D9E20000389601023A
:10825000881300007C3F000052D00102B2E2BEE071
:10826000CAA7B0DCA3ACBCC6CAFDA3BA25640D0A7C
:1082700000000000C0970102C494010254D0010222
:10828000A497010212A701020C990102CC970102E6
:10829000549801020000E03FB1EAC7A94944A3BADB
:1082A00025582CBEE0C0EB3A20256420D0C5BAC5C5
:1082B000C7BFB6C8A3BA25642E0D0A00F0B587B0B3
:1082C00008F0F2FB8E4C607808F094F98D498A88AA
:1082D00005A882800A88498809048918059104F054
:1082E0009DF96078052804D002228749092804D125
:1082F00004E001228449092800D0891849792078AE
:10830000621C08F03BFA607A05F09EFC7F488049C9
:1083100003F06AFC7F4E0025F57005F005FAF06168
:10832000042002F0A1FF7C4A2846294608F0EEFB13
:1083300005F0FAF97949306371634118481C00D09F
:108340000846B06305F0F0F9F063B16B744C8842F5
:1083500003D30919884200D8C3E0724F03F0B6FB7B
:1083600000280AD0FCF750F905F0DEF9F063B16B94
:108370008842F3D909198842F0D205F0D5F9B061E5
:10838000F07801280FD138786749097881420AD1FD
:10839000787A202807D17879B979090208186349D1
:1083A000898D884210D005F0BFF9F061002528467C
:1083B0002946594A08F0AAFBB16BF06B8842CDD32D
:1083C00009198842CAD88CE005F0AEF9B061B87AD4
:1083D000B070024603907879B97909020C18F480DC
:1083E00039460B315500524800912A46F7F79CFE5A
:1083F000E919039F0B314E4832302A46F7F794FEB5
:10840000002F66D04B4800680490002502E06D1CE8
:10841000BD424DD068004649095A049A8A42F6D1B5
:10842000434908183221405E317800290ED0424B72
:10843000243300221F88A7420DD09B1C521C91425E
:10844000F8D10B460A46172908D90BE000231A4633
:10845000172903D906E0D3B2172903D88B4201D1DB
:10846000491C3170B11860230027CF545100324AA3
:1084700051188C840128039FC9DBF8F71BFA0027E9
:108480003A462E4BF8F7C8F802900191706AF8F757
:1084900011FA3A46039F294BF8F7BEF802460B46FD
:1084A00002980199F8F706F8F8F754FA7062AEE707
:1084B000002F0ED01F4801680020009C22786378AE
:1084C0001B029A18914212D0A41C401C8742F5D17D
:1084D00000E000273846FAF703FE194805F0D0FF00
:1084E0000125042002F0B0FE284607B0F0BDC4B25A
:1084F0002046FAF7F5FDB778A742EED1EAE7C04685
:10850000AE900102E4160100A49E0102BDF8000035
:10851000D9E200003896010280841E000098E00E27
:10852000007C312554D00102A497010212A7010258
:108530000C990102CC970102549801020000E03F1F
:108540007C3F000080B582B0002001900448C268E2
:10855000002A02D001A80021904702B080BDC04689
:1085600078950102F0B583B000242046FEF74AFA60
:10857000FEF76DFA274EB060FEF766FA7060264F80
:108580000BE001A8C1888088084319D101A8408860
:1085900024180834B068844235D201AD0821284639
:1085A0002246FEF73BFA28880028EAD0B8422AD0B3
:1085B00001AD0421284600F019FFA9888842E5D0C2
:1085C0003460B06884420CD201AD022128462246B4
:1085D000FEF724FA2888B84203D0A41CB06884426D
:1085E000F2D370682118491E4042084030600DD017
:1085F0000024254601202946FEF7E8F903CE4D194F
:10860000083E8542F6D3346003B0F0BD00243460E8
:1086100003B0F0BDB4960102FFFF000010B5054C99
:108620002070FFF711F82078022801D10020207077
:1086300010BDC046F0950102F0B585B01F4604920A
:108640000646C8170C1844400A2C039114D3012580
:108650000A212046F7F73EFD6D1C632C0446F7D82F
:1086600004998D4200D329460A9C002F09D0039813
:10867000002808D4002207E0012504998D42F2D297
:10868000F2E7002205E00122042323409B08134364
:10869000FA1A0223234004980028029412D1002BD6
:1086A00010D0F468002C62D40398002825D40298D6
:1086B000400734D57068B5686F1C87422FD8306882
:1086C0002B2423E0E407ECD1002A0AD1E9E737683C
:1086D00020203855B560F068441CF460521E002C10
:1086E000DFD49142DDD27768B468651CBD42EED913
:1086F000F468521E002CF4D5D3E740420390706812
:10870000B5686F1C87420AD830682D244455B7607D
:10871000F068441CF4600025ED43A84227DB002BE1
:108720001CD00120029B1840049B184316D1002A3C
:1087300003D113E0521E002C0ED491420CD270686B
:10874000B3685D1C8542F5D830683024C454B560E8
:10875000F068441CF460EDE7002C08D40092029805
:1087600001900A2230460399049B00F003F805B0FB
:10877000F0BD0000F0B587B01F46154602900124F9
:1087800006919142009407D3012406982946F7F7F1
:10879000A1FC641CA842F9D20D980C9ABC42039724
:1087A00000D3039400990140002A009109D00029C8
:1087B000029C25D12021800705D40846002F11D026
:1087C00004E0029C1CE03020002F0BD0084609E09A
:1087D00023685854A260E168491CE1603246721E69
:1087E00000290DD4039991420AD216466368A16804
:1087F0004A1C9A42ECD9E1683246721E0029F1D532
:10880000E068002859D40590012401E07F1E6C43E4
:10881000022FFBD2069821461646F7F75BFC32463C
:10882000A842F4D2029880680490069F01950697AA
:1088300038462146F7F74EFC049D691C029F7A6872
:10884000914206D9069F059A019D0592002A0ED5F0
:1088500016E01B4A125C3B685A55B960FA68521C14
:10886000FA600491069F019D0592002A08D4604396
:108870003F1A20462946F7F72DFCAC420446D6D2D3
:1088800000980028029C059B049D16D0002E14D051
:10889000701C01E0002B10D4401E039981420CD2C1
:1088A000691C62689142F5D8226820235355A16063
:1088B000E268531CE3600D46ECE707B0F0BDC0462C
:1088C000EC190100F0B583B001900291002923D08A
:1088D0000025124F2E460AE013480818410F401891
:1088E000C0103872761CB0B20299884214D2019836
:1088F00000884B24210100B200F018F8400061010B
:108900004018388301B2064881422846E9DB054811
:108910008142E1DD6420E4E703B0F0BDA0970102ED
:10892000E40C0000041000001CF3FFFF074A904213
:1089300001DD054A801800B24143C817400D0818F0
:10894000C00A00B27047C04600F0FFFFFF070000FA
:1089500010B50078012819D1AC480269012A04D168
:10896000614A13680124A3431360032905D08021C1
:108970004161C269002A05D107E001214161C26954
:10898000002A02D001898069904710BDFF222E3253
:10899000024803A107A305F02DFEC046A025010053
:1089A0006164635F646D615F63616C6C6261636B82
:1089B00000000000556E657870656374656420641E
:1089C0006D61206368616E6E656C0D0A00000000C9
:1089D000F0B58DB00D460124EFF31081214002D196
:1089E000EFF3108372B6894E73690F2B06DD102BDF
:1089F00037D0402B2FD0802B2DD005E0002B2AD054
:108A0000012B01D110237361B5813581B061F26111
:108A1000002900D162B63179002929D00294304C66
:108A200005A90A4604950390E8CCE8C2E8CCE8C260
:108A3000029C204600F060FD2A4800902A4D2946FD
:108A400008312046039A049B00F0C6FD2C600024E8
:108A500020460DB0F0BD0029FAD162B620460DB017
:108A6000F0BD02240029F3D162B620460DB0F0BD5E
:108A70003178002907D01C48072181610460002457
:108A800020460DB0F0BD3269B3891749002B15D0CF
:108A9000B5693089012A02D0002A03D003E09FB2D1
:108AA000874200D10C604F68FF07FCD08F6880C5FB
:108AB0005B1E1F04EED10023B381B561012A02D1F0
:108AC0000A68A2430A607461F2690024002ABFD0D8
:108AD000B36931898800181A904720460DB0F0BD5F
:108AE0002C1A01005189000008D00140F0B581B076
:108AF000002856D00446424EF068800754D413250F
:108B0000284600F0B1FB284605F08AFA276861681C
:108B1000012538462840CA07920F1018227C1207F8
:108B2000120E8018627C1207120D8018A27C1207A8
:108B3000120C8018627D13071B0AC0181209120656
:108B4000801830607D2006020029304600D12D4873
:108B5000E3681A0A7D2A1A4629D22B4EB3422AD23A
:108B600000292BD0002A2946254E00D01146F7F7C0
:108B7000B1FA401E80B2706024480761E27C027046
:108B8000237D0371224F3E686902A468012C1BD02B
:108B90002C0226433E60002B1ED00121184A11638F
:108BA00029E0012001B0F0BD022001B0F0BD324645
:108BB000154EB342D4D333460029D3D11A46002AE6
:108BC00029460F4ED2D1D2E73F242401A64376187E
:108BD000F0363E60002BE0D1002A0CD0FF221202BA
:108BE0000C4B1C6894430122D203A2181A60304A2D
:108BF0001160304A116001214161002001B0F0BDD7
:108C000000D001400026B80380841E008895010230
:108C10002C06004008E400E070B5002801D00120D7
:108C200070BD0C461625284600F01EFB284605F0B0
:108C3000F7F9002C05D01B48183014222146F7F70D
:108C400073FA28211748415C002915D04168002992
:108C500016D403220B469343144A9C588D07ED0EFD
:108C6000FF26AE40B4439C501F220A400121914090
:108C70000F4A11600F4A116001210161002070BD8F
:108C80008A07D20EFF2393400F220A40083A03219D
:108C90008A43054954589C435450012101610020E6
:108CA00070BDC0466C9001021CED00E000E400E0E5
:108CB00080E200E000E100E080B552480021017050
:108CC0004B480078C0014B490978890101434A4863
:108CD000007840010843494909780901014348489F
:108CE0000078C000084348490978490001434748D3
:108CF00000780843C0B2FBF7C3FB80BD80B5414894
:108D0000012101703B480078800139490978C90187
:108D1000014339480078400108433849097809017E
:108D2000014337480078C0000843374909784900B3
:108D3000014336480078084304210143C8B2FBF7D9
:108D40009FFB80BD5A21014A505270473C9E010250
:108D5000F0B581B004460078414241412170244879
:108D60000078C0012349097889010143224800782D
:108D7000400108432149097809010143204800784E
:108D8000C00008431F4F3978890001431E4D2878E1
:108D9000400008431D4E31780143C8B2FBF770FB19
:108DA0007D20C00000F038FB207841424141217015
:108DB0000F480078C0010F490978890101430E4826
:108DC0000078400108430D490978090101430C4826
:108DD0000078C000084339788900014328784000B2
:108DE000084331780143C8B2FBF74AFB01B0F0BD3C
:108DF000889D01023696010215940102F0E40102F9
:108E000079AB0102899D010204A1010205A10102C1
:108E1000B0B5094D28600224002120460A4602F020
:108E20002BFA01210522204602F0BAFA2A68032112
:108E3000204602F099F9B0BD849D01025C219D4855
:108E40000022425282847A2141840284C2830283B6
:108E5000C2820282114941608260C2603D214904A0
:108E600041834182090C8183818270475C21914852
:108E70000022425282847A2141840284C283028386
:108E8000C2820282054941608260C2603D2149047C
:108E900041834182090C8183818270474C3C3C3C78
:108EA00070B585484C21016001252C02601C00F042
:108EB0005BF9322000F0B0FA00F044F9284600F0E7
:108EC0004BF9284600F05AF800F036F90C4800F04B
:108ED0004BF900263046314600F056FA2846314616
:108EE00000F052FA204600F03FF9022000F03CF971
:108EF0004834204605F0F6FA05F054FB70BDC04634
:108F00000102000010B50446072106F02DFA0148C1
:108F1000046010BDE895010270B5052004242146C7
:108F200002F016FA0620214602F012FA0A20214623
:108F300002F00EFA0920214602F00AFA002401216B
:108F4000204602F005FA022520462946224602F074
:108F500027FA0B2630462146224602F08DF930468C
:108F60002946224602F01CFA70BD00000248016842
:108F700001229143016070475800004002490A688D
:108F800002408242FBD1704704600040B0B5494DB9
:108F900028688107484C0ED528797F21084022682F
:108FA0008A431018206023680B4002200321434AA3
:108FB00006F07CFB286880040ED55E20285C7F21AB
:108FC000084062688A431018606063680B400220A2
:108FD00003213B4A06F06AFB172000F045F93948A7
:108FE000016802220A4301218A4302603648374958
:108FF000016037480021C17181791F2529408171A5
:10900000817A427C837C1B029A18C37C1B04D21891
:10901000037D1B06D2182F4B9A4218D1427B837BCB
:109020001B029A18C37B1B04D218037C1B06D218A0
:10903000294B9A420BD1C27A037B491E122906D8CA
:1090400019028918254A914201D120210172017823
:10905000CA0602D11022114301701C3C2068202155
:10906000884320601E481F49016041680029FCD5E3
:1090700003F038FA0446022003211BA2234606F01F
:1090800015FB0A20C441032C05D8022003211DA290
:1090900006F00CFBFEE71848C1680F229143C1603F
:1090A0000168164A0A40026019200001144948600C
:1090B0000D60B0BDA49E010248000040E8250100FB
:1090C000D2250100040200400C060040AF6B100ADC
:1090D0006B0001404D383650312E323607340000D7
:1090E00000600040FE1C0080436869702049443ADB
:1090F00020253038780D0A00C8600040FEFFC3FF0D
:109100000C0400404F6C642063686970206D6F64CC
:10911000656C206973206E6F7420737570706F7248
:1091200074656420627920746869732053444B210C
:1091300021210D0A0000000080B5172000F08CF8F6
:10914000002080BD10B51724204600F08DF8204681
:1091500004F066FF002010BD0121C907014301484A
:10916000016070470060004010B5C1B2000AC2B291
:1091700002290CD0012913D0002930D1911E7F483B
:1091800002291BD20121032A2AD0490429E07B4865
:109190004168002A1FD00246203A1143416010BDA9
:1091A00076480168D31E022B10D3012A29D0002A49
:1091B00041D1012292079143016010BD002A16D1CE
:1091C0000121490702688A43026010BD0123042A75
:1091D0001FD05A041EE0012292079143416010BD46
:1091E0000904194A7F32C36A13405918C1621749EA
:1091F0008A699207FCD50121490702680A43026087
:1092000010BD0522120791430246203A0A4302602C
:1092100010BD1A04836A0C4C1C40A21882620B4ACF
:10922000131F00241C600A4B0A4C1C600D235B02B8
:1092300014681C431460054A93695B06FCD505223B
:1092400012071143016010BD80FFFCFF14020040B3
:1092500004010040FF0F00000121814047480268DF
:109260008A4302607047C04601218140434802683A
:109270000A4302607047C04610B5052811D8C046A1
:109280007844007940008744020E192434393B4960
:109290000A680868C0003CD53A4820390A425DD0C7
:1092A0003BE0002010BD35490A680868C00035D58C
:1092B00034480B46203B1A4237D134E02F490A6824
:1092C0000868C00036D52F480B46203B1A424CD1C7
:1092D00035E02A494C680120C0030A680B46203B50
:1092E0001C421AD00C68E4003BD5264C1A423CD0F4
:1092F0003AE0224800680120C00310BD1F490A68F7
:109300000868C0001ED51F480B46203B1A4220D1DA
:109310001DE01B4820390A4220D010BD18480B46DA
:10932000203B1A4201D10120C00349688900890FFE
:10933000C84010BD12480B46203B1A4215D10120EF
:10934000C00312E00E480B46203B1A4201D1012017
:10935000C00349680903890FC84010BD0120C0033C
:1093600010BD074C1A4200D020464A689200920F66
:10937000D04049680901890FC84010BD2000004055
:10938000006CDC020026B80304282CD8164AC0461C
:109390007844007940008744020A121A2100032011
:1093A0000007136883438807800818181AE0032011
:1093B00080061368834388070009181812E0032009
:1093C0008004136883438807000B18180AE0FF2005
:1093D0000002136883430802181803E01068FF2393
:1093E000984340181060704724000040B0B5002238
:1093F00000290CD0074B047895B22D0A65406C000B
:109400001C5B12026240491E401C0029F3D190B23D
:10941000B0BDC046EC17010000280AD030B40725C3
:109420002C02CD256419604340091238001FFDD875
:1094300030BC7047F0B583B01F4616460D46014656
:10944000E8680291F6F7BAFF04460F2E11D8082EED
:1094500004D320462146F6F758FF09E0042E02D334
:109460008120C10501E0412001062046F6F7A6FF54
:1094700004460999089E2B20C043874205DB2046FD
:109480000F462146F6F741FF0DE03F20C0438742DB
:109490000BDA4920C04387420CDBFF200F468105D1
:1094A0002046F6F78BFF39460446688A0880346008
:1094B00003B0F0BD01915320C043874206DB204634
:1094C0002146F6F722FF0446688A10E0A86902994F
:1094D000F7F79EF9002801D1A88B00E0E88BF7F799
:1094E000E2F901462046F6F769FF0446002001999B
:1094F0000880346003B0F0BDF0B581B005460120AE
:10950000072D66D80C46002963D04A4F3868016998
:10951000C90736D105263046FFF7A6FE304604F0CF
:109520007FFD03CF0369012213430361002918D48F
:1095300003200B4683438E481E588807C00EFF2722
:109540008740BE4340278740374389481F501F202C
:1095500008408240874802608748026035480068BA
:109560000FE08A07D20EFF2696400F230B40083BE0
:1095700003218B437D495F58B743402696403E43C5
:109580005E5069014018012109024218E369DB06B7
:109590009B0CA569ED00EDB2EB18536062685207B1
:1095A000520B23685B075B099A18A3685B079B0C47
:1095B000D218E3685B075B0DD21823695B01DBB24D
:1095C000D21863699B07DB0ED218802313434350E4
:1095D000002001B0F0BDC046F0B581B0002A23D014
:1095E00005460835134C2668F668EE40F50702D0AC
:1095F000022001B0F0BD069D8600A619B5604001AD
:1096000024682018009301231D0246197768072457
:10961000A7437760F16032610099B1604159194305
:109620004151002001B0F0BD03A00AA174220DA396
:1096300004F0E0FFBC920102696E636C7564652FF3
:10964000647269766572732F6D6B5F646D612E63F2
:1096500000000000646D615F7472616E7366657214
:1096600000000000496E76616C6964207472616E5E
:109670007366657220647374206164647200000014
:1096800000015849085840687047C046F0B581B09D
:1096900005460120012D4CD80C46002949D0002D4B
:1096A00003D0012D04D10F2000E00E20FFF7DCFDD8
:1096B000A668012E04D0002E4FD1E08900284CD19D
:1096C0002901294843580020D860F507AD0F2768C5
:1096D0006668B607360F76192569EA07920EB6183E
:1096E000022F04D0012F03D10122164300E040369F
:1096F0001D4F9E60E2681A6079188D606269CA60C9
:109700004968002917D403220B469343184A9C58F2
:109710008D07ED0EFF26AE40B4438026AE402643B3
:109720009E501F220A4001219140124A1160124AA4
:10973000116001B0F0BD8A07D20EFF2494400F23C0
:109740000B40083B03218B4308495D58A543802407
:1097500094402C435C5001B0F0BD08A00FA14922F9
:1097600012A304F047FFC046049301021CED00E081
:1097700000E400E080E200E000E100E0696E636C7C
:109780007564652F647269766572732F6D6B5F64A3
:1097900075616C5F74696D65722E63006475616CD0
:1097A0005F74696D65725F6F70656E00636F6E6682
:1097B000696720697320696E76616C6964000000D6
:1097C0000001084A10580160816880220A438260C3
:1097D0007047C046000103490858816880229143C0
:1097E0008160704704930102F0B58DB00193154676
:1097F0000E460A901298002408900480149F3C8022
:10980000139809900460159804900480FF20810546
:109810003046F6F7D3FD0290304603963146F6F710
:1098200074FD2B463D460690274607950B9311E0A5
:109830001180188880002858099908600120079D28
:1098400028800520049908807F1CBCB218888442B7
:1098500000D9A0E028880028F6D1A0000A9D2E5843
:1098600030460699F6F7C6FF002817D03046039910
:10987000F6F7C0FF00280B9B079DE5D1089A1780DB
:10988000099D2E601888011B012934D11080198888
:1098900089000A9A51582960059035E0089A178086
:1098A000099806600B9B1988081B0128C0D00C96EC
:1098B000019825187E1CB0B28542BFD389B2B2B2DE
:1098C0008A420ED880000A990C5820460C99F6F767
:1098D00083FF0B9B002804D1099804600898068038
:1098E0000C94761CB0B28542A8D3198889B2B2B262
:1098F0008A42E7D9F5E70C96019962187D1CA9B256
:1099000016468A4205972CD2059884B2A5000A9E75
:109910007259002C104609D0A819001F0168104682
:109920000C92F6F7F2FC0C9A062C07D80446A819FC
:1099300041681046F6F7E9FC0C902046079D029915
:10994000F6F766FF00280B9B07D10C980299F6F7F3
:1099500051FF0B9B002800D076E7012028800320D0
:1099600070E780B2AAB282420FD888000A990C58D8
:1099700020460C99F6F730FF0B9B002805D109987B
:1099800004600898058005950C946D1CA9B28E4260
:10999000BAD31888E5E70DB0F0BD00000A490A689F
:1099A0000A4802400A60FD214900094A1268515CD8
:1099B000002908D007490A6C02400A640120000609
:1099C0000A6882430A60704700040040FFFFFF7F7F
:1099D0002C9401022000004000207047F0B583B0B5
:1099E0000D4604467C26464350488719F869396A73
:1099F000F6F770FBA84200D892E00195029401218D
:109A0000EFF31080084002D1EFF3108272B63C46AB
:109A100010343B690025062B0CD80A469A40D30621
:109A20005B0F06D161231A4275D00D46002803D082
:109A300003E00225002800D162B6002D02D028469E
:109A400003B0F0BD00943C462034384880591021C2
:109A5000C1613E46143604F09FFD05463868C06972
:109A6000C00605D504F098FD401B31888842F5D921
:109A70000621029D284600F00BFF20680199414312
:109A8000B869091838688160172179563C4617343F
:109A9000002909D5C16920220A43C2610121F96662
:109AA000890502680A4302600521284600F0F0FE9D
:109AB000207840B200250028C1D42B4800687D24BE
:109AC000E100F6F707FB61014143029800F0B2FEA6
:109AD00004F062FD04463868C069C00705D004F090
:109AE0005BFD001B31888842F5D904F055FD044622
:109AF0003868C169890706D504F04EFD001B31881E
:109B00008842F5D938680121009A11605349816172
:109B1000284603B0F0BD0321216000288CD08CE7DB
:109B2000034804A1084A09A304F064FD309301022C
:109B300018260100666C6173685F626C6F636B5F0F
:109B400065726173650000005D020000626C6F6306
:109B50006B20696478206973206F7665722072616A
:109B60006E67650D0A000000D4DC0102F0B583B019
:109B700002907C214143934A5418E56EEAB2511E8B
:109B800002291FD229040126090E18D0019600923D
:109B9000022100F07DFE2746143704F0FDFC064646
:109BA0002068C169890606D404F0F6FC801B398858
:109BB0008842F5D92068007DC007019E08D0304654
:109BC00003B0F0BD032A36D100922804000E36D02F
:109BD00020466C302D0C002101910160274614377E
:109BE00004F0DAFC06462068C069C00705D004F01E
:109BF000D3FC801B39888842F5D904F0CDFC064699
:109C00002068C169890706D504F0C6FC801B398825
:109C10008842F5D9206811498161E9B20120002903
:109C200011D003290099019E00D006202061226FE7
:109C3000002A0ED1C3E70026304603B0F0BD01264E
:109C4000304603B0F0BD0099019E2061226F002ACA
:109C5000B5D002A89047304603B0F0BD000093EBAA
:109C600070B5002801D0012070BD7825CD4E705D03
:109C700000280ED000240921204600F009FE0F2004
:109C8000FFF7CAFB1520FFF7E7FA74553461204649
:109C900070BD042070BDC046F0B581B00C460078A0
:109CA000484EF16881422CD1032C54D1706EB16EB4
:109CB000884261D900240621204600F0E9FD306881
:109CC000F16D81602046214600F0E2FD35466035A9
:109CD0002CCDF0683168B48C414F00975B1BA342D8
:109CE00000D81C46A3081431FFF776FCB06E0019AB
:109CF000B066306E00193066F06D0019F06501B085
:109D0000F0BDB168814255D1032C45D1F08CF16D85
:109D10000918F165316E09183166B16E0818B06620
:109D2000716E814238D900240621204600F0B0FD32
:109D30003068F16D81600121204600F0A9FD316E8F
:109D4000B068F38C3268264C009414329B08FFF7FD
:109D500043FC01B0F0BD30681021C16104F01CFC6F
:109D600005463068C069C00616D504F015FC401BD6
:109D7000B18A8842F5D90FE030681021C16104F042
:109D80000BFC05463068C069C00605D504F004FC2C
:109D9000401BB18A8842F5D90120C1073268136897
:109DA0008B431360F16E22040A4300021043F066F5
:109DB00001B0F0BD4D200201034804A1844B04F022
:109DC00019FCC0463093010218260100666C6173CD
:109DD000685F646D615F63616C6C6261636B0000FE
:109DE000999C0000F0B581B000786E4DAA6882425F
:109DF00000D0D0E001263002032942D16A6DAA6664
:109E0000AB6DAC6AA418EB652C66AB6C5B1CAB64E9
:109E10006B6E934235D95E30FFF7FEFA686CA96C21
:109E200002293AD3814238D1E88C696D08186865F7
:109E30000020062100F02CFD2868E96D81602F6D5F
:109E400004F0AAFB04462868C069C00705D004F0E6
:109E5000A3FB001BA98A8842F5D904F09DFB0446A8
:109E60002A68D069800706D504F096FB001BA98AF2
:109E70008842F5D92A687420285C012841D0F10471
:109E800040E0F2072B681C6894431C60EA6E0904EA
:109E900011430143E96601B0F0BD0229FBD38142C1
:109EA000F9D2E88C696D09186965A96D0818A8656B
:109EB0000020062100F0ECFC2868E96D8160EF8C41
:109EC00004F06AFB04462868C069C00705D004F0A6
:109ED00063FB001BA98A8842F5D904F05DFB0446A8
:109EE0002A68D069800706D504F056FB001BA98AB2
:109EF0008842F5D92A687420285C012822D0F10410
:109F000021E03105334B3B405918012802D019207C
:109F1000400601E00720C00608182F49401850608D
:109F2000002F0DD004F038FB04462A68D069800762
:109F300006D404F031FB001BA98A8842F5D92A68AF
:109F40002B6D1FE03105234B3B40C918012802D07F
:109F50001920400601E00720C00608181E494018D5
:109F60005060002F0DD004F017FB04462A68D0691A
:109F7000800706D404F010FB001BA98A8842F5D99B
:109F80002A68EB8C296EA868144C00941432FFF7F1
:109F900023FB01B0F0BD044804A10C4A0C4B04F0B3
:109FA00029FBC0463093010218260100666C6173DC
:109FB000685F646D615F77726974655F6E62797402
:109FC00065735F63616C6C6261636B0072040000B7
:109FD000FF250100FF3F000000808000E59D00009C
:109FE000F0B587B004460126880E14D01546002A25
:109FF00011D00F468120C004401B88420BD37C2027
:10A000006043F04908180590818C38460691F6F7B0
:10A0100061F8002902D0304607B0F0BD2846069905
:10A02000F6F758F80029F6D1059880693E1A3046AF
:10A030000699F6F74FF80746039670190190069EA9
:10A040003146F6F747F80546C01B04900598006AAC
:10A0500002903146F6F73EF8049981420FD200266D
:10A06000BD42D8D92046394600F018FB2046FFF7FC
:10A070007DFD0028FAD17F1CAF42F3D3CBE70090DF
:10A080000398029D2946F6F725F8064628467043B0
:10A090000399081A019800D0761C2946009D754343
:10A0A000F6F718F80590029941430198401A039079
:10A0B0000699F6F70FF80490AF420BD220463946C6
:10A0C00000F0ECFA2046FFF751FD0028FAD17F1C82
:10A0D000AF42F3D305988642069D009F0CD22046DE
:10A0E0003146FFF77BFC2046FFF740FD0028FAD100
:10A0F000761C05988642F2D30398A84203D2002624
:10A10000304607B0F0BD059847430025E9192046C1
:10A1100000F0C4FA2046FFF729FD0028FAD16D1C93
:10A12000002604988542F1D375E7C046F0B585B0A6
:10A13000002803D00124204605B0F0BD7822A14FAD
:10A14000B85C002803D00024204605B0F0BD04927E
:10A15000002905D0384614300CC90CC01CC91CC0DD
:10A160000020F86615242046FFF77EF8204603F00D
:10A1700057FF38681021C16104F00EFA04463868B0
:10A18000C169C90607D504F007FA001BB98A8842DD
:10A19000F5D9386800E0B98ABA7D1207120B521857
:10A1A000F97DCB07DB08D2188B07DB0F5B05D218D4
:10A1B000CB06DB0FDB05D2184B07DB0FDB06D21813
:10A1C0008B06DB0F5B07D2180907C90F89071143FC
:10A1D000016000240A21204600F05AFB3220FFF7DC
:10A1E0001BF90821204600F053FB04F0D5F9054681
:10A1F0003868C169890606D404F0CEF9401BB98AD3
:10A200008842F5D93868017D0A46C23A5342534123
:10A2100074257B550904027D12025118007D0B182C
:10A220000220032668A2314605F040FA785D012835
:10A23000039619D1F87D029000260621304600F0E1
:10A2400027FB0721304600F023FB012102988143C0
:10A25000785D012847D13868890101750675752137
:10A26000795C012938D048E00020032100F010FB80
:10A2700004F092F906463868C169890606D404F0EC
:10A280008BF9801BB98A8842F5D93868007D460869
:10A290000122F87D014631431640C90701D0304004
:10A2A00036D00295002506212846019200F0F0FAEA
:10A2B00007210095284600F0EBFA019846400298E5
:10A2C000385C012813D13868B10101750099017516
:10A2D0007521795C012910D114307621795C4A42CC
:10A2E0004A41510008E038680675490003E03868C3
:10A2F00000990175710014300170374800687D21A4
:10A30000C900F5F7E7FE28214143002000F092FA4A
:10A310007720385C012803D102200021FFF734F8B0
:10A3200004F03AF906463868C069C00705D004F061
:10A3300033F9801BB98A8842F5D904F02DF9064615
:10A340003868C169890706D504F026F9801BB98AE7
:10A350008842F5D93868D0498161172038560028DD
:10A3600029D57868002816D40146039A91431C4ADF
:10A370008B588507ED0EFF26AE40B3438026AE40D6
:10A380001E438E501F21014001208840154908605E
:10A39000154908600FE08107C90EFF228A400F238C
:10A3A0000340083B039883430C481D589543802283
:10A3B0008A402A431A500120049978543861204673
:10A3C00005B0F0BD309301026A656465635F69643E
:10A3D0002025780D0A000000D4DC01021CED00E00D
:10A3E00000E400E080E200E000E100E0F0B593B0BE
:10A3F0007C270A9047439348C619980704D0F07DFC
:10A400004024044000D017E10125880E2ED0002BF7
:10A410002CD08120C004C01A884227D3099201227F
:10A42000EFF31084144002D1EFF3108072B630467F
:10A43000103005903069002506280891069310D841
:10A44000079414468440E106490F04D161210C426F
:10A4500003D0154604E0022502E00221059B1960A5
:10A46000079C002C00D162B6002D02D0284613B004
:10A47000F0BD344617347348C05910210491C161AE
:10A480003746143704F088F805463068C069C006BE
:10A4900005D504F081F8401B39888842F5D9207829
:10A4A000400665D40297B78C069C20463946F5F7DE
:10A4B00011FE079039464143601A03903546243512
:10A4C000A74200D894E0039800281CD006210A9CDB
:10A4D000204600F0DDF9288807994843089940187C
:10A4E0003168886000272046039C394600F0D0F987
:10A4F000079B099A28885843C0193168097D11546F
:10A500007F1CA742F6D330680499C16104F044F877
:10A510000446029D3068C069C00605D504F03CF8C9
:10A52000001B29888842F5D904F036F804463068C3
:10A53000C069C00705D004F02FF8001B29888842A5
:10A54000F5D904F029F804463068C169890706D5B1
:10A5500004F022F8001B29888842F5D930680121CF
:10A56000059A1160B24981610025284613B0F0BDFB
:10A5700003200025089FF7650999316606997166E1
:10A58000B566F0660120C00731680A6802430A60B8
:10A5900006210A9C204600F07BF93068876020463F
:10A5A000294600F075F93A4F0BAA0A921BCF1BC23D
:10A5B0001BCF1BC2B48CF0680A99FEF79DFFF068B0
:10A5C0003168344A0092069A944200D31446A30894
:10A5D0001431099AFFF700F8B06E0019B066306EBA
:10A5E00000193066F06D0019F065284613B0F0BD13
:10A5F000002404E0641C0798844200D363E706212A
:10A600000A9800F045F92888604308994018316895
:10A61000886000270A98394600F03AF9288800280F
:10A62000099AE7D0604310183168097DC1557F1C35
:10A6300028888742F6D3DDE7034804A1064A07A32A
:10A6400003F0D8FF3093010218260100666C617395
:10A65000685F726561640000C6030000546865208D
:10A66000444D412072656164206C656E677468209A
:10A6700073686F756C6420626520746865206D7501
:10A680006C7469706C65206F6620340D0A000000E0
:10A690008C1A0100999C0000000093EBF0B583B088
:10A6A0000D4604467C26464351488719F869B98C03
:10A6B000F5F710FDA84200D894E00195029401211D
:10A6C000EFF31080084002D1EFF3108272B63C46DF
:10A6D00010343B690025062B0CD80A469A40D30655
:10A6E0005B0F06D161231A4277D00D46002803D0B4
:10A6F00003E00225002800D162B6002D02D02846D2
:10A7000003B0F0BD00943C462434394880591021F0
:10A71000C1613E46143603F03FFF05463868C06904
:10A72000C00605D503F038FF401B31888842F5D9B3
:10A730000621029D284600F0ABF82088019941438C
:10A74000B869091838688160172179563C46173472
:10A75000002909D5C16920220A43C2610121F96695
:10A76000890502680A4302600421284600F090F837
:10A77000207840B22C4600250028C0D42B48006821
:10A780007D21C900F5F7A6FC20492D314143204623
:10A7900000F050F803F000FF04463868C069C007B5
:10A7A00005D003F0F9FE001B31888842F5D903F08B
:10A7B000F3FE04463868C169890706D503F0ECFE4C
:10A7C000001B31888842F5D938680121009A116050
:10A7D00017498161284603B0F0BD0321216000289C
:10A7E0008AD08AE7034804A1084A09A303F002FFBC
:10A7F0003093010218260100666C6173685F73650F
:10A8000063746F725F657261736500002B020000F4
:10A81000736563746F7220696478206973206F7642
:10A8200065722072616E67650D0A0000D4DC01025A
:10A83000000093EBF0B583B001917C22029042437B
:10A8400053498C182546143503F0A6FE064602210E
:10A85000029800F01DF803F09FFE07462068C169CA
:10A86000890606D403F098FEC01B29888842F5D9D2
:10A870002068007DC00708D06420FEF7CDFD03F0FE
:10A880008BFE801B01998842E1D903B0F0BDC04620
:10A89000F0B585B0049104467C2060433C490F1814
:10A8A0003D46143503F078FE06463868C069C00797
:10A8B00005D003F071FE801B29888842F5D903F08A
:10A8C0006BFE06463868C069800705D503F064FE54
:10A8D000801B29888842F5D91421049B5943DC2028
:10A8E00060432C4A1018039002914018018A826834
:10A8F000C47C7426BE5D012E0DD10191012B0299FD
:10A900000CD0012B0DD07526BE5D012E0ED0019E00
:10A91000072B0ED10EE00E4602990BE00222012B0E
:10A92000F1D138247526BE5D012EF0D10326072B08
:10A9300000D0019E184B334024069207D20A121908
:10A94000D218039B5958C907490C52184168CB07C4
:10A950001B0CD218837C5B075B0BD218C0684007C6
:10A96000000A10183A685060002E0ED001290CD150
:10A9700003F012FE04463868C069800705D403F06E
:10A980000BFE001B29888842F5D905B0F0BDC046F2
:10A9900030930102D41B0100FF3F0000F0B59DB0D1
:10A9A0000D460126890E2FD0002B2DD0119281212A
:10A9B000C9041093C91AA94226D30121EFF31084C8
:10A9C0000C4002D1EFF3108272B67C220F9042430A
:10A9D000E74814928718384610303B690026062B4A
:10A9E0000DD80A469A40D3065B0F07D161231A425D
:10A9F00000D16FE30E46002C03D003E00226002CAA
:10AA000000D162B6002E02D030461DB0F0BD0290DB
:10AA1000BD650021139179651098401E1290401970
:10AA2000B964B9690D916E1A1199B962FD62386302
:10AA30007E63F98C0E913046F5F74CFB0446B86303
:10AA4000129830180E9E3146F5F744FB109B011BFF
:10AA50004A1CF86339647A64139A0029194608D0AD
:10AA6000704359190D9BC91A0A1A7443581B80194F
:10AA70000119384648300E90384644300D9038461B
:10AA800040300B90384626300590384658301390A9
:10AA9000384654301290F9643A651498B44908580D
:10AAA0001021C1613846143014903846503004905B
:10AAB0003D464C3503F070FD04463868C069C00659
:10AAC00006D503F069FD001B149909888842F4D962
:10AAD000F87D40060C9500D574E201230E980360C2
:10AAE0000D98016800290F9800D1CDE23A467432E2
:10AAF0000A92DA0407921A0509921922520606925E
:10AB00000722D206089216E09A4800687D21C90003
:10AB1000F5F7E0FA109941430F9C2046FFF78AFEB3
:10AB200020460C9D0E9A11684B1C13600D99096804
:10AB30008B4200D9A8E20B9A1268012A55D0002A4C
:10AB400000D0A8E02E6812990C6813990D680621B0
:10AB50001091FFF79DFE386885601198051903F084
:10AB60001BFD04463868C069C00706D003F014FD19
:10AB7000001B149909888842F4D903F00DFD04469E
:10AB80003868C169890707D503F006FD001B1499D1
:10AB900009888842F4D938680A990A78012A0899FC
:10ABA00000D00699012A099A00D0079A3346724CC0
:10ABB000234013430B4371490B434360002EA3D042
:10ABC00003F0EAFC04463868C069800706D403F045
:10ABD000E3FC001B149909888842F4D93868297865
:10ABE00001756D1C761EFAD18EE7012B00D0C7E0EF
:10ABF0002E6812990C6813990D6806211091FFF7C1
:10AC000047FE386885601198051903F0C5FC0446B5
:10AC10003868C069C00706D003F0BEFC001B149959
:10AC200009888842F4D903F0B7FC04463868C16942
:10AC3000890707D503F0B0FC001B149909888842E6
:10AC4000F4D938680A990A78012A089900D0069937
:10AC5000012A099A00D0079A3346474C23401343F0
:10AC60000B4346490B434360002E69D003F094FC2C
:10AC700004463868C069800706D403F08DFC001BC9
:10AC8000149909888842F4D93868297801756D1CAF
:10AC9000761EFAD154E0012B00D0C9E02E6812993B
:10ACA0000C6813990D6806211091FFF7F1FD3868C3
:10ACB00085601198051903F06FFC04463868C06977
:10ACC000C00706D003F068FC001B1499098888426D
:10ACD000F4D903F061FC04463868C169890707D5D7
:10ACE00003F05AFC001B149909888842F4D938688B
:10ACF0000A990A78012A089900D00699012A099A26
:10AD000000D0079A33461C4C234013430B431B4986
:10AD10000B434360002E13D003F03EFC044638681A
:10AD2000C069800706D403F037FC001B149909881A
:10AD30008842F4D93868297801756D1C761EFAD1DD
:10AD40000C4800687D21C900F5F7C4F9109941430A
:10AD50000F9C2046FFF76EFD20460C9D2A68139B32
:10AD6000196889181960129B196889181960D9E641
:10AD700030930102D4DC0102FF3F0000008080001C
:10AD80008B4200D0CEE604990E6812990C68139994
:10AD90000D6806211091FFF77BFD386885601198DA
:10ADA000051903F0F9FB04463868C069C00706D0EE
:10ADB00003F0F2FB001B149909888842F4D903F0D0
:10ADC000EBFB04463868C169890707D503F0E4FB4B
:10ADD000001B149909888842F4D938680A990A78BE
:10ADE000012A089900D00699012A099A00D0079AE9
:10ADF0003346D44C234013430B43D3490B434360A6
:10AE0000002E00D180E603F0C7FB04463868C06915
:10AE1000800706D403F0C0FB001B14990988884200
:10AE2000F4D93868297801756D1C761EFAD16BE665
:10AE3000129A1268119CA618139A15688B425FD15A
:10AE400004990C6806210391FFF722FD386885609C
:10AE500003F0A2FB05463868C069C00706D003F0BE
:10AE60009BFB401B149909888842F4D903F094FB9A
:10AE700010900C9D3868C169890708D503F08CFBD8
:10AE80001099401A149909888842F3D938680A99A8
:10AE90000A78012A089900D006991091012A099A86
:10AEA00000D0079A2346A7490B40134310990B4340
:10AEB000A5490B434360002C14D003F06DFB1090A8
:10AEC0003868C069800707D403F066FB1099401A00
:10AED000149909888842F3D9386831780175761C4D
:10AEE000641EFAD19A4800687D21C900F5F7F2F88E
:10AEF000039941430F9C2046FFF79CFC204611E636
:10AF000005990C8806210391FFF7C2FC386885601B
:10AF100003F042FB05463868C069C00706D003F05D
:10AF20003BFB401B149909888842F4D903F034FB99
:10AF300010900C9D3868C169890708D503F02CFB77
:10AF40001099401A149909888842F3D938680A99E7
:10AF50000A78012A089900D006991091012A099AC5
:10AF600000D0079A234677490B40134310990B43AF
:10AF700075490B434360002C14D003F00DFB109077
:10AF80003868C069800707D403F006FB1099401A9F
:10AF9000149909888842F3D9386831780175761C8C
:10AFA000641EFAD16A4800687D21C900F5F792F85D
:10AFB000039941430F9C2046FFF73CFC204605992E
:10AFC0000A88CCE65E4815A90A4678C878C278C8CF
:10AFD00078C20125E8073A68136803431360B8682C
:10AFE000FEF78AFA02200026139C2168BA6AF965E6
:10AFF0003A6610997966BE66F8660C980068129AEF
:10B000001168091811600E9B19684A1C1A602268A1
:10B0100010182060002900D0F6E410953846603002
:10B0200013903C465C3438460830129006210F9845
:10B03000FFF72EFC3868216881600C980068119039
:10B0400003F0AAFA04463868C069C00706D003F0C6
:10B05000A3FA001B149909888842F4D903F09CFADA
:10B060000446109D3A68D069800707D503F094FA2A
:10B07000001B149909888842F4D93A687420385C16
:10B0800001282DD0E9042CE003F086FA0446386844
:10B09000C069C00706D003F07FFA001B1499098825
:10B0A0008842F4D903F078FA04463868C169890700
:10B0B00007D503F071FA001B149909888842F4D966
:10B0C00038680121029A11602249816100263046C8
:10B0D0001DB0F0BD04210160002C00D191E491E489
:10B0E0002905119C174B2340591801280C9D02D0AB
:10B0F0001920400601E00720C00608181249401830
:10B100005060002C0ED003F047FA04463A68D0692C
:10B11000800707D403F040FA001B1499098888427D
:10B12000F4D93A682B681398016812980068074CA4
:10B1300000941432FEF750FA30461DB0F0BDC04600
:10B140004C1A0100FF3F000000808000E59D0000D8
:10B15000D4DC0102000093EB3920C00001490968EA
:10B1600008587047BC920102F0B5032920D8C046A8
:10B170007944097949008F4401080F150121814064
:10B180004F4B1B685963D96212E0012181404C4B3F
:10B190001B681963D9620BE001218140484B1B6891
:10B1A000596304E001218140454B1B681963996292
:10B1B00083004349CB18DA608A68002A29D14A689B
:10B1C000002A16D4032314469C43174BE5589607D0
:10B1D000F60EFF27B740BD438027B7402F43E75007
:10B1E0001F23134001229A40104B1A60104B1A6023
:10B1F0000FE09307DB0EFF259D400F241440083C11
:10B2000003229443074AA658AE4380259D40354308
:10B21000A550012282400868026288681043886055
:10B22000F0BDC0461CED00E000E400E080E200E07C
:10B2300000E100E010B501242046FEF715F8204695
:10B2400002F0EEFE002010BD012181401C48006884
:10B2500042688A4342607047194909680968C140D9
:10B26000012008407047C046012181401448006811
:10B2700042680A4342607047012907D0002910D173
:10B28000012181400F4802680A430FE001218140FB
:10B290000B4800684368002A0DD00B4343600161EE
:10B2A000704701218140074802688A4302600448D0
:10B2B0000068416170478B43436001617047C0463D
:10B2C000C09301020801004080B5114A1170114A73
:10B2D00010708001C90101430F4800784001084304
:10B2E0000E490978090101430D480078C000084360
:10B2F0000C490978890001430B4800784000084355
:10B300000A4909780143C8B2F9F7BAF880BDC046C6
:10B31000889D01023696010215940102F0E40102B3
:10B3200079AB0102899D010204A1010205A101027C
:10B33000012282400548002903D0016811430160C1
:10B3400070470168914301607047C04600010040AA
:10B35000124A072809D880000F23834081401940F2
:10B36000106898430843106070470F280AD880007F
:10B3700020380F2383408140194050689843084388
:10B3800050607047800040380F238340814019404F
:10B3900090689843084390607047C046340000406E
:10B3A000F0B54307DC0E0726A640C3089D000E4BF0
:10B3B000EF187D68B5433E1D002908D03560012295
:10B3C000824001290CD1186810431860F0BD01219A
:10B3D0008140186888431860A24015433560F0BD6D
:10B3E000186890431860F0BD0C01004010B582B0A1
:10B3F00014460A460146049800930190082023460B
:10B4000000F092F802B010BDB0B584B014460A4600
:10B4100001460898022500950193029007202346D3
:10B4200000F052F904B0B0BD70B500285BD03149CE
:10B430000A783149002A03D14A68012313434B603B
:10B44000428803881B049A180B46183B1A608288AE
:10B4500083891B049B180C460C3C23600B46083B5D
:10B4600084681C60446903232340057CAD00EB180D
:10B470008569AD072D0D5B19457C2D035B19C569E9
:10B48000AE07B60A9B19867CB6059B190E1F336062
:10B49000036A122B04D107240C60541EA2410AE057
:10B4A000032C05D1012D03D807220A60012202E0F6
:10B4B00006220A600122114C002525700F24640128
:10B4C0002034C57C6D0225401B069B0BD218C37926
:10B4D0001B07DB0ED21880790007C00D1018401929
:10B4E0001439086070BD064806A1862209A303F03E
:10B4F00081F8C046BCCA010218100050BECA010241
:10B50000F53201006C73705F656E67696E655F721E
:10B51000756E0000506172616D65746572206973AB
:10B52000206E756C6C000000F0B58BB0109E34047A
:10B530003ED00D46D64C2140012701977F06B942E7
:10B540003CD111462140B9423FD11C40BC4243D1BD
:10B55000119902AC0027E781E78066802780278267
:10B56000A774E1749908A181A908A1800A9009979C
:10B5700008970797900880B204902046FFF754FF81
:10B58000AA480078002801D00BB0F0BDAB48016894
:10B59000C90708D10168C90705D10168C90702D1E7
:10B5A0000168C907F3D07F48019901700BB0F0BD65
:10B5B000B8480D49AF22C14B03F01CF80095B548BF
:10B5C0000949B022754B03F015F80092B1480649BD
:10B5D000B122724B03F00EF80093AE480249B2223A
:10B5E0006E4B03F007F8C046CB320100F0B58DB0CA
:10B5F0000392139E340446D00A46A54C21400125EF
:10B6000002956F06B94244D103992140B94247D10E
:10B610001C40BC424CD11499129D04ACE1742949E0
:10B6200021820027E781E780668027809908A18131
:10B630009108A1800B95012D01D16121CF43A77401
:10B640000C9002200A9009900398800880B206901E
:10B650002046FFF7E9FE75480078002801D00DB0BC
:10B66000F0BD76480168C90708D10168C90705D14E
:10B670000168C90702D10168C907F3D04948029996
:10B6800001700DB0F0BD83480D49FB228B4B02F0D9
:10B69000B1FF00927F480A49FC22404B02F0AAFF0A
:10B6A000039800907B480649FD223C4B02F0A2FF24
:10B6B000009378480249FE22384B02F09BFFC046B7
:10B6C000D83201008E8E0000F0B58BB0119E34048C
:10B6D00047D00D466E4C2140012701977F06B942A5
:10B6E00045D111462140B94248D11C40BC424CD101
:10B6F0001299109F02ACE174294921820021E18155
:10B70000E180668021809908A181A908A18009971C
:10B71000012F01D0712100E06121C943A1740A9079
:10B72000032008900790900880B204902046FFF70D
:10B730007BFE3E480078002801D00BB0F0BD3F48AA
:10B740000168C90708D10168C90705D10168C9079F
:10B7500002D10168C907F3D01248019901700BB0FA
:10B76000F0BD4C480C49D522544B02F043FF0095E4
:10B7700048480949D622094B02F03CFF009245484F
:10B780000549D722054B02F035FF00934148024995
:10B79000D822024B02F02EFFE732010015330100E0
:10B7A00086860000BECA010210B582B014460A4661
:10B7B000014600200093019004202346FFF7B4FEC9
:10B7C00002B010BD10B584B014460A4601460020F0
:10B7D00000900193029004202346FFF707FF04B076
:10B7E00010BD000070B50D46064604242046FDF746
:10B7F0003BFD204602F014FC0B4805600B48067028
:10B80000002E0ED00A48016880220A437F218A4315
:10B8100002600120000307490860074908600748E3
:10B820000460002070BDC046C0CA0102BCCA01024B
:10B830000CE400E080E200E000E100E01C100050B9
:10B84000B0B582B0144602461148204001256D066D
:10B85000A8420DD1180413D01748016000200093AE
:10B860000190062011462346FFF75EFE02B0B0BDF0
:10B870000094FF228C320748074908A302F0BAFE61
:10B88000FF208C30421C034803490C4B02F0B2FEEF
:10B890000300FCFFF5320100BD3201004473742047
:10B8A0006164647265737320257820697320696E02
:10B8B00076616C69640000000810005033330100A9
:10B8C00080B582B00B460146002000920190032013
:10B8D0000A46FFF729FE02B080BD0000002801D013
:10B8E000042100E00221C24A5172411E88418001B8
:10B8F00003490A6840239A43101808607047C046FD
:10B9000050A00050F0B583B002912E49CD7A0E7B45
:10B91000771987424FD90899019118254543412647
:10B92000F604BF00BE19745B34490C4057033C1940
:10B930009B07D90C6418324B1B681B7A745375191A
:10B940006C880326B60326409B079B0C9B193F245B
:10B9500004401819029CA3061B0DC0186880012A18
:10B96000184E13D8707B14224243307B502343433C
:10B9700024011B199A18F37AC0181C234343D018CA
:10B9800080081E4A104007430F432F8001986860CB
:10B9900001F0CAFEA860E8681A4908403030E86043
:10B9A000286908402721715C4018286100F05CFE7E
:10B9B000686103B0F0BDFF228832034803A108A3E9
:10B9C00002F018FEC4CF0102843301006D61635F91
:10B9D00063735F636F6E737472756374000000004D
:10B9E000435320696E646578206973206F766572B1
:10B9F0002072616E67650D0A00000000FF070000FD
:10BA00002C9401020000F0FFF0B581B000931446C1
:10BA10000D46074606263046FDF726FC304602F066
:10BA2000FFFA26211D4847540021017041708171A1
:10BA3000017181704171C170C17102224272C16293
:10BA400001634163816304734273C572009A561C9B
:10BA5000134A168001724120C00401214903F4F702
:10BA60007CFB502060432901081861198A00801866
:10BA700018224A438018B2B24A4380180949401834
:10BA80000949884204D200F0B5F8002001B0F0BDA9
:10BA9000064807A19A2209A302F0ACFDC4CF010217
:10BAA000C0CF0102280008020120080284330100EF
:10BAB0006D61635F696E697400000000454D206F21
:10BAC000766572666C6F770D0A000000A448C17934
:10BAD000002901D001207047007A411E884170473B
:10BAE000F0B583B002912A494B7B834248D9CB7A87
:10BAF0000C7BE31818245C439B00E3184124E40406
:10BB00001A191424019005466543002656510092E7
:10BB10005519EE882E4F0B467A1C3240F54E36886A
:10BB2000497A711A2B4E0E40B618EE803740997B39
:10BB3000EF80AA88284F17404A424A41910079185D
:10BB4000264A8918A980264F0F402D1D02980128EA
:10BB50000AD124490E400921C902711869800121C6
:10BB6000C9037918298000E02F8001984443009888
:10BB70000019074A918C4182118C018203B0F0BDFB
:10BB80003520C200034804A109A302F033FDC046DA
:10BB9000C4CF0102843301006D61635F6C696E6B19
:10BBA0005F646573635F636F6E7374727563740053
:10BBB0004C696E6B206465736320696E64657820E0
:10BBC0006973206F7665722072616E67650D0A0079
:10BBD000FFFBFFFFFF03000003D0FFFFE80F0000A3
:10BBE000EF1F0000FF830000BE4A5063916370475F
:10BBF000C4CF0102F0B581B04348CC2101600321DC
:10BC00004160B8490A7BD304404C1B19CC7AA21876
:10BC1000541E1C431823534392009A184B7B14253F
:10BC20005D43521992012243012463061343436189
:10BC300000228262C262026342638263C26342651F
:10BC40000267334B1A605A609A60324B1A601A616D
:10BC50009A61DC61304C1C62304C251D1D63254609
:10BC60000C3D5D632546283D9D632D4EDE631C64BF
:10BC70005C642C4D2F461C379F642746143FDF64BD
:10BC8000103C1C65284C5C65284C9C650C369E67F6
:10BC9000274CA5634035E563DA651A665A669A66ED
:10BCA000DA661A67234DDD6702258561224DC5617D
:10BCB000C325AD03CD620A63D2435A601F4A13689D
:10BCC000FF25AB4326254D5DAD072D0EEB18136008
:10BCD0001B4A102313601B4A1360272260238B54D6
:10BCE00019498160C160016121607D2109010166FE
:10BCF00041661649C164164941641649016400F061
:10BD0000A3FC01B0F0BDC04604A000500000F8FF45
:10BD100094A0005034A10050FF185A003004004095
:10BD2000041000401C20004054300040604000409F
:10BD3000B8A1005014001400FF3F3FFF04E400E0EE
:10BD400080E200E000E100E0DC05DC053F0270027B
:10BD50000133D007D007D0072921C64A5054704775
:10BD6000C4CF0102F0B58BB0079208910146C14FD4
:10BD7000B8780991FFF7B4FE78793A7B7979069122
:10BD8000824200D89FE0FB7A9A181823534392000E
:10BD90004124E10404915218D2187B7B14214B43B7
:10BDA000D21850246043155801230A93DB022E4613
:10BDB0009E4316504E4B2B4005937D7B03914D4384
:10BDC0003E7B7443F97A0B011B195B1971181C2413
:10BDD000029461435918A84B1B88069C5C430919BF
:10BDE000C904490D059BC9181150101807994160E5
:10BDF00038787979089A00920322099BFFF782FD2F
:10BE0000F87A397B09183878814263D9830009931D
:10BE1000049AD45C0894F7212140D154D1184D786C
:10BE20008E7836027619CB781B04F31807900A989F
:10BE300086051E43330CCB70FB7A387BBC784D7083
:10BE40009F4D3540039E6643C018029B434398199B
:10BE500040029C4B03405C19200A8870200CC8707B
:10BE6000F023089D2B401B1D3D7B0895FE7A099D04
:10BE70005355C8700620079A50438019089A8018B5
:10BE800048701F22D20222400243100A887078793B
:10BE9000401C7871387B7979814201D30021797116
:10BEA0003978491C3970F97A08183978884201D8EC
:10BEB0000020387028200A993954387A401C38728A
:10BEC000387A0BB0F0BDA7204200D2480649074B94
:10BED00002F090FBA72042007A32CE487349744B9F
:10BEE00002F088FBC4CF0102A43301004D330100EE
:10BEF00000F0FFFFC0CF01020320000605490A68D9
:10BF000082430A600A6802430A6003480121016013
:10BF10007047C0461C0000401CA0005080B50120A6
:10BF2000FDF758FC80BD0000F0B587B006930646CB
:10BF3000504C607A504B1B88181A0C9DA84200DCAC
:10BF400089E00F460592012E06D156480021C162B4
:10BF50000169554A89180160A0783146FFF7C0FD94
:10BF6000E078E178069A2B4600F0AEF82078E17888
:10BF70000097002206923346FFF7C4FCE07A217B4B
:10BF80000818217888426ED94120C20404918800A3
:10BF9000815C0391F7250D40029285544549455C2B
:10BFA0004549465C360276194449475C3F04F61918
:10BFB0000127BF0537433E0C4654E67A217BA37820
:10BFC0003C4A85543E4D3D4014275F4389191C234C
:10BFD0004B43D91949023B4B0B405D19290A364B9B
:10BFE000C1542E0C35494654F02703990F4005994A
:10BFF000002900D13F1D217BE37A029A87542F4A02
:10C0000086540622049E7243D2185118294A81543C
:10C010001F22D20215400D43290A274A8154E07895
:10C02000401CE070E07AE178814201D30699E1702A
:10C030002178491C2170217B08182178884201D879
:10C0400006982070E079401CE071A07A401CA07234
:10C05000E07907B0F0BD3920C2001632074808A1C8
:10C0600009A302F0C7FA3920C20004480F49104B57
:10C0700002F0C0FAC4CF0102C0CF01028433010034
:10C080006D61635F747800004D4143205458206C0B
:10C09000656E206973206F7665722072616E6765C8
:10C0A0000D0A00000804004090D00300BA330100DC
:10C0B0006B330100010008020200080203000802BD
:10C0C000FF07C0FF00F83F00F0B589B00893019268
:10C0D00004914F4DEF7A874200D891E0297B50269A
:10C0E00032464A434124E3040693D218CC19A100F6
:10C0F00051181822059254430A19697B1423079397
:10C100005943531802900001195804460390504AAD
:10C110000A40A97AC902511808988205D2088A18DB
:10C120001A514C4911402A7B00965643384CE57A07
:10C130002C0106982418A719354E5419A5007D190D
:10C14000059844432819747B079D6C430519049F87
:10C15000D2194148048854432A19089CD204520D2C
:10C1600051181D460398195000F088FA0146707A5C
:10C17000001902043E460CD080B2C000002900D154
:10C18000801E029FA5214900F3F7A4FF1F21014053
:10C1900001E00021029F38012818427983791B02AF
:10C1A0009A18C3791B04D2182C4B1340437109040D
:10C1B0005918090CC171002C20D015483546064687
:10C1C000007B009B4343F17A0A01069F3A43D21851
:10C1D00041188B00D218059B4B43D118727B079BEB
:10C1E0005343C91840191C4A1288424388180199C0
:10C1F000884203D001992246F3F796FF09B0F0BDBB
:10C20000FF225C32034804A109A302F0F3F9C046FF
:10C21000C4CF0102843301006D61635F74785F6491
:10C220006573635F636F6E7374727563740000008F
:10C230005458204445534320696E646578206973DF
:10C24000206F7665722072616E67650D0A000000CE
:10C25000FF0700E000F8FFFFC0CF0102EFFFE000A2
:10C2600082B0FCF71DFE052000252946FFF770F877
:10C2700006202946FFF76CF80A202946FFF768F8E0
:10C2800009202946FFF764F80124204603F074FBD7
:10C290002846254603F070FBFCF73EFE2046FCF7DF
:10C2A00031FE01F03DFE01F035FE7C4801687C481E
:10C2B0000068890308D40321090708402907884238
:10C2C00002D0FCF7BBFD06E0FCF74CF9FCF7CEFD15
:10C2D0000020FDF7C5FCFCF759FE0024204604F0C1
:10C2E00069FC03266FA23046314603F0DFF9304681
:10C2F0002146FBF709FCF8F7C1F9FBF765F8FEF7F3
:10C3000099FF6E4F381DFCF7F1FBF7F7AFFEF6F71C
:10C31000ABFEF8F740F9042630462146FFF718F83F
:10C32000304629462246FEF7A7FF05223046294619
:10C33000FFF736F8019420462946FEF7C5FF754EF3
:10C34000304628305E4A00902946FCF741FBFAF758
:10C3500081FBAA025B495C4B284603F00BFE01F00F
:10C36000BDFBF6F76FFE594A2846294602F058F8F9
:10C37000574802F085F85748FCF74AFD78780028BE
:10C3800010D107E0F8F772F94142414171637878C2
:10C39000002807D1F8F76AF9002803D1F0790028BE
:10C3A00016D140E0FCF7AAFCB079002803D0019830
:10C3B000B071F6F7B5FCF8F76DF9F7F77FF9F7F715
:10C3C000AFFBFBF70FF8FCF777FCF07900282AD0D9
:10C3D0002C460198F071B078411CB1703D2806D30D
:10C3E0000020B07001210098354AFCF7F1FAFBF704
:10C3F000A3F9012538480570F8F738F9002802D06C
:10C400000198787005E0F0781E2800D3019D7D70BA
:10C41000401CF070F7F7C0FB7F20C105F069F3F70F
:10C4200074FFF06125460B20FEF716FF39780028CF
:10C430000BD0002916D1012028490870387000203F
:10C440002749087003F072FA0CE001290AD1002094
:10C4500038705D49C883214908700120204908705F
:10C4600003F040FAFBF7A0F90B20FEF7F5FE41427E
:10C4700041413163F8F7FAF8002805D00020FAF7B7
:10C48000F7FD0028294681D17878002800D179E786
:10C49000002171637878002884D17BE71800004080
:10C4A000300001405557422073696D706C652065FE
:10C4B00078616D706C650D0A000000001C9001022F
:10C4C000C5880000C0CB0102AD010100D5E300002A
:10C4D0007C3F00000DC50000369601021890010255
:10C4E00019900102014800687047C0460C000040E6
:10C4F00081B080B581B0039303AB009302F050FD8F
:10C5000001B080BC02BC01B0084700000148002116
:10C51000C1617047A0970102F0B581B00026304696
:10C520003146FDF703FE0125AC022649264F304671
:10C530003A462346FDF75AFF3988244881423FD0C6
:10C5400064217E5262217E5260217E524422BE527C
:10C55000FD87BD8778227A8702223A874322FA86AE
:10C56000BE83FE811A4ABA817E810A223A81194A23
:10C57000BA803880FE8306203885F984FF20123087
:10C5800078840146E331F9808730B88450203E52E8
:10C590003A83EFF3108072B630463146FDF7C6FDA0
:10C5A00000280CD12A0300263046064D2946FDF707
:10C5B00017FD054A304629462346FEF7EFF962B6D5
:10C5C00001B0F0BD00E0020412A70102AA5500006C
:10C5D000E1FF0000341200000020704710B5002475
:10C5E000002809D0002905D003464A00034819460F
:10C5F000F3F79AFD204610BDE04310BD24930102DD
:10C60000014600200A2901DAC0437047014A11801F
:10C610007047C046AC9301020020704780B5018886
:10C62000064A11808178064A1170C178054A117056
:10C630000079FCF787FB002080BDC04616940102FC
:10C640001894010210D00102044805490160152127
:10C6500009044160034981607047C0469C30004036
:10C66000410008003400070007480068406970472F
:10C67000FD20400004490968085C704702480068D2
:10C680006221405C7047C0462C9401020A491A227C
:10C690000A600A4948704878FF210902084A13686D
:10C6A0008B43800380B2C0181060064820210160CF
:10C6B0000548016000207047702000401C94010272
:10C6C00004E400E080E200E000E100E0F0B5A9B0A1
:10C6D00016460F460546C648002B024600D01A46AD
:10C6E0003921CC003D21C900511811918242189284
:10C6F00006D001204202BE491898F3F715FD189A9A
:10C700006120111913910E21119C0A91A170002F23
:10C710000D9501D00A2100E00921592317938300C8
:10C72000E170784278411399087030781090107059
:10C73000F17AE17471785170B7789770F178D170AF
:10C740003579157174795471B1799171F179D1712B
:10C75000317A1172717A5172B17A91727E1EF0B291
:10C7600000210328169106D870B28000A1A21058AB
:10C770006A00805A1690179882001898C018149072
:10C78000F81E022804D3012E084604D89D4800E074
:10C790009D48031918781290189DA81817902846DC
:10C7A000303015902C4656346D2080002950974A21
:10C7B000974B149E33627262B362F2623176F182F9
:10C7C000139B597009229A70281841608160C160DA
:10C7D0000161109880008F490858F4F7DFF8012FA5
:10C7E00010900F9104D0022F05D17F217E2004E00C
:10C7F0007C217B2001E05B215A20159DA9842070BB
:10C8000003200C90A080012666701F200B90A88248
:10C810001820A8740A46083A179BDA76169B129AD3
:10C82000D2184A439100189A9163B702791E8B423D
:10C830000E9109D97848608034206884774828822E
:10C8400077481399088339E07F2B10DD802B18D0AF
:10C8500031028B421BD071028B4227D16E4961801D
:10C8600068846F4813990883CF20C00025E0202BEF
:10C8700017D0402B1AD1684860800420688469482A
:10C880001BE06548608006206884674815E06248C0
:10C89000608010206884624813990883C520C00016
:10C8A0000BE0624860800220688404E00420688411
:10C8B000812040006080FF2002302882104600F076
:10C8C000D7FE1298102806D0402808D108201499C5
:10C8D000C876072000E004201799887002E01798B6
:10C8E0000C9981701898169A8078C11E02290CD371
:10C8F000022811D001280CD12672BA4200D9002694
:10C900006672BA4213D8F44812E00D200002119961
:10C9100008800120800201E00C9800022081BA42C8
:10C9200001D8EE4800E0FA20179988600EE0FA205E
:10C9300017998860139800780028119901D0E84869
:10C940004880E848139A1083E7480880A88CF3F7DA
:10C95000C5FF0026E54B3246F3F75EFE02460B4666
:10C96000E3493046F3F7C0FEE24B3246F3F754FE9C
:10C97000F3F7F0FF0746E080DF493046109A0F9B3F
:10C98000F3F7B2FEDD4B3246F3F746FEF3F7E2FF74
:10C9900078434042800B608116990E98814208D9F5
:10C9A0000C20149FB872D648179988831220189AC1
:10C9B0000EE0480A189A149F01D00D2003E0080ADF
:10C9C00000D1DBE20A98B872CE481799888312200A
:10C9D000F872D078052844D878440079400087441C
:10C9E0000227402C3339C848B881C8482FE0C046D8
:10C9F000BC900102FC190100FC1901000C1A010095
:10CA00000C1A0100EA160100F11601003075000051
:10CA100010270000AC17010005020000FF0600000F
:10CA2000040800000A0400003604000003020000AD
:10CA3000B748F881B748388013E0B748F881B7485D
:10CA40003882B74838600CE0B448B881B5481799C7
:10CA5000C88306E0B4487882B448B8800B980006D2
:10CA60009064AE483881A748F880B14802882A848B
:10CA7000B0480078E874B0480078119F7875387D28
:10CA8000139000285ED0AD490A681023DA413A605D
:10CA90000A794B79CF8867801B029A186A840A7AD0
:10CAA0004B7A8F7AC87A0D7B65701B029A183B040B
:10CAB000D21800061018179FF860487B8A7BCB7B42
:10CAC0003B77120210186081087C7877487C149AB2
:10CAD0009072887CD072C87C159B1874087D58743D
:10CAE000487D11909874C87D0A7E120212181A842B
:10CAF000887DD87418464B7EC375887ECD7E2D0206
:10CB00002818B880087F4D7F2D022818F880887F6C
:10CB1000B877C87FF8772020085C149D28732120FF
:10CB2000085C68732A20085C2A314D782D02281889
:10CB30008D782D044019C978090640181899886421
:10CB4000119801E0EB7DA87C7D498B700A80800004
:10CB50001F38C882C883139800281FD02222774824
:10CB6000825C034622335B781B029A180A842422D3
:10CB7000825C034624335B781B029A18CA842622FF
:10CB8000825C034626335B781B029A188A8328222C
:10CB9000825C283040780002801888846948032528
:10CBA00069A2294602F082FD189F387814907B789C
:10CBB000B8780F90FA78B8791390F8791190387A9C
:10CBC0001090787AB97A0890099100930F980190A3
:10CBD0000292169803901298049013980590119859
:10CBE000069010980790FAA2F8482946149B02F084
:10CBF0005DFD3D46643580212846F3F7AEFAB878EE
:10CC0000C11E02290ED3012800D18FE1022800D0D5
:10CC1000ABE11691149078787F225043F749401881
:10CC2000F74907E01691149078785B225043F14958
:10CC30004018F14941182846F3F776FA0D9D1898E7
:10CC4000C6870E34324602E0641C0F2A0ADA2178C5
:10CC50000029F9D0491C8907C90F91400E43C687A6
:10CC6000521CF1E71699022907D31499491E01298C
:10CC700000D97DE14279D24901E04279CF49891852
:10CC80000C78002D00D177E1C1790E91032900D9EC
:10CC90004AE14279062A00D979E1492189004118FF
:10CCA0001191E43010900E98401E129019A80019AE
:10CCB0000F9000231392149403E01898290600D1D2
:10CCC0005AE1052A5AD8C0467A441279520097444C
:10CCD000455C728598ABC04688130000E2040000F2
:10CCE0000C080000060A0000040F000000001041BC
:10CCF00030C1BD41000070400000F0400000D04154
:10CD0000120C0000140B000012120000140E0000A0
:10CD10000E160000130D0000121600000E12000087
:10CD2000140B0E0A12080000101600000E0B000073
:10CD3000169401021894010210D001021CD00102C5
:10CD400084940102010800004361736520706172E0
:10CD5000616D65746572733A200D0A001693DFB237
:10CD6000002F04D019A801223946F3F7EFF9002C5F
:10CD700000D191E019A8C019BB498AE0E8B20228A5
:10CD800067D00027022867D06BE00E98022872D186
:10CD9000E8B2022800D103461693DFB2002F04D078
:10CDA00019A801223946F3F7D1F9002C74D019A83B
:10CDB000C019ACA16DE0E8B2022800D1042316939B
:10CDC000DFB2002F04D019A801223946F3F7BEF9CB
:10CDD000002C61D019A8C0199FA15AE0E8B202281E
:10CDE00000D106231693DFB2002F04D019A8012228
:10CDF0003946F3F7ABF9002C4ED019A8C01992A10F
:10CE000047E0E8B2022800D10C231693DFB2002FCE
:10CE100004D019A801223946F3F798F9002C3BD029
:10CE200019A8C019874934E0E8B2811E4A424A4134
:10CE30009700022804D119A801223946F3F786F990
:10CE4000002C16D019A8C0197CA12246F3F76CF962
:10CE50000FE00627022804D119A801223946F3F76A
:10CE600075F9002C05D019A8C01980492246F3F79E
:10CE70005BF9169710E01693DFB2002F04D019A8C3
:10CE800001223946F3F762F9002C05D019A8C01920
:10CE900073492246F3F748F93C193F2C05D80F98FF
:10CEA000C0194021091BF3F758F912980228189865
:10CEB00001D2002002E0C078411E88411599087017
:10CEC000611E2E46E8B202280CD1179A517019A99A
:10CED000119AB8C9B8C2B8C9B8C2B8C9B8C2B8C935
:10CEE000B8C20DE0179A117019A9109AB8C9B8C242
:10CEF000B8C9B8C2B8C9B8C2B8C9B8C2C10709D19F
:10CF000080073546149C139A169B00D4D5E6022060
:10CF10008543D2E6FE20354605401898149C139AA6
:10CF2000169B290628D0CCE637A231E01691149042
:10CF300078780B994143334808181F386F21C9434B
:10CF40000D9D7A180378D427D3554378D827D35525
:10CF50008378DC27D355002900D170E6C378E02719
:10CF6000D3551031001D189FEBE70120404A10E017
:10CF70000024002D00D087E629B0F0BD80290ED313
:10CF80000F20B872104817998883102020E525A239
:10CF90000120014602F08AFB189829B0F0BD10204C
:10CFA000402904D3B8720849179B998310E5B872D9
:10CFB00004481799888314200AE5C046F116010039
:10CFC000EA160100150F0000140B00000108000014
:10CFD00025642025642025642025642025642025DF
:10CFE0006420256420256420256420256420256490
:10CFF0000D0A0000403D01001DF7FFFF58340100FD
:10D0000089FBFFFF483C01007472785F6D6F6465B7
:10D0100020706172616D65746572206572726F72E5
:10D020000D0A00004E73666420706172616D657454
:10D030006572206572726F720D0A0000FFFFFFFFBC
:10D0400001FF0000AC1A0100FFFFFFFFFF0101FF1D
:10D05000FF01FF01FFFF01FFFFFFFF01FFFF01FFD6
:10D0600098200100FFFF01FFCC1A01001C1A0100EB
:10D07000F6330100002800D10148064908607047D6
:10D08000BC900102F0B586B0002805D101480068C7
:10D0900002E0C0462C9401023121C90004914118DC
:10D0A0008A791F231A40CD79ED06AD0DAA180D7AA5
:10D0B000ED066D0C52194D7AED062D0B52198D7A35
:10D0C000ED06ED095219CD7AED06AD0852194D7CE9
:10D0D000ED075219BD4C22600A7B1A404E7BF606C2
:10D0E000B60DB2188E7BF606760C9219CE7BF6063C
:10D0F000360B92190E79F606F60992194E79F60654
:10D10000B608921962604A6AB14D2A40A2608A6AE2
:10D110002A40E2602D22D20087183A7E1A400393FB
:10D120007E7EF606B60DB218BE7EF606760C921915
:10D13000FE7EF606360B92193E7FF606F609921928
:10D140007E7FF606B60892190E7CF60792192261C8
:10D15000BA7F1A400597FE7FF606B60DB218049BFB
:10D16000C35CDB065B0CD2184B78DB061B0BD218BA
:10D170008B78DB06DB09D218CB78DB069B08D2184C
:10D180006261CA692A40A2610A6A2A40E2618A7C15
:10D1900001252A40CB7CDB079B0F9A180B7DDB0710
:10D1A0005B0FD2184B7D9B07DB0ED2188B7DDB0704
:10D1B0009B0ED218CB7D1B079B0D9A180B7E1B076D
:10D1C0009B0CD2184B7E5B06DB0A13438A7E520609
:10D1D00012091A43CB7E5B075B0813432362CA6ABA
:10D1E00062620A6BA2624A6BE2628A6B2263392234
:10D1F000D200835C1E462E4066635E425E41B304ED
:10D20000AE04744F3C68B443E3183B6083185A780B
:10D210002A409C782407E40EA2188C8F6401A2187F
:10D220006D4C1440C98FC905490A0919DA78D2072B
:10D23000120A89181A791207120989185A79D2071D
:10D24000D2088918FB4EB1639968F1639979049506
:10D250002940DA79D207920F51181A7B5207D20E61
:10D2600089185A7BD206920D51189A7B5207D20C1C
:10D270008918DA7BD206920B89181A7CD206520AD8
:10D2800089185A7C520792090A43997CC9064908B1
:10D2900051183164D97C039A11401A7DD206920D3F
:10D2A00051185A7DD206520C89189A7DD206120B5B
:10D2B0008918DA7DD206D20989187164197E0F2483
:10D2C00021405A7E120151189A7E12038918DA7E83
:10D2D0001207120A51181A7F1207120989185A7F69
:10D2E00012078918B164997F01942140DA7F1207EF
:10D2F000120E51183D22D200835C5B075B0D59185A
:10D30000841862781207520C8918A278D206120B80
:10D310008918E278D206D2098918F16421790722A6
:10D320000A406179C9008918A2795206920B5118F6
:10D33000E2799207120B8918227AD2078A18BF491C
:10D340000A60627AA37A1B029A18E37A1B04D21845
:10D350004A60E289BA4B13400394228AD2049209AC
:10D36000D2188A6003463033598CB64A1140029372
:10D370009A8CD205D20A51185622825C120689185C
:10D38000B14D2960014656314A788C782402A218A2
:10D390008C8864056409A218CC78240712196A6085
:10D3A000CA880C7AA407A40BA2184C7A6407E40A72
:10D3B0001219AA604989E960492189004118FF22B0
:10D3C0006632821800921035002207E000300040DB
:10D3D000FFFFFF0004040040FF3F000084186427A3
:10D3E000E65D03273E406523E35C9B071B0F9B190B
:10D3F0006626A65DB607B60EF3186726A65DB601CB
:10D40000F318DBB26826A65DB607B60DF3186926D9
:10D41000A65DB607360DF3186A26A65DB607B60CEC
:10D42000F3186B26A65DB607360CF3186C26A65DBE
:10D43000B607B60BF3186D26A65DB607360BF318C4
:10D440006E26A65DB607B60AF3186F26A65DB60768
:10D45000360AF3187026A65DB607B609F3187126CA
:10D46000A65DB6073609F3187226A65DB607B6089C
:10D47000F3187326A45DA407E31808C51032802AA8
:10D48000ACD1019AD243704EB4180B783B404D7822
:10D49000AD072D0FEB188D78AD07AD0EEB18CD78DD
:10D4A000AD01EB18DBB20D79AD07AD0DEB184D7981
:10D4B000AD072D0DEB188D79AD07AD0CEB18CD79BF
:10D4C000AD072D0CEB180D7AAD07AD0BEB184D7AAF
:10D4D000AD072D0BEB188D7AAD07AD0AEB18CD7AA1
:10D4E000AD072D0AEB180D7BAD07AD09EB184D7B91
:10D4F000AD072D09EB188D7BAD07AD08EB18CD7B83
:10D50000AD07EB18A3641031121DBDD1009B197833
:10D510005A785207520D51189A78D207120D89186D
:10D52000B164059B1968F164D97D5A6812025118DB
:10D5300031659968454A0A40998A49058918716593
:10D54000D9683D4C2140B16519692140F165029EC1
:10D550003178049D294082785207120F5118C27900
:10D560009207920E8918427A9207920D5118827A88
:10D570009207120D8918C27AD207920C89189A7DE7
:10D58000D207520C891872789207D20B8918B27898
:10D590001207D20A8918F2781207D2098A182C4980
:10D5A0000A60327C737C1B071B0D9A18B37C9B06A8
:10D5B0009B0BD218F37C1B079B0AD218337DDB062A
:10D5C0005B09D218737DDB071B09D2184A60B27D54
:10D5D0002A40C38F5B009A188A60826CCA60C26C52
:10D5E00022400A61F27D7F231340328C5204520A9A
:10D5F000D2184A6102698A614269CA6182690A6213
:10D60000C2694A62026A8A62426ACA62826A0A63BA
:10D61000C26A4A63039A927CD201121D0A64027A9A
:10D620003A40CA65808F074A10400866002006B05D
:10D63000F0BDC04600300040FFFFFF009C300040BE
:10D64000FF1F0000FF03000000400040FFFF1F001D
:10D650000020004004480068806B80080349096886
:10D6600049004018093070472C9401021004004012
:10D6700010B52D21C9004118027A032A04D100797E
:10D68000002807D0082006E08378DA1E022A05D297
:10D69000032412E0142088601C203DE0012B02D1FD
:10D6A000C8228A6012E00479042C01D3462404E0E5
:10D6B000032C01D1322400E014248C605B1E022B69
:10D6C00004D3022A10D24279154B01E04279154B5E
:10D6D0009B181B78402B04D0102B06D11423442414
:10D6E00005E02A233E2402E04279342348244B807B
:10D6F0000C80022A06D0062A08D0052A08D1182252
:10D700004C2301E0142250230B8000E01C224A80AD
:10D71000C078042803D1142048806420088010BDFC
:10D72000F1160100EA160100134800687047C04670
:10D7300010B5104A107091700F49002813D050682E
:10D740000861042048619078FF2212020B4B1C688C
:10D750009443800380B20019186001204007084AF2
:10D760001060084A106000200860074901220A6022
:10D7700010BDC0461C940102180400401CE400E0E7
:10D7800080E200E000E100E070000040F0B591B000
:10D79000002801D1C04800688778F91E022913D3F8
:10D7A000012F21D0022F3CD11021CA4344782146B9
:10D7B000193991423DD800970125B94A2846294692
:10D7C000234601F073FF53E10821CA434478214600
:10D7D0002139914218D800970125B14A2846294697
:10D7E000234601F063FF43E10821CA434478214600
:10D7F0000939914234D800970125A94A284629467B
:10D80000234601F053FF33E1032F3CD0042F43D1D3
:10D81000C3780125042B00D02DE106462A020423FB
:10D8200043E00125A6A2284629463B4601F03EFFDB
:10D830001EE1C3780125052B0AD806462A02284690
:10D8400098401B21084230D10021052B08462ED0DC
:10D8500002200090914A2846294601F027FF07E15F
:10D860000646C3780021022B1ED3032B1CD0042BA9
:10D8700008460A461BD001250095884A28462946B5
:10D8800001F014FFF4E0C3780125032B00D0FAE087
:10D8900006462A02032308E0012583A228462946DA
:10D8A0003B4601F003FFE3E00A46012148020F91E5
:10D8B000592189007518FD214900711802913146DE
:10D8C00062313F05D219641E1F2727405C013C19B5
:10D8D0001443044332795207D20C22432B789B061F
:10D8E0005B0BD218B379DB071B0B13436D4D2B6019
:10D8F000F279032310931A40737A9B079B0E9A18B0
:10D90000B37A5B07DB0D9A18F37ADB079B0DD2180D
:10D91000337BDB075B0DD218737B1B075B0CD218C4
:10D92000AA603269EA6072692A61B2696A61F26961
:10D93000AA61326AEA61726A2A62B26A6A620F98FE
:10D940000870F06AA8623F20C4432C353046E430AA
:10D950000F903046E5300E903046E6300D90304660
:10D96000E7300C903046E8300B903046E9300A90B2
:10D970003046EA3009903046EB3008903046EC30C3
:10D9800007903046ED3006903046EE300590304638
:10D99000EF3004903046F03003903746F137304690
:10D9A000F230F3360F990A194021525C109B1A404D
:10D9B0000E9B1B195B5C9B071B0F9A180D9B1B1979
:10D9C0005B5C9B079B0E9A180C9B1B195B5C9B0175
:10D9D0009A18D2B20B9B1B195B5C9B079B0D9A1884
:10D9E0000A9B1B195B5C9B071B0D9A18099B1B1953
:10D9F0005B5C9B079B0C9A18089B1B195B5C9B0745
:10DA00001B0C9A18079B1B195B5C9B079B0B9A18B6
:10DA1000069B1B195B5C9B071B0B9A18059B1B192C
:10DA20005B5C9B079B0A9A18049B1B195B5C9B071A
:10DA30001B0A9A18039B1B195B5C9B079B099A188E
:10DA40003B195B5C9B071B099A1803195B5C9B07DE
:10DA50009B089A183319595C8907891802C5103434
:10DA6000A0D102980078042101430E48C16300252B
:10DA7000284611B0F0BD04200090084A28462946E7
:10DA800001F014FEF4E703200090044A28462946DA
:10DA900001F00CFEECE7C0462C940102CB330100F0
:10DAA0001134010000100040556E646566696E65B2
:10DAB00064206D65616E205052462025640D0A0079
:10DAC000496E76616C6964206D65616E20505246C6
:10DAD0002025640D0A0000007047704780B50E498C
:10DAE0000E480246083A1268920000D4603142683B
:10DAF0000A4342600A490A6808239A430A60091FD8
:10DB0000012252040A600321890402688A430260E8
:10DB1000FBF72CFA80BDC0462000008028000040A2
:10DB200004020040B0B5032000072D490A68824373
:10DB3000012568071018086000242046FFF7CDFF74
:10DB40002046FFF7C9FFEFF31080284002D1EFF322
:10DB5000108172B68021C943224A53680B4053603A
:10DB600093680B409360D3680B40D36013690B40FC
:10DB7000136153690B405361002800D162B6B0BDF8
:10DB800070B50C4603210907154A13680B4313604F
:10DB90000122EFF31081114002D1EFF3108272B62F
:10DBA0008025EA430F4B5E6816405E609E682E43F8
:10DBB0009E60DD681540DD601D6915401D615D6971
:10DBC00015405D61002900D162B6002802D0012015
:10DBD000FFF783FF002C02D00120FFF77DFF70BD0F
:10DBE00000040040A89501020D4A002907D0012930
:10DBF0000BD10121814010688843106007E00121AA
:10DC0000814010680843106001E001218140101F2D
:10DC100002680A430121C907114301607047C046E9
:10DC200044000040032804D840000649085A00B2C6
:10DC30007047002000B27047032802D84000014A14
:10DC4000115270474AD001029E4908707047C04681
:10DC500070B58AB00C460546FF20FC30A8490E6816
:10DC6000315C59208000335CB278307808AE06967B
:10DC700009AE05960C4E04962126760603960B4EA9
:10DC80000296012601960E2600965B1CDBB2F7F782
:10DC90007FFE0998F2F730FE28700898F2F72CFE04
:10DCA00020700AB070BDC04600002041000004434F
:10DCB000F0B58BB00446457C824800788249002844
:10DCC00022D000200880814A1080814B01269E7658
:10DCD0001E830A907F4800787F4E36786DB2059596
:10DCE0007E4D04957E4D03950AAD02957D4D0195BF
:10DCF0000096F7F78BFB0A9D112020567A497B4A44
:10DD000000F0E0FB064626E000260E806F4A1680F3
:10DD10006F4B01209876188309966E4800786E4FF5
:10DD20003F786DB205956D4D04956D4D039509AD28
:10DD300002956C4D01950097F7F768FB099D11203E
:10DD400021567F20C005009001900296664A674BDD
:10DD50003046F8F7AFFC432001062846F2F72EFBC9
:10DD6000F2F7CAFD089062480078002824D05120BC
:10DD7000800060494A7D42438D185F480068A8646E
:10DD80002F46403750480078B87450480078F874EF
:10DD900055480078387555480078787557480078A8
:10DDA000F87550480069F2F7A7FDB8755248406908
:10DDB000E8644C4800686864FF20FE3050490968F8
:10DDC000085C3922D2008918022812D303D04E48A9
:10DDD000007801280DD14B480660434800883A4A34
:10DDE000108042480088394A108009200790089620
:10DDF00005E04448089A02603548C08B07900B78CC
:10DE00000022002B01D0114600E0D1430125002B58
:10DE100001D0042300E0EB43A67AAD1BEE175B199B
:10DE200071416568AE0F277AAD00ED195641677AEA
:10DE30003F1FF817ED1970414000EE0F80196D007B
:10DE4000EB1848418001990E4118980127239B0245
:10DE5000C31A91411D4805881B480088854201D09E
:10DE60000798421B10202056C001194D2D8C032D00
:10DE700007D1E468E5176D0A6419E4150519EC1774
:10DE80000FE0E468E5176D0A6519EC17ED15C61784
:10DE90004519744197B2002F00D03446002F00D0AE
:10DEA0000546581BA141130409D012B2D2015242B7
:10DEB000D31780185941089BDA17C01A91410BB04B
:10DEC000F0BDC046AE9301021CAB01021AAB0102C9
:10DED00084940102AD900102AC90010208A10102FC
:10DEE000049F010220AB01026AAB010268AB010290
:10DEF000D4A401020CA201026420004018AB01026C
:10DF00002C94010214AB010278AB0102C10D400256
:10DF1000803070470120C0071B4908607047C04629
:10DF200010B519480068C10710D1810711D4410705
:10DF300012D4010713D4C10614D4810615D44106A6
:10DF400016D48021084016D031A215E001240FA27A
:10DF500013E0022411A210E0032414A20DE0042413
:10DF600016A20AE0052419A207E006241CA204E078
:10DF7000072421A201E0254A04090220032101F01F
:10DF800095FB204610BDC0465C000040526573659D
:10DF90007420627920504F520D0A0000526573655B
:10DFA0007420627920424F520D0A00005265736559
:10DFB000742062792050494E0D0A00005265736545
:10DFC00074206279205744540D0A0000526573652D
:10DFD00074206279204C4F434B55500D0A000000CD
:10DFE0005265736574206279205357205265626FC1
:10DFF0006F740D0A00000000526573657420627929
:10E00000205359535245510D0A0000007626010055
:10E01000526573657420627920445644440D0A00A9
:10E0200001218140044A1F2802D0106888431060F3
:10E0300010680843106070471C000040F0B583B0C2
:10E04000029104469949F2F745F80546984901942A
:10E050002046F2F73FF897494618974971430095D3
:10E060006F189649441864212046F2F733F838189F
:10E07000A108471A92492046F2F742F83818914908
:10E080004518914F05D464213046F2F723F80C4629
:10E0900014E0A6B264213046F2F71CF8B720400025
:10E0A000A20701D1002907D1884B73430422D34131
:10E0B000874A934200D3401E0C46451900984743B7
:10E0C00002980680192001013046F2F703F82A462B
:10E0D0001F3A284600DB1046019BFF18B30705D105
:10E0E000002C03D01F2D05DA0120C5E01F2D0BDA0F
:10E0F0000120C1E005461D3D034600DB2B461C28E0
:10E1000008DC02201546B7E000290CD01C21451A76
:10E110000CD50CE019461F39184600DB08461F2BAA
:10E120001DDA0320A8E01D21451A00D42846002D41
:10E1300008D401461F39024600DB0A461F2804DACC
:10E14000032099E00220154696E015461E3D104634
:10E1500000DB28461E2A0CDA04200D468CE005461A
:10E160001E3D024600DB2A461E280BDA04200D461F
:10E1700082E001461F39024600DB0A461F280ADA00
:10E18000052079E011461F39104600DB08461F2A9A
:10E190000BDA052070E015461E3D104600DB2846D0
:10E1A0001E2A0CDA06200D4666E005461E3D024694
:10E1B00000DB2A461E280BDA06200D465CE00146ED
:10E1C0001F39024600DB0A461F280ADA072053E0FF
:10E1D00011461F39104600DB08461F2A0BDA0720BC
:10E1E0004AE015461F3D134600DB2B461F2A0CDA7A
:10E1F00008200D4640E005461F3D024600DB2A464A
:10E200001F280BDA08200D4636E019461E3918463D
:10E2100000DB08461E2B0ADA09202DE011461E39C4
:10E22000104600DB08461E2A0BDA092024E01F28CE
:10E23000054601DB05461F3D1F280CDA0A200D4666
:10E240001AE01F28054601DB05461F3D1F2806DA98
:10E250000A200D4610E01E2D05DB0C2004E01E2DCB
:10E2600006DB0C2005E00B201E2D05DB1E3D03E028
:10E270000B201E2D00DB1E3D029EB070681CF0704E
:10E28000E12001013846F1F725FF3071C0B2114994
:10E290004143CC193C212046F1F71CFF70713B2112
:10E2A000C94341430819B07103B0F0BD805101006A
:10E2B0008033E101B207000093FEFFFFB1070000C9
:10E2C00070FEFFFFA7FA0A0080AEFEFF295C8FC236
:10E2D0000BD7A300F0F1FFFFF0B581B00446FFF7C4
:10E2E00021FCA08A00280ED0FFF71EFA22490861FF
:10E2F00022482CCC2CC02CCC2CC02CCC2CC00020E8
:10E30000888101B0F0BDE08A1B4FB881A169BA894C
:10E310001B48F1F709FF194D204629464CC84CC14E
:10E320004CC84CC14CC84CC1FFF7FEF938616E684F
:10E33000FFF790F9301AB8622846FFF7B9FC064695
:10E340000D461048007BFFF76DFC0121F9700E4966
:10E3500000220A70617C3971396C491C396481B2C0
:10E36000C90B401800B2C1174010301A38658D41F2
:10E370007D6501B0F0BDC046389601025498010297
:10E3800054D00102AE90010252D00102F0B581B02A
:10E39000EFF3108072B600200146FBF7C7FE04467B
:10E3A000002803D062B6204601B0F0BD01273A0331
:10E3B0000025074E28463146FBF712FEBB02164ADF
:10E3C00028463146FCF7EAFA62B6204601B0F0BDB5
:10E3D00000E0020480B5F6F7DEF8F9F719FAF8F76D
:10E3E00029FA0C490120C8720A7B03469343CB717A
:10E3F000521C0A73084A928F002A08D08A7A4B78F6
:10E40000134304D04A7A501C4872012090430349B8
:10E41000087080BDA097010212A7010215940102A5
:10E4200070B514460D4606461120FAF71DFF224826
:10E43000042101600C4804601E4805608660002EBF
:10E440000DD0FF20000609490A6882430120C00759
:10E4500010180860064808210160064801601A206B
:10E460000221FFF7C1FB70BD54D1010200E400E0BE
:10E4700080E200E000E100E00C4908607047C0461F
:10E4800010B504460948006860430949F1F738FEB1
:10E4900000190849486008480022026002460C3A08
:10E4A0004B6813600968016010BDC04650D101027D
:10E4B00040420F000C9001022C1001400048004720
:10E4C000C100000080B582B013460A4600900348A0
:10E4D000011D0348F8F79AF802B080BD90D10102FF
:10E4E0003C9E010210B50C498A1C90420DD2401E80
:10E4F0000D4A50600D4803680B4003218C071B191F
:10E50000036000209060116010BD04480449E622B9
:10E51000044B00F06FF8C046FFFFFF004D260100DE
:10E52000672601003326010010E000E020ED00E046
:10E53000B0B50120EFF31081014002D1EFF310825A
:10E5400072B6124A1368124C226864688506114834
:10E5500000682840850E5D192923DB006B43002CE1
:10E560001D4606D1002809D11E20684300290AD083
:10E57000B0BD121BD218551C0028F5D01D461E2018
:10E5800068430029F4D162B6B0BDC046C0DC0102C8
:10E5900014E000E004ED00E080B50020FBF770F827
:10E5A000404280BDB0B586B0104869460A4638C8BA
:10E5B00038C238C838C200242046FBF767F80399F0
:10E5C0002046FBF7FDF80198012803D00824002815
:10E5D00004D102E00424002800D104460220FAF706
:10E5E0004BFEE0400249086006B0B0BDF8160100DD
:10E5F000D4DC010290B01C4605AB07C3EFF31080DA
:10E60000C00702D1EFF3108072B6EFF310800B90C9
:10E6100068460E907046089010AB0F93CF4F3E1D8A
:10E6200001200490C50230462946224600F0B8FC7D
:10E6300000213154EFF303800990EFF308800C9030
:10E64000EFF309800D90EFF314800A9000F02CFC9A
:10E650003868012833D80028C14F00D0C14F2A2084
:10E66000C1497A69920703D50A783A60401E491C6D
:10E670000028F6D1B948041D2046F1F783FD002893
:10E6800007D079698907FAD521783960401E641C62
:10E69000F5E70220B5497A69920703D50A783A600E
:10E6A000401E491C0028F6D12A20AF497A699207FA
:10E6B00003D50A783A60401E491C0028F6D1FFF7BE
:10E6C00037FF0346AA4A30462946FDF711FF0446A4
:10E6D0003018291B089F3B1F049A9343A5A2FDF7FE
:10E6E00007FF9E490968012966D8001900299C4C3A
:10E6F00000D09C4C00280AD09849091D62699207F5
:10E7000003D50A782260401E491C0028F6D10A2051
:10E710009F496269920703D50A782260401E491C0E
:10E720000028F6D10598F1F72DFD002809D0616980
:10E730008907FAD5059A11782160401E521C05926E
:10E74000F3E7022089496269920703D50A782260BB
:10E75000401E491C0028F6D10A208EA1626992074A
:10E7600003D50A782260401E491C0028F6D106987D
:10E77000F1F708FD002809D061698907FAD5069AE2
:10E7800011782160401E521C0692F3E7022077495F
:10E790006269920703D50A782260401E491C00284E
:10E7A000F6D10A207EA16269920703D50A78226019
:10E7B000401E491C0028F6D17CA230462946079B02
:10E7C000FDF796FE6549096801290E9B1BD80029B3
:10E7D000634900D0634900280AD0604A121D4C6981
:10E7E000A40703D514780C60401E521C0028F6D1F3
:10E7F00002205E4A4C69A40703D514780C60401EC1
:10E80000521C0028F6D16AA230462946FDF770FE58
:10E8100004463018291B694A3B46FDF769FE4F49FB
:10E820000968012911D8001900294D4900D04D4926
:10E8300000280AD0494A121D4B699B0703D513785B
:10E840000B60401E521C0028F6D15D4A3046294616
:10E85000099F3B46FDF74CFE0446F800C00FB90087
:10E86000C90F7A00D20F0092019102903019291B32
:10E87000FB0F544AFDF73CFE04193019291B3F23B6
:10E880003B40514AFDF734FE34490968012911D84B
:10E8900020180029324900D0324900280AD02F4AD6
:10E8A000121D4B699B0703D513780B60401E521C49
:10E8B0000028F6D1454A304629460B9BFDF718FE45
:10E8C00004463018291B424A0A9BFDF711FE2349D2
:10E8D0000968012911D800190029214900D02149CE
:10E8E00000280AD01D4A121D4B699B0703D51378D7
:10E8F0000B60401E521C0028F6D1364A304629468D
:10E900000C9BFDF7F5FD04463018291B324A0D9B80
:10E91000FDF7EEFD114909680129114A0DD80019CA
:10E92000002908D00F4A06E05169890703D53178DC
:10E930001160401E761C0028F6D128490E98091A4D
:10E94000A94200D32946890800F03AFE244800680D
:10E95000002800D0804700F045F8C046DCDC01020A
:10E960000090014000A00140A726010035340100BD
:10E97000902601000D0A232323204153534552546E
:10E98000204020307825303858202323230D0A00DA
:10E990006A27010046554E4354494F4E3A20000025
:10E9A0004C494E45202020203A20000025640000DC
:10E9B0000D0A53503D253038580D0A002F2701000D
:10E9C000452701005127010039270100EE260100EB
:10E9D000FD2601000C2701001727010000F80202A4
:10E9E000D8DC0102F7480068012811D8002801D0BE
:10E9F0000B4800E0FC480C210A4A01E0002907D03E
:10EA000043699B07FAD513780360491E521CF5E74A
:10EA10001E20FFF705FB00BF00BF00BF00BFFAE7E5
:10EA200000A001409A2601008AB00646E448B0667C
:10EA300000F03AFAFFF77CFD0346E248041D01208E
:10EA40000590C502E04A20462946FDF751FD0746DC
:10EA500008942018DB4C0995E91BF36C3F220692C1
:10EA60001340DAA2FDF744FD2168012910D8C0192E
:10EA70000029DD4900D0DD49002809D0221D4B695D
:10EA80009B0703D513780B60401E521C0028F6D15B
:10EA9000F36BD7A2089C2046099D2946FDF728FD67
:10EAA0000746291A2018336C069A134007D1D8A2BA
:10EAB000FDF71EFDC34C2168012907D917E0CEA23E
:10EAC000FDF716FDBF4C2168012910D8C019002997
:10EAD000C54900D0C549002809D0221D4B699B07B4
:10EAE00003D513780B60401E521C0028F6D1002776
:10EAF000CBA5B80030580090089809992A463B46A3
:10EB0000FDF7F6FC216801290FD80029B64900D08D
:10EB1000B649002809D0221D4B699B0703D51378FD
:10EB20000B60401E521C0028F6D17F1C0D2FE0D137
:10EB3000736BBFA2089C2046099D2946FDF7D8FCAF
:10EB4000074620189F4CE91BB36BBC4AFDF7D0FC6D
:10EB50002168012910D8C0190029A34900D0A34970
:10EB6000002809D0221D4B699B0703D513780B6041
:10EB7000401E521C0028F6D1336CB14A089C204636
:10EB8000099D2946FDF7B4FC0746326CD000C00F42
:10EB90009100C90F5300DB0F009301910290E0191F
:10EBA000E91BD30FA74AFDF7A3FC3246C619A019EB
:10EBB000A91B1546136C069A1340A34AFDF798FC4F
:10EBC00080490968012911D880190029864900D097
:10EBD000864900280AD07B4A121D4B699B0703D542
:10EBE00013780B60401E521C0028F6D12E466B6C29
:10EBF000964A089C2046099D2946FDF779FC074660
:10EC00002018E91B0796B36C914AFDF771FC6D4A19
:10EC10001168012910D8C0190029734900D073491F
:10EC2000002809D0121D4B699B0703D513780B6090
:10EC3000401E521C0028F6D10798426E0423602122
:10EC40005C2004931A400B4600D003460693002A2A
:10EC500000D00846079E33587E4A089C2046099DEE
:10EC60002946FDF745FC074606983358E019E91B8D
:10EC7000794AFDF73DFCC619A019A91B079A536EE6
:10EC800076A2FDF735FC4F490968022911D2801997
:10EC90000029554900D0554900280AD0494A121D7B
:10ECA0004B699B0703D513780B60401E521C00284C
:10ECB000F6D10798C36C06466DA2089C2046099DB4
:10ECC0002946FDF715FC07462018E91B336D6B4AF2
:10ECD000FDF70EFCC619A019A91B079F7B6D68A242
:10ECE000FDF706FC8619A019A91BBB6D67A2FDF7ED
:10ECF000FFFB344909680129059C11D880190029B6
:10ED0000394900D0394900280AD02E4A121D4B69D2
:10ED10009B0703D513780B60401E521C0028F6D1C8
:10ED20000798476B5D4A974237D2032087430026F6
:10ED3000059CB00039580246049B1A43BA58082370
:10ED40000343FB580C2505437D5900910192029322
:10ED500003953B1808980999514AFDF7C9FB1949D1
:10ED6000096801290FD800291F4900D01F49002830
:10ED700009D0089A4B699B0703D513780B60401E96
:10ED8000521C0028F6D11B2E444A06D80798406B27
:10ED9000361DB10040189042CBD30798406B111A32
:10EDA000099A914201D8890800E0610200F008FC4C
:10EDB0003C480068002800D08047FFF713FEC0469B
:10EDC00022224B4DDCDC0102902601000D0A0D0AC7
:10EDD00023232320455843455054494F4E20256452
:10EDE000202323230D0A00000090014000A00140D1
:10EDF00050433D25303858002C20457863657074A9
:10EE0000696F6E4E756D6265723D25640D0A000076
:10EE10002C205468726561644D6F64650D0A0000B2
:10EE200052252D32643D253038580D0A000000006F
:10EE300053503D253038580D0A0000002F2701009F
:10EE4000452701005127010039270100EE26010066
:10EE5000FD2601000C270100172701004558435FDC
:10EE600052455455524E3D253038580D0A00000089
:10EE7000494353523D253038580D0A0022270100DE
:10EE80005343523D253038580D0A00004343523D4C
:10EE9000253038580D0A0D0A0000000000F8020263
:10EEA000D2260100D8DC0102F0B583B0344D2C68C5
:10EEB000012C06D8601E8441204601F057FB002833
:10EEC000FAD10120EFF310810140019102D1EFF35B
:10EED000108072B62B48285A2B49695A814245D076
:10EEE0002A68002A01D02A4E00E0284E1F23DB02A8
:10EEF0000293284C022A27D205E01046214AA85244
:10EF000082B2914232D087B2B9420A4600D8621C1E
:10EF1000131A21482B5218040DD0E819001D9FB276
:10EF200001E0002F07D073699B07FAD5037833609F
:10EF30007F1E401CF5E7A242DFD902981018DDE7DA
:10EF4000304683B299420CD0024680B281420E46CE
:10EF500000D8661CA642F3D90298301883B29942B1
:10EF6000F2D108496852B01A0B4968520B48002187
:10EF700029540198002800D162B603B0F0BDC04604
:10EF8000DCDC01020A0800000808000000900140D3
:10EF900000A00140FF0700000C0800000F0800005F
:10EFA000F0B58DB00793174600240C9409AA13C23C
:10EFB00015E006986849F1F701FAF1F79DFCC117D1
:10EFC000401848406549F1F785F8009509A80622E0
:10EFD0003346F9F731FBBDE0002C00D5BEE13878AF
:10EFE0007F1C25280DD0002800D1B7E10B9A511CB9
:10EFF0000A9B9942F0D8099B9854641C0C940B917D
:10F00000EAE708940025397823390D2914D801201E
:10F010007944097949008F44090F0F0F0F0F0F0F23
:10F020000B0F060F0F0D05437F1CECE70820FAE7D6
:10F030000420F8E70220F6E738780146303900244A
:10F04000092902D9264639460BE000260A217143D8
:10F050000E18303E791C78780246303A0A2A0F465C
:10F06000F4D32E2817D14A1C487801463039092993
:10F0700005D911464F1C2538532811D96AE00024C0
:10F080000A2161430C18303C511C50780246303A3A
:10F090000A2A0A46F4D34F1C2538532800D959E0D0
:10F0A0004000C0467844808840008744A000530058
:10F0B00053005300530053005300530053005300B8
:10F0C00053005300530053005300530053005300A8
:10F0D0005300530053005300530053005300530098
:10F0E000530053005300530053005300530060007B
:10F0F0005300530053005300530053005300530078
:10F100005300530053005300530053005300530067
:10F110005300980053005300530053005300530012
:10F120005300530053005300AD00B600530060007D
:10F13000530059005300530053005900530053002B
:10F140005300DE0053005300BD005300D3005300B2
:10F15000530098000C9C3FE70024744940420F0084
:10F16000791C38780F4625385328F3D898E7079943
:10F17000C91D07208143086807914968F1F722FCFF
:10F1800000210690F1F744FB00280BD10B99481C95
:10F190000A9A904206D8099A2D2353540899491C7B
:10F1A0000C910B900798083007900698F1F7A4FB94
:10F1B0000095C2178118514009A822463346F9F735
:10F1C0003BFA0B98411C0A9A914200D9F1E6099A40
:10F1D0002E2313540B910C98401C0C90E9E60798D1
:10F1E00002C807900096019509A8102239E00B98F3
:10F1F000411C0A9A9142ADD8099A252313540B91C8
:10F200000C98401C0C90A5E70B9A511C079C201DE4
:10F210000A9B994239D907909CE7079802C8079042
:10F22000009509A82246D3E6079901C907910999D3
:10F230000A9A089E02E0401C002E8BD40378002B13
:10F2400088D00B9D6C1C9442F5D84B55761C0C96BF
:10F250000B94F0E7079802C807900096019509A85B
:10F260000A222346F9F786FA74E7079B10CB102C85
:10F27000079308D300202146401C0A09FF291146A4
:10F28000FAD806280AD8082009E02368099CA35464
:10F29000089A521C0C920B9107905BE7401C069059
:10F2A00009230C980B9D099905910A9E04940DE081
:10F2B000202104463046059E715506462046049C92
:10F2C000401C15460146089100290AD45B1E069988
:10F2D000994206D26A1CB242EAD9089908910029DB
:10F2E000F4D50C900B950898002800D532E701263C
:10F2F000082501E06D1E3601022DFBD22046314665
:10F30000F0F7E8FE0F28F6D80C98059009980390BE
:10F310000A9806900B9D20463146F0F7DBFE691CEB
:10F32000069A914204D90899089100290CD511E058
:10F330000C4A125C039B5A55089A521C0D460592C2
:10F3400011460891002905D47043241A3009102E63
:10F350000646E0D205980C900B95FBE620460DB0D2
:10F36000F0BDC046EC19010070B588B0002203283A
:10F3700003D9D243104608B070BD7F4CC34D2A510B
:10F380000F4B104EEE5081231E010123AB55286018
:10F390002C1962600128EDD807930022069205928D
:10F3A000049203230393029201920091411E88412B
:10F3B000694600F00BFD0246104608B070BDC0461D
:10F3C00004080000FFC0FFC0F0B583B00C46002366
:10F3D000D943012C56DB074602910126EFF3108535
:10F3E000354002D1EFF3108072B65849584A505C4C
:10F3F000002800D0A3E056545E48115A5E48105AC7
:10F400000196F202161A814240D832465218A242A0
:10F4100040DB00930295A642354600DB25464C4969
:10F420000818001D39462A46F0F77EFEA642484ECF
:10F4300004DA7919621B301DF0F776FE4E48305A17
:10F44000001981B24D4A914201D94D494018029D9F
:10F45000009B4949705230464A4E805D002865D174
:10F46000EFF310850198054002D1EFF3108072B6DA
:10F47000374A4048115A4048105A884232D14248CF
:10F4800013524FE00C46204603B0F0BD42425218E2
:10F49000A242BEDA3B4A2E4EB25C002A0CD03A4A57
:10F4A000B25A51188AB2354CA242284C029F01D957
:10F4B000334A8918304A02E0244C2F4A029F3355C0
:10F4C000B152421A89B2884202D22C488018421C9A
:10F4D00093B22F4801212FA200F0E8F83C46002DFE
:10F4E000D1D128E0019F9755884201D82348401C7C
:10F4F000421A90B2800A01D0019882022248144F29
:10F500003A52386801280DD8431E9841104B5918BB
:10F51000091D92B21D4B00F06FFE009B002801D028
:10F520000B488355002D029D00D162B6074808495B
:10F530000B54002DA7D162B6204603B0F0BD2120A8
:10F540000201044804A108A3FFF754F80E080000C4
:10F55000DCDC0102E627010074726163655F6F7590
:10F5600074707574000000005452414345204255A8
:10F57000535900000A08000008080000FF070000B7
:10F5800000F8FFFF0F0800000C080000D9F700008A
:10F5900002FF00000D0A54726163652062756666A1
:10F5A00065722069732066756C6C2C2064697363C6
:10F5B000617264732025752062797465730D0A0089
:10F5C000F0B587B005460026069605960496039684
:10F5D0000296800701D007B0F0BD019102A8142166
:10F5E00026A2FCF785FF29490968012911D80029BD
:10F5F000274900D0274900280BD002AA01E00028A3
:10F6000007D04B699B07FAD513780B60401E521C3C
:10F61000F5E701990029DED0204C3746B8002B5879
:10F62000D80724D0581EA04204D31B4818181C4ADF
:10F6300090421CD802A814211AA2FCF759FF1349C2
:10F640000968012911D80029114900D01149002861
:10F650000BD002AA01E0002807D04B699B07FAD51E
:10F6600013780B60401E521CF5E7761C01997F1C35
:10F670008F42B0D2322ED1D3ADE7C0460D0A4261DF
:10F68000636B74726163653A200D0A00DCDC010271
:10F690000090014000A00140FFFFFFFCFFFF0200BF
:10F6A000FEFF0100253038580D0A000081B0F0B58A
:10F6B000C4B00E4607464993812000012F49085CDB
:10F6C000002845D002920120050204A82946F0F73F
:10F6D00044FDFCB20021C8430C2C3AD8721E032A08
:10F6E00037D82748005DB042084632D3F80535D5F3
:10F6F0000021B8050DD404A801904018691AA20091
:10F7000022A39B582E4AFCF7F3FE0198F0F73AFD2E
:10F71000014678050ED404AF7818691AB20029A3FF
:10F72000D218121F1368264AFCF7E2FE3846F0F79B
:10F7300029FD0146029A04AE70180C46691A49ABBD
:10F740000393FFF72DFC01193046FFF73DFE00E063
:10F75000002044B0F0BC02BC01B00847FEF7E8FE50
:10F76000034604A8019007A22946FCF7C1FE0198B0
:10F77000F0F708FD0146B805BDD5CAE7DCDC01029B
:10F780001840010025313075207C20008A270100B7
:10F79000E0270100DA270100B927010084270100D2
:10F7A000A5270100D3270100CC270100C7270100AE
:10F7B0007D27010090270100A02701007527010087
:10F7C00099300100BF270100AB270100B2270100DB
:10F7D0009627010000000000F0B581B00B46012023
:10F7E000EFF31084044002D1EFF3108172B6990F49
:10F7F00007D0022001212DA2FFF758FF002C3DD198
:10F8000041E02249224D00276F54224AAB5A224A36
:10F81000AE5AF3189EB2F60A01D0204E9B19AB5295
:10F82000EFF31086064002D1EFF3108372B6AA5AA6
:10F830001C4BEB5A934202D116482F521AE06854DF
:10F84000934201D8164B5B1C9B1A99B2890A00D0CF
:10F85000830210482B52286801280BD8411E88418A
:10F86000A918091D9AB2104B00F0C6FC002801D05F
:10F8700006482F54002E03D0002C04D001B0F0BD58
:10F8800062B6002CFAD162B601B0F0BD0F080000DC
:10F89000DCDC01020C0800000A08000000F8FFFF91
:10F8A000FF07000008080000D9F700005541525436
:10F8B000204572726F722025780D0A0010B504463B
:10F8C000FEF730F9A08A002800D010BDFDF72CFF0C
:10F8D000034908620861486C401C486410BDC0467A
:10F8E00038960102B0B50A2000242146FBF730FD0E
:10F8F00009202146FBF72CFD0124204600F03CF8AE
:10F900000E2004252946FBF723FD0D202946FBF791
:10F910001FFD0549204600F059FAA2021449154B73
:10F92000204600F027FBB0BDC8940102B0B50E2000
:10F9300000242146FBF70CFD0D202146FBF708FDB6
:10F940000124204600F018F80A2004252946FBF778
:10F95000FFFC09202946FBF7FBFC2046F9F7D2FA09
:10F96000A2020349034B204600F004FBB0BDC04691
:10F97000C0CB0102AD01010070B5012801D9012001
:10F9800070BD48224243734B9C58A5691F218D438B
:10F99000A5610625A5600F2525629C18A27C002A7A
:10F9A00005D1627C002A02D1227C002A14D063682F
:10F9B000002B11D4251D0B40012216469E400C4BF6
:10F9C0001E60BFF34F8FBFF36F8F2B68002B03D4E4
:10F9D0000B409A4007490A60002803D0012804D14F
:10F9E000092000E00820F9F737FC0020A06170BD75
:10F9F00080E100E080E200E0F0B585B00D460278DD
:10FA0000E348C368934219D0446D944216D083688A
:10FA1000934203D0016D914200D07FE09B1A591EA2
:10FA20008B41049348215943032D46D14418E16981
:10FA300000294ED01C34002020606DE09B1A5A1E15
:10FA400093410493032D1AD1039548225A438418F5
:10FA5000A26B0121EFF310850D4002D1EFF3108767
:10FA600072B6A7691026B743A761A669002E01D117
:10FA700018342160002D00D162B6039D0CE04821AE
:10FA80005943421891691832302902D0116810295F
:10FA90004CD1802111600022482159434018002197
:10FAA000816301628162243000210160002A33D029
:10FAB00004A82946904705B0F0BD42189169183254
:10FAC000302902D01168202939D18021116000220B
:10FAD00016E00395E26B0126EFF31085354002D165
:10FAE000EFF3108172B6A1692027B943A161A16922
:10FAF000002901D118342660002D00D162B6039D83
:10FB00004821594340180021C163C162416330302C
:10FB100000210160002ACBD105B0F0BD00920E4A51
:10FB20002E329C480D490E4BFEF764FD1068009381
:10FB3000019098480949084A0A4BFEF75BFD106896
:10FB400000930190044A243292480449054BFEF781
:10FB500051FDC046E8940102B10200006228010094
:10FB6000372801001B280100F0B585B0049048211A
:10FB70000A464243864B9C58E6690F2535409A1841
:10FB8000167C002E31D04F2040026169014200D125
:10FB900085E0A06904218843A06102202062012041
:10FBA00081076918D161D36BEFF31084044002D14F
:10FBB000EFF3108572B695692026B5439561956976
:10FBC000002D00D173E010463C30002C00D162B60D
:10FBD00000240460D4625463303200201060002B93
:10FBE00063D004A8984705B0F0BD0C2D5DD8C04681
:10FBF0007D442D796D00AF4467586B580658A1635A
:10FC00005858585806009569202D04D015461835C7
:10FC10002D68302D49D1156B566B3432AE4217D258
:10FC20006669360714D5646815686E1C166048430B
:10FC30001818C06A445504980C4644431A19156BA9
:10FC4000566B3432AE4203D21C5966693607EAD489
:10FC50001268AA4229D14143585882690524A24317
:10FC600082615A18D36B0121EFF31080084002D152
:10FC7000EFF3108472B694692025AC4394619469C3
:10FC8000002C02D114461834216014463C3400285C
:10FC900000D162B600212160D16251639CE70C2D36
:10FCA00000D176E7012D00D173E705B0F0BD154610
:10FCB0001835286010463C30002C00D187E787E7D4
:10FCC0000420206205B0F0BD0120206205B0F0BD27
:10FCD00008252562164618369569102D02D035681C
:10FCE000302D4BD10396566A15462835976AB74290
:10FCF00028D1A06902218843A061936B0121EFF311
:10FD00001080084002D1EFF3108472B6039E34686D
:10FD10001027BC4334603468002C00D13160144695
:10FD20003834002800D162B60021216029601162B8
:10FD3000243200201060002BB7D052E7022020624E
:10FD400005B0F0BD2A68B242AFD262699207ACD565
:10FD50002A68561C2E6048431818006A805C206090
:10FD600004980A4642439D18AC6A6E6AB4429CD21B
:10FD700028359C5862699207EAD496E7316800906A
:10FD80000191044804A1094A09A3FEF733FCC046C7
:10FD9000E894010201280100756172745F69727153
:10FDA0005F68616E646C6572000000003D030000D6
:10FDB0005561727420256420737461746520676FC7
:10FDC00065732077726F6E6720256400F0B585B08B
:10FDD0000E460546022804D3002E02D1012005B0AC
:10FDE000F0BD002D03D0012D08D1092400E0082426
:10FDF0002046F9F739FA2046FEF712F948216943FF
:10FE0000E74A505883691F240294A3438361062361
:10FE100083600F230193036257180023BB62BB6307
:10FE2000FB633B627B62FB623B63317F3974727FB1
:10FE30007A74B27FBA7404937B637368B268F468AF
:10FE4000920022435B1E032B0ED8C0467B441B79D5
:10FE50005B009F4401050307082304E0282302E018
:10FE6000182300E038231A43C260C907090F7269DA
:10FE70009201D2B28918B2699207920E8918491C70
:10FE8000816079613169012901D122210161012D4E
:10FE90005CD831680E2959D23846123003900324B9
:10FEA000002D01D0204600E004204C432D490E19BE
:10FEB000B178F9F769FA3968CA688025104628438D
:10FEC000C8602848005D73781B021818C862AA43EE
:10FED000CA60F9F7A1FA03980078002809D13846DA
:10FEE00011300078002804D13846103000780028FE
:10FEF00027D07868002815D4032102468A431B497D
:10FF000053588407E40EFF26A640B343A5401D4383
:10FF100055500299014001208840A24908601449C7
:10FF200008600EE08107C90EFF228A40019C044050
:10FF3000083C032084430C48235893438D401D43C1
:10FF400025500120B861049805B0F0BD024803496E
:10FF5000DA22034BFEF74EFB012801007428010052
:10FF600051280100801701001CED00E000E400E0D2
:10FF700000E100E0F0B58FB00E900125002900D11E
:10FF80004BE0039304910592002A00D145E0012142
:10FF9000EFF3108201910A4002D1EFF3108172B6A3
:10FFA0004827029747437E49CE19B5690023302D73
:10FFB00023D831461831C0467D442D796D00AF44B9
:10FFC00020242626262626262626262626262626D9
:10FFD0005E26262626262626262626262626262689
:10FFE00018262626262626262626262626262626BF
:10FFF00018000223002A0CD00CE0402D01D0802DE7
:020000040001F9
:1000000005D10123002A04D004E020240C60002A3A
:1000100000D162B61D46002B02D028460FB0F0BDBD
:10002000002575630399F1630499F16205993163C1
:100030005B4CE35959691322D202114205D00621C3
:1000400099600F21196271699960317C00290CD087
:10005000F56109950895079506950D950B95022173
:100060000A91012810D017200FE0717C9A690029AD
:100070002CD0952002439A6128460FB0F0BD302461
:100080000C60002AC5D0C5E71920049F0C90706849
:10009000002805D41F210840019981404148016092
:1000A00014209861B06806A9F9F726FA0E9802990B
:1000B00041436018806861583B4A0092091D3A46E6
:1000C000059BF9F789FA28460FB0F0BD34361106C2
:1000D00002D580218A439A6131680025059A9142B0
:1000E0002DD205955D694F214A0215421BD1E905C4
:1000F00002D4029CF24F0AE0596833685C1C3460F9
:10010000029C6043EE4F3818C06AC1540E982146D5
:1001100041437E18736B346BA34238D234367B581C
:100120005D691542E3D002211962019EB10729439E
:100130003546E34CEFF31082324006D008E0294602
:10014000019EEFF31082324002D1EFF3108372B6BA
:10015000029B4343E01883692024A343836183699E
:10016000002B05D0002A08D0C26B002A0AD154E720
:10017000034618331E60002AF6D162B6C26B002A0D
:1001800000D14AE70EA8904728460FB0F0BD294697
:10019000059D019E3C46EFF310823240D5D0D7E753
:1001A000E894010280E200E0F9F9000080B5012046
:1001B00082020249024BFFF7DDFE80BDC0CB010287
:1001C000AD010100B0B582B079208400E54D285D15
:1001D00001A90870652080002818F3F7B1FA2F20D4
:1001E000C000285829190122024BFFF7C3FE02B0B4
:1001F000B0BDC046C5010100F0B591B01090012618
:10020000002900D19BE003930591002A00D196E0DC
:1002100007900121EFF310800291084002D1EFF323
:10022000108172B604924823069307994B43D6492E
:10023000C9188D690026302D6ED80C461834AD00D3
:10024000374602A675593E46AF46C0462103010017
:10025000290301002D0301002D0301002D030100DE
:100260002D0301002D0301002D0301002D030100CA
:100270002D0301002D0301002D0301002D030100BA
:100280002D0301002D0301002D03010011030100C6
:100290002D0301002D0301002D0301002D0301009A
:1002A0002D0301002D0301002D0301002D0301008A
:1002B0002D0301002D0301002D0301002D0301007A
:1002C0002D0301002D0301002D030100BF030100D8
:1002D0002D0301002D0301002D0301002D0301005A
:1002E0002D0301002D0301002D0301002D0301004A
:1002F0002D0301002D0301002D0301002D0301003A
:100300002D0301002D0301002D0301001103010045
:10031000022600280CD00CE0402D01D0802D05D104
:100320000126002804D004E010252560002800D113
:1003300062B6002E069D944F049C079802D030466A
:1003400011B0F0BD00268E62039A8A63059A0A6294
:100350004C620A7C002A0BD00C960B960A960996E2
:1003600008960E9602220D9201282DD018202CE01E
:100370008A7C2831002A3BD00A68A24216D22B463A
:100380004343FA585469A40710D50868441C0C600C
:10039000F918096A085C10601098294641437A18D8
:1003A00011462831936A526A9342E8D345437859FB
:1003B000816982220A438261304611B0F0BD302546
:1003C00025600028B4D0B4E71A200F90C86808A9A7
:1003D000F9F792F8109845437A597819C068394965
:1003E000009105992346F9F7F7F8304611B0F0BDB2
:1003F000FB589A69140602D58024A2439A610A68C0
:100400000026049882422ED25D694F225202154284
:1004100007980AD002211962029EB10729431FE002
:1004200028315D6915423E46F4D137465C69A40720
:1004300002D40699544E0AE00C68661C0E600699B8
:100440004843514E3018006A005D186010984143CF
:10045000735871188C6A4E6AB442E1D329463E46FD
:10046000069D494F01E0314607985A6A002AFCD19F
:10047000EFF31082029B1A4002D1EFF3108372B6A1
:100480004543781983691024A34383618369002B52
:1004900005D0002A09D0826B002A0BD14FE7034612
:1004A0001833029C1C60002AF5D162B6826B002AC8
:1004B00000D144E710A89047304611B0F0BDC046C7
:1004C000E8940102F9F90000B0B5264900684A68CD
:1004D000824202D10D1D002016E080228A588242FD
:1004E00003D10D46803501200EE0FC228A5882425D
:1004F00003D10D46FC35022006E02F22D2008B5896
:1005000083422ED18D1803207C2242438C18A06890
:10051000012814D0002824D140342046F3F7FFFCF2
:1005200001462046F3F7D1FC2046F3F7F8FC0028FB
:1005300017D006C828680C4BFFF75EFEB0BD4034EC
:100540002046F3F7ECFC01462046F3F7BEFC2046BC
:10055000F3F7E5FC002804D006C82868024BFFF733
:100560004BFEB0BD38BC0102C90401004821414323
:10057000054842189269D20601D4002070474058BD
:100580004169012008407047E894010280B5114894
:100590000078C00110490978890101430F480078AB
:1005A000400108430E490978090101430D480078CC
:1005B000C00008430C490978890001430B480078C2
:1005C000400008430A4909780143C8B2F3F758FFCD
:1005D00080BDC046889D0102369601021594010235
:1005E000F0E4010279AB0102899D010204A101023C
:1005F00005A10102F0B587B00146012702250528B3
:100600003A4600D02A4600200929014600D011466A
:10061000C900374A54180E210591615EFDF70CFBA5
:100620001026A15F3846FDF707FB1227E15F284639
:10063000FDF702FB06951425615F03200490FDF78A
:10064000FBFA0598235EA05FE15F625F00AD07C51E
:1006500028A2069F3846049D2946FFF727F8204622
:10066000263004263146FBF7B9FF2620235E2820DA
:10067000205E2A21615E2C22A25E009001910292EE
:1006800024A238462946FFF711F827463E37384658
:100690003146FBF7C1FF3E20235E06983C5EB95F02
:1006A0000622BA5E00940191029221A207462E46CC
:1006B0002946FEF7FBFF56240D4D285FFBF7A0FFF0
:1006C0002B5F2C4621A2384631463546FEF7EEFF19
:1006D000264658363046FBF77FFF5820235EF05FF2
:1006E00000901FA238462946FEF7E0FF07B0F0BD94
:1006F000A49E0102546F4620616E742064656C6193
:1007000079732025642025642025642025640D0A42
:100710000000000050446F412064656C61797320D3
:1007200025642025642025642025640D0A0000002E
:1007300050446F41206761696E73202564202564F1
:100740002025642025640D0A0000000050446F41FC
:1007500020616E742073706163652025640D0A004A
:1007600050446F4120616E676C65206F66667365EB
:1007700074732025642025640D0A0000F0B587B04D
:1007800015467A4B1A680F24A2432F783A431A6011
:10079000774C23462C3B774A1A6004900346224646
:1007A000283A12681207FAD5734E092F029306D918
:1007B000754A326072600C2F09D175480FE0042F22
:1007C00007D9704A3260704A7260092F06D37148A7
:1007D00005E06A4830607060694800E06B486E4A26
:1007E0001060EB7AFF2B039102D10020B0620AE087
:1007F00003210B406948C05C40220243B2620220E0
:10080000674AFEF753FF029F0021384605952A46A6
:100810000B46FBF75BFF06460225032161A2284633
:1008200001913346FEF742FF06963046FCF722FC64
:1008300001210498009108402CD13D4033D16049FA
:1008400000283AD1002D1ED06548A062E0622063E6
:1008500060636448606264480860152085046E1C0B
:100860008E608D60642420460F46F8F7D5FD3E600B
:100870003D602046F8F7D0FD281D386003215BA2BB
:100880004E48FEF713FF0598007BFBF727F8069804
:1008900007B0F0BD2E4605460698FCF777FF2846C0
:1008A00035463D40CBD02E4605460698FCF7EAFB80
:1008B0002846354642490028C4D04248086142488B
:1008C0004861424888611520C8614148016840225A
:1008D0000A43026007210803274B5A6982430098A4
:1008E0004003101858610522039842432A480368C0
:1008F0009818334E766B47780F40995C0907490E7C
:10090000C919CA03334B33409A18C9015118324AE6
:1009100089182B4A51632A49896B3822914382787E
:100920005207920E891804220A4325498A63124B02
:1009300019690279019E3240C0784007C00E8018C4
:100940001F2291430818186155204003411C216063
:1009500020606420F8F760FD204A18483146039B68
:10096000FEF7A4FE1649002D8DD06DE7040400406B
:100970002C60004000040080000600400F040F04BB
:100980000922010003040304000400043A230100C7
:10099000D82001006B240100309401029C25010045
:1009A000A028010050485920706172616D73207356
:1009B00065747320253038780D0A000002080000A5
:1009C0009060004012A83E009DD79B5AD579BD4942
:1009D000340200403F0080FF4040000082280100B8
:1009E0002008820002D50F00020255007577625F71
:1009F00072785F696E69740D0A00000080B5224844
:100A00000021017022480078C0012049097889013D
:100A1000014320480078400108431F490978C90074
:100A200001431E480078800008431D4909784900A9
:100A300001431C4800780843C0B2F3F721FD80BD94
:100A400080B51148012101701048007880011049DB
:100A50000978C90101430F480078400108430E4955
:100A60000978C90001430D480078800008430C490B
:100A70000978490001430B480078084310210143DD
:100A8000C8B2F3F7FDFC80BDF0E401023696010226
:100A9000889D01021594010279AB0102899D010232
:100AA00004A1010205A10102F0B581B01820FDF7F3
:100AB000B7FA1920FDF7B4FA002420462146F8F7CA
:100AC000ABF820462146FAF78DFE012603257F2349
:100AD000304629462A46FAF797FF3046FBF73CF99D
:100AE00002273846FBF7D2FD30463146FCF720FEA0
:100AF00003A238462946FEF7D9FD204601B0F0BDD5
:100B00007577625F6F70656E0D0A0000F0B581B099
:100B1000164600910446002001273946FDF730F8BB
:100B2000EFF310853D4002D1EFF3108072B627201D
:100B3000400170430A21EFF7CDFA0246002C02D0A3
:100B40000020009901E002200021FBF70BF9044688
:100B5000FBF7D2F9002D00D162B6204601B0F0BDFE
:100B6000F0B581B01D460E460446022A09D1012780
:100B700038463946FDF704F80096002238462946E3
:100B80000FE0174601200021FCF7FAFF012F04D1E6
:100B9000009600202946024603E00096022000212C
:100BA0000A462346FBF7C0F90446FBF7A5F92046A1
:100BB00001B0F0BD70B5002801D0012070BD032543
:100BC000A9020F4802680F4B535000249460012281
:100BD00053030D4E3360BFF34F8FBFF36F8F0B4E38
:100BE000336003685A50847204811020F8F734FB94
:100BF000022007A22946FEF759FD204670BDC046D7
:100C00007895010251E5CC1A80E100E080E200E035
:100C100057445420636C6F73650D0A000FB47CB5A4
:100C20000C0009AD01D0611E00E00021019100908F
:100C3000074B6A462946089800F012F9002C02D0AA
:100C4000009A002111707CBC08BC04B01847000059
:100C5000991501007CB51D4616460C0001D0611E99
:100C600000E0002101910090054B6A46294630467C
:100C700000F0F6F8002C02D0009A002111707CBD23
:100C8000991501002021020C01D010211046020A02
:100C900001D010460839020901D01046091F820808
:100CA00001D01046891E420801D0881E7047081ADC
:100CB00070470000004870470890010202E008C831
:100CC000121F08C1002AFAD170477047002001E0C6
:100CD00001C1121F002AFBD170470000F0B51FB4FC
:100CE00086B00998089A030D0021024314D0514898
:100CF000514A1818504305141198012810981AD019
:100D0000281A401C00264D4F4D4900960191049031
:100D1000002812DA444211E01198012449A3012865
:100D200001D11098C1430698119A84600360C26093
:100D300041600BB0F0BD4042E4E7044621050020CD
:100D40003F4A001C51410391029012E0E00707D096
:100D500032463B4601990098EFF75EFC0191009006
:100D600032463B4610461946EFF756FC06460F46FC
:100D70006410002CEAD10498039B0028029A099978
:100D8000089806DAEFF748FC019B009AEFF744FC5D
:100D900005E0EFF7A9FC019B009AEFF7A5FC0446DC
:100DA0000E460022284BF0F717F803D80020C04366
:100DB000014607E00022254B20463146EFF77AFB3B
:100DC000EFF7EAFF102409E0002C0ADB0A220023D7
:100DD000EFF714FE079B30321A55641E02460A4391
:100DE000F2D11122641C079B121B1C19119B012BB1
:100DF00003D0012308430ED10AE0084304D0112098
:100E000010900020119077E71098151A6D1E0BE0D6
:100E10001098824202DD00236D1C03E0824201DA59
:100E200000236D1E002BEED0069811998260C160E0
:100E300030C07EE701FCFFFF104D000000001440B1
:100E40000000F03F300000000000F0430000E03FF1
:100E500030380A2801D20120704700207047000076
:100E6000FFB597B00646002518E2252877D1002463
:100E70002746FD49049400E00443761C32780120A3
:100E8000203A90400842F7D130782A280ED002222A
:100E9000307801463039092916D804990A23594374
:100EA000303940181443761C0490F1E7189802C8B2
:100EB00004911890002904DA0120400304434842B9
:100EC000049002200443761C30782E2814D104208C
:100ED00004437078761C2A2809D11898761C80C89B
:100EE000189009E00A214F43303FC719761C30782B
:100EF000014630390929F5D930786C2810D006DC44
:100F00004C281AD068280ED06A2817D104E074281B
:100F100013D07A2812D110E00120400504430CE0E0
:100F20000121090501E0032109050C437178814283
:100F300003D1012000052418761C761C307811900E
:100F400066280BD013DC58287DD009DC00287BD024
:100F50004528F6D04628F4D047281AD1A5E118E054
:100F6000632835D0642870D0652812D19DE170289F
:100F70006CD008DC6728F1D069287BD06E280DD0B2
:100F80006F2806D1BAE073282ED0752871D0782842
:100F900059D01A9A199990476D1C7EE16002400F52
:100FA000022809D003280DD00428189801680DD014
:100FB0000D60001D189070E11898EA1701680D6027
:100FC0004A60F6E7189801680D80F2E70D70F0E7C7
:100FD00018986A4601781172001D1890002050720E
:100FE00002A80090012005E0189802C8189000207F
:100FF0000091C04361070DD5002101E00199491C12
:101000000191B94212DA8142F8DB009A515C002961
:10101000F4D10BE0002101E00199491C01918142CA
:10102000FADB019A0099895C0029F5D101990498AD
:101030001A9B471A21463846199A00F097FA0199E7
:10104000401945180BE04FE02CE113E04EE000980A
:1010500000990078491C00911A9A199990470198B3
:10106000401E0190401CF2D1214638461A9B199A25
:1010700010E137E00A200021009001916002410F49
:10108000022907D0189A01CA1892C2179446032958
:1010900008D00AE01898C01DC108C90005C91891F8
:1010A000944607E000B2C2179446042902D140B228
:1010B000C1178C4600226146944506DA0A46002193
:1010C000404291418C462D2102E0210504D52B217F
:1010D0006A461173012103E0E10701D02021F7E7FF
:1010E000029155E00A200AE0102008E0102000904C
:1010F0000021042004430191082703E00820002177
:10110000019100906002410F022907D0189A01CA8C
:10111000189200229446032908D008E01898C01DB0
:10112000C108C90005C91891944603E080B204299A
:1011300000D1C0B200210291210729D5119970294F
:1011400006D0009A1021019B4A401A4305D00EE0B8
:1011500040216A461173012108E06146014306D02F
:1011600030216A4611731199517302210291009A3C
:101170000821019B4A401A430AD16146014301D12B
:10118000610705D530216A46117301217F1E029146
:101190001199582904D035A10E910DA90D910DE09A
:1011A00037A1F9E76146019B009AEFF727FC0E9BF8
:1011B0008C469B5C0D9A521E0D9213706146014342
:1011C000F0D10D9805A9081A20300190600703D5C9
:1011D00001200004844300E001270198874201DDDB
:1011E000381A00E00020019900904118029809186F
:1011F0000498401A0490E00306D421461A9B199AD9
:10120000049800F0B3F94519002706E003A81A9ADC
:10121000C05D199990476D1C7F1C02988742F5DBD1
:10122000E0030CD521461A9B199A049800F09EF908
:10123000451904E01A9A3020199990476D1C0099BD
:10124000481E00900029F5DC08E00D980D99007803
:10125000491C0D911A9A199990476D1C0199481EC5
:1012600001900029F1DC63E10928010030313233BB
:1012700034353637383961626364656600000000D2
:1012800030313233343536373839414243444546BC
:101290000000000000F05AF94519761C307800284B
:1012A00000D0E2E528461BB0F0BD600700D4062759
:1012B0001898C01DC108C90048680A680831C30FE2
:1012C000DB071891190001D09CA108E0210501D588
:1012D0009BA104E0E10701D09AA100E09AA143009C
:1012E00011985B08109165280CD006DC452809D0C0
:1012F00046281DD0472841D141E0662818D06728EC
:101300003CD13CE00021112F01DB112000E0781CD2
:101310000191009008A911A8FFF7E0FC139905912D
:101320000021119A15927F1C12980197009150E0AC
:101330000120C00703900120019008A9009711A87F
:10134000FFF7CCFC139A149905920022119B00928E
:1013500012981593059A0192002901D0104602E0D7
:10136000791C40180190381A01D5019804E04042D8
:10137000401E0090781C0190C01B029043E0012F9A
:1013800000DA01270021112F01DD112000E038468D
:101390000191009008A911A8FFF7A0FC13990591ED
:1013A000119A0021129815920091019721070CD4EF
:1013B0000599B94201DB019900E00191012904DDA1
:1013C000159A491E515C302906D0B84201DA011D38
:1013D00005DA0121029115E00199491EEDE7002887
:1013E00005DC0099411800910199091A03E0019A5E
:1013F000411C914200DD01910099401A401C02906D
:101400000120C0070390200706D402990198814269
:1014100002DB0020C043029000206946C87707AF76
:10142000012103980337C907884224D00220119074
:101430002B201290039800280CDA404203902D20B4
:10144000129007E00A210398EEF744FE30317F1E28
:10145000039039701199481E11900029F2DC03980D
:101460000028EFD1791E12980870307820210840AA
:101470004530BF1E387006A8C01BC01D03901098D1
:101480000078002800D00120019941180298C01767
:101490000918039809180498401A401E0490E003A4
:1014A00006D421461A9B199A049800F05FF8451952
:1014B00010980078002803D01A9A199990476D1C4B
:1014C000E00324D521461A9B199A049800F04EF89F
:1014D00045191CE00098002807DB00990598884210
:1014E00003DD1598405C199901E0199930201A9A8A
:1014F000904700986D1C401C00900298401E02907E
:10150000002804D11A9A2E20199990476D1C019930
:10151000481E01900029DDDC05E038781A9A7F1C0E
:10152000199990476D1C0399481E03900029F4DC1B
:1015300021461A9B199A0498ACE600002D00000081
:101540002B0000002000000000000000F8B5044659
:1015500000251E461746880404D405E0394620209D
:10156000B0476D1C641EF9D52846F8BDFFB504468A
:10157000002581B01E46C80301D5302700E0202792
:10158000880404D505E038460399B0476D1C641EF5
:10159000F9D5284605B0F0BD4A68002A06D00A6889
:1015A000531C0B6010704868401E4860704700B5BF
:1015B0000A4683B00021009101910146012368464B
:1015C000EFF7D8FA0199009803B000BD0040404001
:1015D0004040404040404141414141404040404006
:1015E00040404040404040404040404040050202B2
:1015F0000202020202020202020202020220202071
:1016000020202020202020020202020202029090CC
:1016100090909090101010101010101010101010CA
:10162000101010101010101002020202020288881E
:10163000888888880808080808080808080808082A
:101640000808080808080808020202024000000012
:10165000CD1501001E3101008813000001000000BB
:101660000E31010088130000010000000431010068
:1016700088130000010000001831010088130000E9
:1016800001000000C63001008813000001000000C6
:10169000D430010088130000010000009C300100DC
:1016A00060EA0000030000002831010060EA000049
:1016B0000300000033310100E803000005000000D2
:1016C000B13001008813000005000000000084C153
:1016D000000008C10000C03F000038410000AC41DC
:1016E0000000D44128000400000008400800000861
:1016F0001008040810200000000000000000000096
:1017000001000000FFFFFFFF0000000000000000DC
:1017100000000000B00400000100000060090000AB
:1017200002000000C012000003000000802500003D
:1017300004000000004B00000500000000960000BF
:101740000600000000E100000700000000C20100E8
:1017500008000000008403000900000000080700E2
:101760000A00000000100E000B00000000201C000A
:101770000C00000040420F000D00000080841E009D
:1017800059062014032145012882003241003219F4
:1017900000411300390300B506002D03002D02009F
:1017A0002201002201003E01002000008009EE4DD0
:1017B0005048504F80096E4F58E5854F80096E4F55
:1017C000B867C14F5048D04FB867C14FE828DF4FC6
:1017D0008009EE4F18EAFC4F8009EE4F58E505509E
:1017E000A4550D50F0C51450A4550D500000211003
:1017F000422063308440A550C660E770088129917B
:101800004AA16BB18CC1ADD1CEE1EFF13112100222
:1018100073325222B5529442F772D66239931883CA
:101820007BB35AA3BDD39CC3FFF3DEE362244334EE
:1018300020040114E664C774A44485546AA54BB51A
:1018400028850995EEE5CFF5ACC58DD553367226C2
:1018500011163006D776F6669556B4465BB77AA76A
:1018600019973887DFF7FEE79DD7BCC7C448E5580E
:101870008668A7784008611802282338CCC9EDD9BA
:101880008EE9AFF9488969990AA92BB9F55AD44A62
:10189000B77A966A711A500A333A122AFDDBDCCB0A
:1018A000BFFB9EEB799B588B3BBB1AABA66C877C2E
:1018B000E44CC55C222C033C600C411CAEED8FFD5A
:1018C000ECCDCDDD2AAD0BBD688D499D977EB66E02
:1018D000D55EF44E133E322E511E700E9FFFBEEFAA
:1018E000DDDFFCCF1BBF3AAF599F788F8891A9816C
:1018F000CAB1EBA10CD12DC14EF16FE18010A10056
:10190000C230E3200450254046706760B983989345
:10191000FBA3DAB33DC31CD37FE35EF3B1029012A5
:10192000F322D2323542145277625672EAB5CBA511
:10193000A89589856EF54FE52CD50DC5E234C324F5
:10194000A01481046674476424540544DBA7FAB7E5
:101950009987B8975FE77EF71DC73CD7D326F23645
:101960009106B01657667676154634564CD96DC931
:101970000EF92FE9C899E9898AB9ABA94458654895
:1019800006782768C018E1088238A3287DCB5CDB85
:101990003FEB1EFBF98BD89BBBAB9ABB754A545AE5
:1019A000376A167AF10AD01AB32A923A2EFD0FED51
:1019B0006CDD4DCDAABD8BADE89DC98D267C076C35
:1019C000645C454CA23C832CE01CC10C1FEF3EFF25
:1019D0005DCF7CDF9BAFBABFD98FF89F176E367E85
:1019E000554E745E932EB23ED10EF01E303132331E
:1019F00034353637383941424344454610004000BB
:101A0000800000010002000400080010100018000F
:101A1000200030004000600080000001FFFFFFFF59
:101A200001FF01FFFF0101FFFF01000002000000B4
:101A3000010000000200000002000000020000009F
:101A4000000000001B00000000000000000000007B
:101A50000000000000000000000000000000000086
:101A6000020000000000000014000000020000005E
:101A7000070000000200000002000000000000005B
:101A8000020000000000000014000000020000003E
:101A9000010000000200000002000000020000003F
:101AA000000000001400000000000000FFFFFFFF26
:101AB000FFFFFF01FFFF01FFFF01FF01FF01FFFF2C
:101AC000FF0101FFFFFF01FF0101FFFF000100FF18
:101AD000010000FF000064009E00C800E800020151
:101AE00019012C013D014C015A01660172017D0171
:101AF000870190019901A101A901B001B701BE01BF
:101B0000C401CA01D001D601DB01E101E601EB010C
:101B1000EF01F401F801FD010102050209020D02C5
:101B20001102140218021B021F02220225022802BF
:101B30002B022E023102340237023A023D023F02EA
:101B40004202450247024A024C024F02510253022E
:101B5000560258025A025C025F0261026302650289
:101B6000670269026B026D026F02710273027502F5
:101B7000760278027A027C027E027F028102830270
:101B800084028602880289028B028C028E028F02F6
:101B90009102920294029502970298029A029B0285
:101BA0009D029E029F02A102A202A302A502A6021A
:101BB000A702A902AA02AB02AD02AE02AF02B002B6
:101BC000B102B302B402B502B602B702B902BA0258
:101BD000BB02BC0200000000000000000200000088
:101BE00004000000001003EB0000000001000000F2
:101BF00001000000040000000001003200000000AD
